:100000000C946B0A0C948C0A0C948C0A0C94E40FDC
:100010000C941E100C948C0A0C948C0A0C948C0A70
:100020000C948C0A0C948C0A0C948C0A0C948C0AF8
:100030000C948C0A0C948C0A0C948C0A0C9450131B
:100040000C948C0A0C948C0A0C948C0A0C948C0AD8
:100050000C948C0A0C94416F0C948C0A0C948C0AAE
:100060000C948C0A0C94BC6F0C948C0A0C948C0A23
:100070000C948C0A0C948C0A0C948C0A0C948C0AA8
:100080000C94AE840C948C0A0C948C0A0C948C0AFC
:100090000C94EB6F0C948C0A0C948C0A0C948C0AC4
:1000A0000C948C0A0C948C0A0C948C0A0C948C0A78
:1000B0000C948C0A0C948C0A0C948C0A0C948C0A68
:1000C0000C948C0A0C948C0A0C948C0A0C948C0A58
:1000D0000C948C0A0C948C0A0C948C0A0C948C0A48
:1000E0000C948C0A0C9487760C947D760C94917603
:1000F0000C941B760C949B760C9473760C94677618
:100100000C945B760C948C0A0C948C0A0C948C0ADC
:100110000C948C0A0C948C0A0C948C0A0C948C0A07
:100120000C948C0A0C948C0A0C948C0A0C948C0AF7
:100130000C948C0AD38AF28A618B528C728C928CCA
:100140009A8C478C084AD73B3BCE016E84BCBFFDDE
:10015000C12F3D6C74319ABD56833DDA3D00C77F97
:1001600011BED9E4BB4C3E916BAAAABE0000008030
:100170003F07634236B79BD8A71A39685618AEBAFC
:10018000AB558C1D3CB7CC5763BD6DEDFD753EF690
:10019000177231BF000000803F08000000BE9224AB
:1001A00049123EABAAAA2ABECDCCCC4C3E000000E0
:1001B00080BEABAAAAAA3E00000000BF00000080DB
:1001C0003F0000000000084178D3BB4387D1133DB6
:1001D000190E3CC3BD4282AD2B3E68EC8276BED97F
:1001E0008FE1A93E4C80EFFFBE01C4FF7F3F0000BE
:1001F000000000000C94FA7C0C944D6E0C94247852
:100200000C9480840C94A97F0C945B830C94927161
:100210000C94254F0C944C700C9417770C94431548
:100220000C94377D0C94A4700C94D47C0C94877D32
:100230000C94D9920C94516E0C94F28A0C941584FF
:100240000C9425740C94586E0C94D0700C94F75F39
:100250000C94627D0C94DE4F0C94BF730C94167357
:100260000C94478C0C9446390C9456830C94537F11
:100270000C94CE7D0C94556E0C94BB7F0C948984A9
:100280000C943C500C94720E0C94AE7F0C949D71A7
:100290000C9478740C94E9100C949A8C0C947381DF
:1002A0000C945B720C94528C0C94117E0C94618BA8
:1002B0000C9464720C94728C0C94B37F0C94FA8D31
:1002C0000C94FA830C94A47F0C94477F0C94D38AEB
:1002D0000C9431160C94168F0C94B87F0C947C1DE2
:1002E0000C94928C0C94AB7C0C945E830C94580E02
:1002F0000C94458D0C94A2756E616E00696E66005B
:1003000000407A10F35A00A0724E18090010A5D4CC
:10031000E80000E87648170000E40B54020000CA29
:100320009A3B000000E1F50500008096980000006F
:1003300040420F000000A0860100000010270000CE
:100340000000E803000000006400000000000A0054
:10035000000000000100000000002C76D888DC6757
:100360004F0823DFC1DFAE59E1B1B796E5E3E453AF
:10037000C63AE651997696E8E6C28426EB898C9BCC
:1003800062ED407C6FFCEFBC9C9F40F2BAA56FA56C
:10039000F490055A2AF75C936B6CF9676DC11BFCEE
:1003A000E0E40D47FEF520E6B500D0ED902E030009
:1003B000943577050080841E080000204E0A000056
:1003C00000C80C333333330F986E12831141EF8D15
:1003D0002114893BE65516CFFEE6DB18D1844B3855
:1003E0001BF77C1D901DA4BBE424203284725E2286
:1003F0008100C9F124ECA1E53D274E414E494E490B
:100400005459494E46CDCCCC3D0AD7233C17B7D1E1
:100410003877CC2B329595E6241FB14F0A00002087
:10042000410000C84200401C4620BCBE4CCA1B0E06
:100430005AAEC59D74256300496E76616C6964206F
:1004400069326320737065656420696E204545508C
:10045000524F4D2E2053657474696E6720313020E1
:100460006B6269742F730025730A00776474206EC1
:100470006F7420656E61626C65640A005854414C6B
:100480005F5452494D3D25640025730A0025730AC7
:10049000005465737420362025730A005465737404
:1004A00020352025730A0054657374203420257389
:1004B0000A005465737420332025730A0054657351
:1004C0007420322025730A0054657374203120256E
:1004D000730A006368616E3D25640A007478707762
:1004E000723D25640A003530306B0A003235306BBE
:1004F0000A003131356B0A0035366B0A0033386B30
:100500000A0025730A00765F6C6F773D252D332E28
:1005100032660A0025730A0073656E743D252D75D9
:10052000206475703D252D752069676E6F72656456
:100530003D252D752074746C5F7A65726F3D252D95
:10054000750A0025372E33662025372E33660025A1
:10055000352E326620004572726F72203020566F41
:100560006C74004E6F7420737570706F7274656474
:100570000A004572726F72203020566F6C7400450D
:1005800072726F72203020566F6C740062756C6BE3
:100590005F64656C61793D252D750062756C6B3DFE
:1005A000252D750056616C7565206E6F7420616C29
:1005B0006C6F7765640062756C6B3A206D61783D95
:1005C00025752073746172743D25752C20656E64E9
:1005D0003D25752C20696E5F7573653D25750A0094
:1005E0007062323D25730A007062313D25730A0046
:1005F000256C7500416C6C6F776564207370656560
:100600006420312F31302F3130302F343030206B97
:100610006269742F730025630074746C3D252D642A
:10062000200074746C3D252D6420004E6577207485
:10063000746C3D252D6420002563004D5335363103
:100640003120503D252D372E326620252D372E3274
:10065000666D0A00424D5030383520256C642043C9
:100660002000424D5030383520256C6420506120E8
:1006700020252D372E32666D00256300545F4845D6
:1006800041545F4944583D252D352E326620005493
:100690005F4445573D252D352E3266200041483DAB
:1006A000252D352E32662000545F53485432583D74
:1006B000252D352E3266200052485F53485432585B
:1006C0003D252D352E32662000545F52483D252DA4
:1006D000342E3166200052483D252D342E316620BF
:1006E0000025630025630025630025630025630062
:1006F0007265706F72745F616C6C3D007265706FD3
:1007000072743D006175746F0025630025630025D8
:100710006300256300204F534343414C3D25642033
:100720000020467573653A2065653D253032782096
:1007300068663D25303278206C663D253032782061
:100740006C623D25303278004D43553D2530366C86
:10075000780025630074785F6C656E3D252D6C759F
:100760002C765F6C6F773D252D6C752C7368743219
:10077000783D252D6C752C62756C6B3D252D6C7547
:10078000002563004F4B0A002563002563002563A5
:1007900000256300256300256300256300256300B1
:1007A00064656275675F616C6C3D00646562756766
:1007B0003D0064656275673D0025730A00646565E8
:1007C000700A006E6F6E650A00707772733D007775
:1007D00064743D25730A007062323D25730A00700F
:1007E00062313D25730A00696E74725F7365635FE1
:1007F00070313D252D372E33660A00696E74725FA5
:1008000070313D252D6C640A00696E74725F7365EA
:10081000635F70303D252D372E33660A00696E7494
:10082000725F70303D252D6C640A00765F6D6375D4
:100830003D252D352E32660A00745F6D63753D25AA
:100840002D352E32660A00707077723D25730A00CE
:1008500064656275673D0072636D643D25730A00CF
:1008600025730A006175746F0A006C6F675F6D6FA6
:1008700064653D007573625F7077723D25730A0091
:1008800072656C61793D25730A0074746C3D252D89
:10089000640A0052494D455F616464723D252D64D0
:1008A0002E252D640A006E65696768626F725F7439
:1008B00061626C655F73697A653D25640A00765FE5
:1008C0006C6F773D252D332E32660A007478707771
:1008D0003D25640A006368616E3D25640A00696411
:1008E0003D006932635F6275733D006932635F7317
:1008F000706565643D252D6C750A007478743D251E
:10090000730A0053797374656D2053756D6D617250
:10091000790A002530366C780041744D6567613284
:100920003536524652320041744D65676131323876
:10093000524652320041744D656761363452465218
:10094000320041744D6567613132385246413100A1
:100950004D43553D006D61736B3D002C00696E7415
:10096000657276616C3D252D750023252D642C0064
:10097000626F6F745F636175736500705F626D6550
:100980003238300072685F626D6532383000745FF3
:10099000626D65323830007062320070623100740E
:1009A0005F686561745F69647800745F646577008F
:1009B000616800705F6D73353631310072685F7346
:1009C0006874327800745F73687432780070610004
:1009D00070006164340061643300616432006164FA
:1009E0003100613300613200613100765F696E0071
:1009F00072680065727200757074696D650070319F
:100A00005F6C73740070315F740070310070305F20
:100A10006C73740070305F7400703000765F6D63CB
:100A20007500745F6D637500743100740069640053
:100A300065363400747874002D002B006E6F6E657F
:100A40000062756C6B00706F7765725F73617665BD
:100A50005F6C656472790072656C61795F6C656466
:100A60007900636F6D7061737300616363656C001F
:100A70007072657300705F707772006165730070EB
:100A8000315F6C6564790070305F6C65647200651D
:100A900076656E74006C6564006F7700706B74002F
:100AA00074785F6C6564790072785F6C656472005D
:100AB0006F706572006E6F6E65002530327800765B
:100AC0005F6164343D252D382E3666002000765F48
:100AD0006164333D252D382E3666002000765F6137
:100AE00064323D252D382E3666002000765F616425
:100AF000313D252D382E3666002000765F6C696703
:100B000068743D252D382E3666002000765F6132F0
:100B10003D252D372E3366002000765F61313D255F
:100B20002D372E3366002000765F696E3D252D350A
:100B30002E326600204E657665722D7573656420D1
:100B4000737461636B203E20256420627974657341
:100B50000A00757074696D653D252D642D64617999
:100B6000732D253032643A253032643A25303264B0
:100B70002D686F7572730A0074657374205B6F66FD
:100B8000667C317C327C337C347C355D20202020B7
:100B9000202020202D2074657374206D6F64657390
:100BA0000A0D007478205B706B74207061796C6F33
:100BB00061645D2020202020202020202020202D66
:100BC0002073656E6420726164696F20706B74209D
:100BD0006B6579626F6172640A0D00776474205BE3
:100BE0006F6E7C6F66667C746573745D2020202058
:100BF000202020202020202D207761746368646FDE
:100C0000670A0D00765F6C6F77205B765F6C6F779D
:100C10005D20202020202020202020202020202097
:100C20002D206C6F77657374207265706F727420FD
:100C3000766F6C746167650A0D00757067722020AD
:100C400020202020202020202020202020202020A4
:100C50002020202020202D207265626F6F74207666
:100C6000696120626F6F746C6F616465720A0D0058
:100C700075617274205B33386B7C35366B7C313137
:100C8000356B7C3235306B7C3530306B5D202D2000
:100C9000736574207465726D2F7561727420737042
:100CA0006565640A0D00626F6F742020202020208B
:100CB0002020202020202020202020202020202034
:100CC00020202D207265626F6F740A0D007077729C
:100CD00073205B646565707C6E6F6E655D2020209F
:100CE0002020202020202020202D206D63752073BF
:100CF0006C656570206D6F64650A0D0072657374B4
:100D000020656570726F6D2020202020202020201B
:100D100020202020202020202D20726573746F72E7
:100D20006520656570726F6D0A0D007070777220B6
:100D30005B6F6E7C6F66665D202020202020202067
:100D4000202020202020202D2070726F6772616D7E
:100D50006D61626C65207077720A0D0070623220DE
:100D6000205B6F6E7C6F66665D2020202020202037
:100D700020202020202020202D2070726F6772619B
:100D80006D6D61626C652070696E2062320A0D00C3
:100D900070623120205B6F6E7C6F66665D20202064
:100DA0002020202020202020202020202D2062759F
:100DB0006C6B204750494F2070696E0A0D007478A3
:100DC00074205B737472696E675D20202020202080
:100DD000202020202020202020202D20536574203A
:100DE0007265706F727420746578742073747269A0
:100DF0006E670A0D0074787077205B31352D305D99
:100E000020202020202020202020202020202020E2
:100E1000202D205458205077722E2048696768652D
:100E20007374203020283364426D290A0D007474D5
:100E30006C205B302D31355D2020202020202020AB
:100E4000202020202020202020202D2074696D6566
:100E50002D746F2D6C69766520666F7220706163EA
:100E60006B6574730A0D00737320202020202020EE
:100E70002020202020202020202020202020202072
:100E80002020202D2073797374656D2073756D6D2E
:100E90006172790A0D00727320202020202020200A
:100EA0002020202020202020202020202020202042
:100EB00020202D20726164696F2073746174730A3D
:100EC0000D007269205B236E5D205B696E745D208E
:100ED00020202020202020202020202020202D2005
:100EE0007265706F727420696E74657276616C0AD7
:100EF0000D0072636D64205B6F6E7C6F66665D20B3
:100F000020202020202020202020202020202D20D4
:100F1000616C6C6F7720636D642066726F6D206EFC
:100F200065746F726B0A0D007265205B236E5D2025
:100F30005B2B7C2D5D205B6D61736B7C6175746FC9
:100F40002C6D61736B5D202D206D6F746520726553
:100F5000706F7274207365742F6D6F646966790A9F
:100F60000D006F772020202020202020202020200E
:100F700020202020202020202020202020202D2064
:100F80006F6E652D776972652073656E736F72730E
:100F90000A0D006C6F67205B6175746F7C6F6E7CEF
:100FA0006F66665D20202020202020202020202D1C
:100FB000206D6F7465732064617461206F6E2055BD
:100FC00053420A0D006E65205B666C7573685D2088
:100FD0002020202020202020202020202020202011
:100FE000202D206E65696768626F72207461626C83
:100FF000650A0D006572722020202020202020200C
:1010000020202020202020202020202020202020E0
:101010002D206572726F722073746174730A0D00F3
:101020006D637520202020202020202020202020DB
:101030002020202020202020202020202D206D6313
:101040007520696E666F0A0D00693263205B7072ED
:101050006F62657C737065656420236E5D2020205F
:1010600020202020202D206932632070726F62655D
:10107000206275737C73657420627573207370656C
:1010800065640A0D006964205B72657365745D2098
:101090002020202020202020202020202020202050
:1010A000202D2069642068616E646C696E670A0D8A
:1010B0000068756D20202020202020202020202066
:1010C000202020202020202020202020202D2068CB
:1010D000756D69646974792073656E736F720A0D3A
:1010E0000072656C6179205B6F6E7C6F66667C73E5
:1010F000746174735D20202020202020202D207218
:10110000656C6179206E6574776F726B20726570A3
:101110006F7274730A0D006465205B6D61736B5DA3
:1011200020202020202020202020202020202020BF
:101130002020202D2064656275670A0D00636861B8
:101140006E205B31312D32365D2020202020202082
:101150002020202020202020202D206368616E2068
:1011600031312D32362028322E3430352D3234387C
:1011700030204D687A290A0D0063616C69205B5B41
:10118000765F696E7C61317C61325D20766F6C7454
:101190007C72657365747C6E6F6E655D202D206357
:1011A000616C6962726174650A0D0062756C6B2016
:1011B0005B5B73686F777C666C7573685D205B73CF
:1011C00065742074687273682064656C61795D5D14
:1011D00020202D2062756C6B696E67207061636BD7
:1011E000657473200A0D0061646320202020202094
:1011F00020202020202020202020202020202020EF
:101200002020202D2073686F7720765F696E2C2058
:1012100061312C20613220766F6C74616765730ACE
:101220000D0075202020202020202020202020209C
:1012300020202020202020202020202020202D20A1
:10124000757074696D650A0D0076202020202020BD
:10125000202020202020202020202020202020208E
:1012600020202020202D2076657273696F6E0A0D74
:101270000068202020202020202020202020202046
:10128000202020202020202020202020202D206809
:10129000656C700A0D00256300756E6B6E6F776E5E
:1012A00020636D640A00484D433538383300257398
:1012B000002573000A00202573002025362E326693
:1012C0002000253032780074656D705F6578746534
:1012D000726E3D252D362E326600202573002025A6
:1012E000362E3266204F6E2D426F617264002530BB
:1012F00032780074656D705F626F6172643D252D98
:10130000362E32660042756C6B2072656D3A207322
:10131000746172743D25752C20656E643D25752CB5
:1013200020696E5F7573653D25750A0042756C6BAB
:10133000206164643A2073746172743D25752C20B9
:10134000656E643D25752C20696E5F7573653D255E
:10135000750A0042756C6B207468726573683A2078
:1013600074696D65723D25750A00503A20256C64DC
:101370002050612020252D372E3266206D0A005224
:101380004553455454494E4720454550524F4D21F1
:10139000004932433A20004F6E6C696E650A005274
:1013A0006F7574696E6720456E61626C65640A00D2
:1013B00052504C20456E61626C65640A00257320B2
:1013C00025732C206368616E6E656C202575202C5A
:1013D00020636865636B2072617465202575204801
:1013E0007A20747820706F7765722025750A000A5C
:1013F0002A2A2A2A2A2A2A426F6F74696E672025B0
:10140000732A2A2A2A2A2A2A0A00726E67206973F6
:10141000737565732025640A00454550524F4D2071
:10142000697320636F72727570742C2072657772A5
:101430006974696E67207769746820646566617590
:101440006C74732E0A006C6F63616C686F73740048
:1014500041544D45474132353672667232000200C2
:1014600000FFFE000001452025642E256420636CEA
:101470006F636B20256C752063707520256C75205B
:101480006C706D20256C752069727120256C75203B
:10149000676C656420256C7520796C656420256C0B
:1014A0007520726C656420256C7520747820256C1D
:1014B00075206C697374656E20256C752073656E7C
:1014C000736F727320256C752073657269616C206F
:1014D000256C750A000011241FBECFEFD1E8DEBFD6
:1014E000CDBF00E00CBF1BE0A0E0B2E0E2EAFFE30A
:1014F00001E00BBF02C007900D92A037B107D9F7EA
:101500002BE3A0E7BBE001C01D92A336B207E1F7D1
:101510000E94AB6D0C94CF9F0C9400002F923F92D1
:101520004F925F926F927F928F929F92AF92BF92F3
:10153000CF92DF92EF92FF920F931F93CF93DF939F
:10154000CDB7DEB760970FB6F894DEBF0FBECDBF44
:101550007C011B016A01FC0117821682838181FFD5
:1015600044C39E012F5F3F4F3901F7019381F10181
:1015700093FD859193FF81911F01882309F431C365
:10158000853239F493FD859193FF81911F01853256
:1015900039F4B70190E00E94AB9C56016501E5CF9C
:1015A00010E0512C912CFFE1F915D8F08B3279F035
:1015B00038F4803279F08332A1F4F92DF0612EC035
:1015C0008D3261F0803369F4292D21602DC0392DD1
:1015D0003260932E892D8460982E2AC0E92DE86010
:1015E00015C097FC2DC020ED280F2A3088F496FEF8
:1015F00006C03AE0139F200D1124122F19C08AE073
:10160000589E200D1124522EE92DE0629E2E10C00E
:101610008E3231F496FCE5C2F92DF0649F2E08C09D
:101620008C3621F4292D2068922E02C0883641F490
:10163000F10193FD859193FF81911F018111B3CF3A
:101640009BEB980F933020F4992D9061805E07C03A
:101650009BE9980F933008F066C1992D9F7E96FF05
:1016600016E09F73992E853619F49064992E08C060
:10167000863621F4392F3068932E02C01111115093
:1016800097FE07C01C3350F444244394410E27E0D6
:101690000BC0183038F027E017E005C027E09CE3C6
:1016A000492E02C0212F412C560184E0A80EB11C06
:1016B000F6016081718182819381042DA3010E94D2
:1016C000229B6C01F981FC87F0FF02C0F3FF06C08A
:1016D00091FC06C092FE06C000E205C00DE203C008
:1016E0000BE201C000E08C858C7019F001115AC228
:1016F0009BC297FE10C04C0CFC85F4FF04C08A818D
:10170000813309F44A94141474F528E0241578F50B
:1017100088E0482E2CC096FC2AC0812F90E08C15C2
:101720009D059CF03CEFC3163FEFD30674F0892D66
:101730008068982E0AC0E2E0F0E0EC0FFD1FE10F98
:10174000F11D8081803319F411501111F4CF97FEEF
:101750000EC044244394410E812F90E0C816D90650
:101760002CF41C1904C04424439401C010E097FEDB
:1017700006C01C141D0434F4C601019605C085E0A2
:1017800090E002C081E090E001110196112331F058
:10179000212F30E02F5F3F4F820F931F252D30E028
:1017A0008217930714F4581A01C0512C892D89709F
:1017B00049F4552039F0B70180E290E00E94AB9CDB
:1017C0005A94F7CF002329F0B701802F90E00E94B0
:1017D000AB9C93FC09C0552039F0B70180E390E041
:1017E0000E94AB9C5A94F7CF97FE4CC04601D7FE9F
:1017F00002C0812C912CC60188199909F301E80FC8
:10180000F91FFE87ED87960124193109388B2F8740
:10181000012F10E01195019511093FEF83169306F2
:1018200029F4B7018EE290E00E94AB9CC814D90461
:101830004CF08F8598898815990524F4ED85FE85EF
:10184000818101C080E3F1E08F1A91082D853E85EA
:101850002F5F3F4F3E872D87801691062CF0B701F2
:1018600090E00E94AB9CD9CFC814D90441F49A816E
:10187000963320F4953319F43C8534FF81E3B701A6
:1018800090E04EC08A81813319F09C859F7E9C87B1
:10189000B70190E00E94AB9C111105C094FC18C0E8
:1018A00085E690E017C0B7018EE290E00E94AB9C05
:1018B0001E5F82E001E0080FF301E80FF11D808157
:1018C000B70190E00E94AB9C802F0113F3CFE6CFCD
:1018D00085E490E0B7010E94AB9CD7FC06C0C11420
:1018E000D10441F4EC85E4FF05C0D194C194D10842
:1018F0008DE201C08BE2B70190E00E94AB9C80E3D7
:101900002AE0C216D1042CF08F5FFAE0CF1AD1087A
:10191000F7CFB70190E00E94AB9CB701C601C0961B
:101920000E94AB9C54C1833631F0833779F0833504
:1019300009F056C020C0560132E0A30EB11CF601DA
:101940008081898301E010E0630112C05601F2E05A
:10195000AF0EB11CF601C080D18096FE03C0612F8E
:1019600070E002C06FEF7FEFC6010E94579C8C01B0
:10197000F92DFF7714C0560122E0A20EB11CF6012A
:10198000C080D18096FE03C0612F70E002C06FEF6F
:101990007FEFC6010E940C9C8C01F92DF0689F2EF0
:1019A000F3FD1AC0852D90E008171907A8F4B701B8
:1019B00080E290E00E94AB9C5A94F4CFF60197FC31
:1019C000859197FE81916F01B70190E00E94AB9CD9
:1019D00051105A94015011090115110579F7F7C0FA
:1019E000843611F0893661F5560197FE09C024E06E
:1019F000A20EB11CF60160817181828193810AC0BF
:101A0000F2E0AF0EB11CF60160817181072E000C6F
:101A1000880B990BF92DFF769F2E97FF09C09095A3
:101A20008095709561957F4F8F4F9F4FF0689F2EE7
:101A30002AE030E0A3010E94BF9DC82EC6183FC017
:101A4000092D853721F40F7E2AE030E01DC0097F83
:101A50008F3691F018F4883559F0C3C0803719F0EB
:101A6000883711F0BEC0006104FF09C0046007C0E0
:101A700094FE08C0066006C028E030E005C020E102
:101A800030E002C020E132E0560107FF09C084E0E7
:101A9000A80EB11CF601608171818281938108C01A
:101AA000F2E0AF0EB11CF6016081718180E090E040
:101AB000A3010E94BF9DC82EC6180F77902E96FED8
:101AC0000BC0092D0E7FC11650F494FE0AC092FC83
:101AD00008C0092D0E7E05C0DC2C092D03C0DC2CAE
:101AE00001C0D12E04FF0DC0FE01EC0DF11D80815F
:101AF000803311F4097E09C002FF06C0D394D39449
:101B000004C0802F867809F0D39403FD11C000FF34
:101B100006C01C2DD51480F4150D1D190DC0D5144B
:101B200058F4B70180E290E00E94AB9CD394F7CFC9
:101B3000D51410F45D1801C0512C04FF10C0B7017A
:101B400080E390E00E94AB9C02FF17C001FD03C040
:101B500088E790E002C088E590E0B7010CC0802FD4
:101B6000867859F001FF02C08BE201C080E207FDD8
:101B70008DE2B70190E00E94AB9CC11638F4B7012A
:101B800080E390E00E94AB9C1150F7CFCA94F30120
:101B9000EC0DF11D8081B70190E00E94AB9CC1105B
:101BA000F5CF15C0F4E0F51560F584E0581A93FE02
:101BB0001FC0011127C02C8523FF2AC008EF12E0A7
:101BC000392D3071932EF8018491811124C0552054
:101BD00009F4E4CCB70180E290E00E94AB9C5A94F7
:101BE000F6CFF7018681978126C08FEF9FEF23C044
:101BF000B70180E290E00E94AB9C5A945110F8CF5C
:101C0000D8CF512CB701802F90E00E94AB9CD3CF4E
:101C10000CEF12E0D5CF91108052B70190E00E94F6
:101C2000AB9C0F5F1F4FCFCF23E0251510F483E04F
:101C3000BDCF512CC0CF60960FB6F894DEBF0FBE5B
:101C4000CDBFDF91CF911F910F91FF90EF90DF906B
:101C5000CF90BF90AF909F908F907F906F905F904C
:101C60004F903F902F9008958115910511F00197A5
:101C7000F1F7089589EC97E09F938F930E94FB9C66
:101C80008091660290916702A0916802B09169020A
:101C90000F900F9093FF03C083EC97E002C08DEB91
:101CA00097E09F938F930E94FB9C0F900F90089555
:101CB000E091491EEF73F0E0E656F14E808380918B
:101CC000491E8F5F8093491E8091F636886080930D
:101CD000F6364CE452E061E1CA010E94167A80E0D7
:101CE00090E00895CF93DF93EC018091C914909117
:101CF000CA14A091CB14B091CC1486FF1DC08E8164
:101D00001F928F938D811F928F938C811F928F933F
:101D10008B811F928F938A811F928F9387EF92E01E
:101D20009F938F930E94E79C8DB79EB70C960FB63A
:101D3000F8949EBF0FBE8DBFBE018BEB9BE00E944F
:101D40000D7BBE0188E092E0DF91CF910C94687C1E
:101D500052985A981DBAE9E6F0E08081806280834B
:101D6000EA9A53985B98EB9A808180688083E8E6D2
:101D7000F0E08081816080830895EFEFFEE11182C1
:101D8000128210820895CF92DF92EF92FF920F930A
:101D90001F93CF93DF93EC019B018091FF1E843151
:101DA00008F0BBC08091011F64E10E94C491909330
:101DB000011FC0901C32D0901D32E0901E32F09076
:101DC0001F32092F10E08DE8989FD0011124A150F7
:101DD000B14E1396CD92DD92ED92FC92169741157D
:101DE000510559F0FA018081FD01EA57FF4F8083C8
:101DF000FA018181A957BF4F8C932097A9F089815F
:101E00009DE8909FF001919FF00D1124E150F14E5B
:101E1000DF01A657BF4F8C93E557FF4F88818F7026
:101E2000808388818F70808321153105E1F1D9018C
:101E300016964C9116975DE8509FC001519F900DEA
:101E400011248150914EFC01E757FF4F40831596B6
:101E50004C9115973197408334961B964D915D9127
:101E60006D917C911E97452F562F672F77275183B1
:101E700040837C01BEE8EB0EF11CF901238534851B
:101E800045855685A4E6B0E00E945F92672F782FC3
:101E9000892F992724E630E040E050E00E94F89135
:101EA000D7016D937C938DE8809FD001819FB00D09
:101EB0001124AA5FB04EFE0132968FE701900D9279
:101EC0008A95E1F78091011F8F5F8093011F9091A8
:101ED000FF1E9F5F9093FF1E4091C9145091CA143A
:101EE0006091CB147091CC1460FF2DC01F929F9312
:101EF0001F928F938091001F1F928F938CE293E12A
:101F00009F938F930E94FB9CEDB7FEB738960FB658
:101F1000F894FEBF0FBEEDBF16C080912C32909199
:101F20002D32A0912E32B0912F320196A11DB11DFC
:101F300080932C3290932D32A0932E32B0932F3277
:101F400080E090E002C081E090E0DF91CF911F91AE
:101F50000F91FF90EF90DF90CF9008952091FF1E9A
:101F6000222361F18091001F8F5F21502093FF1E7B
:101F700064E10E94C4919093001F4091C914509154
:101F8000CA146091CB147091CC1460FF1AC01F92D8
:101F90002F938091011F1F928F931F929F9385E033
:101FA00093E19F938F930E94FB9C8DB79EB70896F9
:101FB0000FB6F8949EBF0FBE8DBF03C080E090E0C7
:101FC000089581E090E008951F920F920FB60F924E
:101FD00011248F939F93AF93BF938091680080FFEC
:101FE00024C08091C5369091C636A091C736B09175
:101FF000C8360196A11DB11D8093C5369093C63693
:10200000A093C736B093C8368091C9149091CA1472
:10201000A091CB14B091CC1487FF07C0749882E0D4
:1020200090E09093920280939102BF91AF919F9123
:102030008F910F900FBE0F901F9018951F920F92C7
:102040000FB60F9211248F939F93AF93BF938091FC
:10205000680080FF24C08091C9369091CA36A09153
:10206000CB36B091CC360196A11DB11D8093C936F7
:102070009093CA36A093CB36B093CC368091C914D6
:102080009091CA14A091CB14B091CC1490FF07C0CA
:10209000739882E090E09093920280939102BF91B6
:1020A000AF919F918F910F900FBE0F901F90189539
:1020B00080937C0080917B00877F80937B00809160
:1020C0007C00806C80937C0085E080937A00809116
:1020D0007A00806880937A0080917B0087FFFCCF34
:1020E00080917B0085FFFCCF80917A008064809393
:1020F0007A0080917A0086FDFCCF109279001092D0
:10210000780084E090E060E070E020917A00206444
:1021100020937A0020917A0026FDFCCF2091780050
:1021200030917900620F731F019779F710927C004C
:1021300080917A008F7780937A007695679576956F
:10214000679580E090E00E94A295089580E00E944B
:1021500058102091890230918A0240918B0250914F
:102160008C020E949C9721EE3AE744E95EE30E94CC
:102170000D9408950F931F93CF93DF930FE110E019
:10218000CBE5DEE00093510182E991E00E94340E3C
:102190008091510185FD0DC00031110521F02CF019
:1021A000CB54D10903C0C4ECD9E0E2970150110926
:1021B000E9CFBE0180E090E00E94A29520E030E0EF
:1021C0004AE754E40E94F094DF91CF911F910F9160
:1021D0000895CF93DF93EC0188819981009799F05E
:1021E000803C924121F01982188283E011C0623153
:1021F00071F40E94BA106093183270931932809370
:102200001A3290931B3280EC92E19983888381E0AB
:10221000DF91CF91089580917B00886080937B004F
:1022200089EC80937C0085E080937A0080917A002D
:10223000806880937A0080917B0087FFFCCF80913B
:102240007B0085FFFCCF80917A00806480937A00C8
:1022500080917A0086FDFCCF80917A008064809323
:102260007A0080917A0086FDFCCF609178007091B1
:10227000790080917A008F7780937A0080E090E0F7
:102280000E94A29527ED33EA40E95FE30E949C9704
:1022900026E636E648E853E40E940C940895AF928F
:1022A000BF92CF92DF92EF92FF921F93CF93DF9373
:1022B000CDB7DEB729970FB6F894DEBF0FBECDBFFE
:1022C0005C011092C3148FEF898782E5E82E8EE1BE
:1022D000F82E10E06E0189E0C80ED11C8985882394
:1022E000D1F11830D1F1BE016F5F7F4FC6010E945E
:1022F000B56389858F3F11F08E3F19F48093C31425
:102300002AC0CE010196A114B10479F40E94CE63D3
:102310008093E736FE013196AFEDB6E381918D9360
:10232000EC15FD05D9F781E019C00E94CE63F701D5
:102330008087FE01319680E090E02191D701A80FBF
:10234000B91F2C93019688309105B9F71F5FF9E00A
:10235000EF0EF11CC3CF812F01C088E029960FB684
:10236000F894DEBF0FBECDBFDF91CF911F91FF90DC
:10237000EF90DF90CF90BF90AF9008952F923F9253
:102380004F925F926F927F928F929F92AF92BF9285
:10239000CF92DF92EF92FF920F931F93CF93DF9331
:1023A000EC015B01009711F427E003C0019749F4A9
:1023B00026E04AE250E06BE270E089E290E00E94A1
:1023C0009562CE010E944F119E012C533B4E690134
:1023D000F9018083CD2B69F0C2E5DEE1E12CF12C1F
:1023E00096EB292E92E1392E24EB822E22E1922EB9
:1023F000C2C08FED96E30E945B64BC01990F880B0D
:10240000990B0E94A4956B017C01AB2801F120E09F
:1024100030E048EC52E40E94F0949F938F937F93B6
:102420006F9383EF92E19F938F930E94FB9C84EBC9
:1024300092E19F938F930E94FB9C2DB73EB7285F3C
:102440003F4F0FB6F8943EBF0FBE2DBFCBC0CFEDB0
:10245000D6E387EEA82E86E3B82E0EEE12E1899120
:102460001F928F931F930F930E94FB9C0F900F90CE
:102470000F900F90AC16BD0691F720E030E048ECCD
:1024800052E4C701B6010E94F0949F938F937F930B
:102490006F938EED92E19F938F930E94FB9C0F9020
:1024A0000F900F900F900F900F908091E736811151
:1024B00003C088EA93E002C086E293E09F938F9383
:1024C0008AED92E19F938F930E94FB9C84EB92E1B3
:1024D0009F938F930E94FB9C0F900F900F900F90F3
:1024E0000F900F907FC000E010E0FE01E00FF11FA1
:1024F00080811F928F93E2ECF2E1FF93EF930E94B1
:10250000FB9C0F5F1F4F0F900F900F900F900830A4
:10251000110559F720E030E048EC52E4C301B20164
:102520000E94F0949F938F937F936F938AEB92E135
:102530009F938F930E94FB9C0F900F900F900F9092
:102540000F900F90888581114AC088EA93E09F938D
:102550008F933F922F920E94FB9C9F928F920E949A
:10256000FB9CFFEFEF1AFF0A29960F900F900F9038
:102570000F900F900F90F601808190E0E816F90619
:102580008CF5CE010E945B64BC01990F880B990BFE
:102590000E94A4952B013C01A114B10409F4A3CF1E
:1025A00020E030E048EC52E40E94F0949F938F9337
:1025B0007F936F9387EC92E19F938F930E94FB9C94
:1025C00084EB92E19F938F930E94FB9C8DB79EB703
:1025D00008960FB6F8949EBF0FBE8DBF03C086E26B
:1025E00093E0B5CFDF91CF911F910F91FF90EF90C6
:1025F000DF90CF90BF90AF909F908F907F906F9023
:102600005F904F903F902F900895CF93DF931F924C
:102610001F92CDB7DEB7EFEDF6E381818983878125
:102620008A83CE0101960E945A810F900F90DF910C
:10263000CF910895CF93DF93EC012091DF36309155
:10264000E0364091E1365091E2366091E336709188
:10265000E4368091E5369091E636AFEF0E94009423
:10266000E1F427E04AE250E06BE270E089E290E0BA
:102670000E94956280E090E00E944F11CC53DB4EA7
:10268000888349E050E06EE070E08FED96E30E94B1
:10269000B29FDF91CF910C940513DF91CF910895F4
:1026A0001F920F920FB60F9211240BB60F92FF924A
:1026B0000F931F932F933F934F935F936F937F934A
:1026C0008F939F93AF93BF93CF93DF93EF93FF933A
:1026D0008091F63682608093F6368091660286FDA0
:1026E0002B9A8091660287FD2B9A8091910290919E
:1026F00092021816190614F4749A739A8091C914E8
:102700009091CA14A091CB14B091CC1485FF02C053
:1027100074987398809106029091070201979093A4
:10272000070280930602892B09F073C180917E0B0A
:1027300090917F0B019690937F0B80937E0B8091FD
:102740001C3290911D32A0911E32B0911F32019621
:10275000A11DB11D80931C3290931D32A0931E3297
:10276000B0931F3280E190E09093070280930602BD
:102770008091660280FD02C01D9B05C01092C814A6
:102780001092C71406C081E090E09093C814809323
:10279000C7148091C9149091CA14A091CB14B09120
:1027A000CC1497FF08C08091C7149091C814892B4E
:1027B00049F0749A739809EF1DE1C1E3D2E3FF2455
:1027C000F39441C0739A7498F6CF80917E0B9091E8
:1027D0007F0B0196BF010E94D091892BE1F5D801B2
:1027E00012964C91417020E030E050E060E070E0E3
:1027F00080E090E0A0E00E94009469F177988091D9
:10280000C9149091CA14A091CB14B091CC1492FF2A
:1028100005C074981092920210929102F80160859E
:10282000718561157105C1F4D80118966D917C917F
:1028300019976115710511F5065F1F4F2596B2E3D3
:10284000C534DB0779F1D8011896ED91FC91199701
:10285000309721F3BACFBF0180917E0B90917F0B0F
:1028600001960E94D091892BF9F61C821B82AE0141
:1028700062E184E292E00E94167AD6CF80917E0BCC
:1028800090917F0B0E94D091892BB1F6F8821A8328
:1028900009831C821B82AE0162E182E492E00E9405
:1028A000167ACACF60916C0270916D026115710544
:1028B000A1F180917E0B90917F0B0E94D091892B8A
:1028C00061F58091C5369091C636A091C736B0911A
:1028D000C83640910E2A50910F2A6091102A7091AB
:1028E000112A841B950BA60BB70B8093211E909386
:1028F000221EA093231EB093241E8091C536909172
:10290000C636A091C736B091C83680930E2A9093F0
:102910000F2AA093102AB093112A60916A02709135
:102920006B0261157105A1F180917E0B90917F0B77
:102930000E94D091892B61F58091C9369091CA3659
:10294000A091CB36B091CC364091122A5091132AE7
:102950006091142A7091152A841B950BA60BB70B56
:102960008093251E9093261EA093271EB093281EA9
:102970008091C9369091CA36A091CB36B091CC36B1
:102980008093122A9093132AA093142AB093152AA5
:10299000E091980AF091990A80E090E01995892BCE
:1029A000D9F481E08093313289EF9DE19093333205
:1029B000809332321092353210923432749882E021
:1029C00090E0909392028093910241E352E362E19E
:1029D00082E492E00E94167A8091660286FD2B982E
:1029E0008091660290916702A0916802B09169029D
:1029F00091FF0FC00E9454738A3119F0C1E0C80FD3
:102A000001C0CBE00E9492718C2F0E9465730E94DE
:102A10005B7240E050E060E089EB92E00E94167A41
:102A2000FF91EF91DF91CF91BF91AF919F918F91E6
:102A30007F916F915F914F913F912F911F910F91D6
:102A4000FF900F900BBE0F900FBE0F901F90189528
:102A50008091491E90913032891B08950E9428155B
:102A6000882371F0E0913032EF73F0E0E656F14EDA
:102A7000808190E0209130322F5F20933032089592
:102A80008FEF9FEF0895CF93DF93EC011092AF0B80
:102A90001092AE0B888199810097C1F08C3F9340D2
:102AA00021F01982188283E0B8C0613109F0B4C006
:102AB0000E942E1599279093AA0B8093A90B8D3015
:102AC000910509F444C08F3F910549F40E942815EF
:102AD0008111EECF8CEF93E0998388839DC0823182
:102AE000910509F45AC08F37910509F052C08091C1
:102AF000A70B9091A80B181619060CF560915D3B79
:102B000070915E3B88E090E00E94AB9C60915D3BE1
:102B100070915E3B80E290E00E94AB9C60915D3BD7
:102B200070915E3B88E090E00E94AB9C8091A70B87
:102B30009091A80B01979093A80B8093A70B80917D
:102B4000A70B9091A80B8F37910509F0BFCF10927A
:102B500030321092491E8091A70B9091A80BFC0176
:102B6000EB5BFD4C10829093AF0B8093AE0B1092F9
:102B7000A80B1092A70B8091E8369091E936009748
:102B800009F4A4CF40E050E06091C1140E94167A8D
:102B90009DCF8830910571F5AACF60915D3B709112
:102BA0005E3B8DE090E00E94AB9C1092A60B1092D1
:102BB000A50B8091A50B9091A60B2091A70B3091AE
:102BC000A80B821793070CF0BACFFC01EB5BFD4C0E
:102BD000808160915D3B70915E3B90E00E94AB9C78
:102BE0008091A50B9091A60B01969093A60B8093D4
:102BF000A50BDFCF60915D3B70915E3B0E94AB9C6B
:102C00008091A70B9091A80B2091A90BFC01EB5B85
:102C1000FD4C208301968FCF81E0DF91CF91089505
:102C20008091C7149091C814892BD1F080916602CD
:102C300090916702A0916802B091690293FD10C063
:102C40000E94927183B7817F866083BFF89483B7B7
:102C5000816083BF7894889583B78E7F83BF789493
:102C60000895CF93DF93FC01208131812115310537
:102C700051F0273F324129F0FC011182108283E09C
:102C800015C0653891F4EC010E9492700E941016F4
:102C900040E050E065E880913316909134160E9430
:102CA000167A87EF92E19983888381E0DF91CF9153
:102CB0000895CF93DF93EB01892B61F05F934F93DE
:102CC00081EB92E19F938F930E94FB9C0F900F905A
:102CD0000F900F90DF93CF938EEA92E19F938F93A3
:102CE0000E94FB9C0F900F900F900F90DF91CF915F
:102CF0000895CF93DF93D62FC42F0E941E658D2F8A
:102D00000E944F658C2F0E944F65DF91CF910C94EC
:102D10004765CF92DF92EF92FF920F931F93CF936D
:102D2000DF93C82FD62FF42E152F022F0E941E6579
:102D30008D2F0E944F658C2F81600E944565CF2D9D
:102D4000D12F10E0E12CF12C680181E0C81AD108E4
:102D5000E016F10671F0CE14DF0419F40E946A65E2
:102D600002C00E94606588838FEFE81AF80A2196F6
:102D7000EFCFDF91CF911F910F91FF90EF90DF90F8
:102D8000CF900C944765CF92DF92EF92FF920F9312
:102D90001F93CF93DF931F92CDB7DEB70E9492703F
:102DA00080EB0E94EA6481111CC00E9447658091FB
:102DB000162E9091172E81609093172E8093162EC9
:102DC0008FE293E09F938F938EEA92E19F938F938C
:102DD0000E94FB9C0F900F900F900F9001E010E06D
:102DE00002C000E010E08EB18470F82E729A64E2A6
:102DF00078E680E090E00E94C7640E9492708EE4C2
:102E00000E94EA64811117C00E9447658091162EC6
:102E10009091172E82609093172E8093162E680142
:102E20008FEFC81AD80A47EE59E067E373E0C8018C
:102E30000E9459168601F11001C0729864E278E68A
:102E400080E090E00E94C7640E9492708EEE0E9423
:102E5000EA64811159C019820E94476521E030E07F
:102E6000AE014F5F5F4F60ED70E08EEE90E00E942C
:102E7000891689818535A9F48091162E9091172E97
:102E800084609093172E8093162E78018FEFE81AA6
:102E9000F80A47EE59E06FE373E0C8010E94591643
:102EA000870189818835A9F48091162E9091172E7B
:102EB00080619093172E8093162E78018FEFE81A79
:102EC000F80A47EE59E066E473E0C8010E9459161B
:102ED000870189818036C1F48091162E9091172E3A
:102EE00080629093172E8093162E78018FEFE81A48
:102EF000F80A47EE59E06DE473E0C8010E945916E4
:102F000081E00E945468870164E278E680E090E006
:102F10000E94C7640E94927086EA0E94EA6481114E
:102F200017C00E9447658091162E9091172E8064DD
:102F30009093172E8093162E78018FEFE81AF80AD7
:102F400047EE59E064E573E0C8010E945916870115
:102F500064E278E680E090E00E94C7640E9492708C
:102F60008CE30E94EA6481111FC00E944765809132
:102F7000162E9091172E80689093172E8093162E00
:102F800078018FEFE81AF80A47EE59E06CE573E034
:102F9000C8010E94591686EA92E19F938F930E947E
:102FA000FB9C0F900F90870164E278E680E090E050
:102FB0000E94C7640E94927082ED0E94EA648111AF
:102FC00017C00E9447658091162E9091172E916030
:102FD0009093172E8093162E78018FEFE81AF80A37
:102FE00047EE59E064E673E0C8010E945916870174
:102FF00064E278E680E090E00E94C7640E949270EC
:1030000080E80E94EA64811117C00E9447658091A0
:10301000162E9091172E98609093172E8093162E4F
:1030200078018FEFE81AF80A47EE59E06DE673E091
:10303000C8010E945916870164E278E680E090E0BA
:103040000E94C7640E94927080ED0E94EA64811120
:1030500017C00E9447658091162E9091172E94609C
:103060009093172E8093162E78018FEFE81AF80AA6
:1030700047EE59E063E773E0C8010E9459168701E3
:1030800064E278E680E090E00E94C7640E9492705B
:103090008CEE0E94EA64811117C00E9447658091FE
:1030A000162E9091172E90619093172E8093162EC6
:1030B00078018FEFE81AF80A47EE59E06BE773E002
:1030C000C8010E945916870187E0E82EF12C64E2BE
:1030D00078E680E090E00E94C7640E9492708CE7DE
:1030E0000E94EA64811113C00E9447658091162EE8
:1030F0009091172E92609093172E8093162E47EE84
:1031000059E062E873E0C8010E94591604C081E0EA
:10311000E81AF108E1F60E94476584EB92E19F937B
:103120008F930E94FB9C0F900F900F90DF91CF9197
:103130001F910F91FF90EF90DF90CF900895AF9285
:10314000BF92CF92DF92EF92FF920F931F93CF9394
:10315000DF93CDB7DEB760970FB6F894DEBF0FBE32
:10316000CDBFF82EE42E6623E9F18E010F5F1F4FCD
:1031700080E1F80111928A95E9F728E0A80168E951
:1031800080EB0E948916FF2041F08BE893E09F932B
:103190008F930E94E79C0F900F905E01F8E0AF0EB6
:1031A000B11C92E9C92E93E0D92EF80181918F01CB
:1031B0001F928F93DF92CF920E94E79C0F900F9007
:1031C0000F900F900A151B0581F788851F928F932A
:1031D00087EE93E09F938F930E94E79C0F900F9050
:1031E0000F900F90EE20E9F18E010F5F1F4F80E1ED
:1031F000F80111928A95E9F720E1A80160E880EBD7
:103200000E948916FF2041F087E993E09F938F93F6
:103210000E94E79C0F900F906E01F0E1CF0ED11C41
:1032200082E9E82E83E0F82EF80181918F011F9248
:103230008F93FF92EF920E94E79C0F900F900F9058
:103240000F90C016D10681F788891F928F9387EE61
:1032500093E09F938F930E94E79C0F900F900F90A5
:103260000F9060960FB6F894DEBF0FBECDBFDF9112
:10327000CF911F910F91FF90EF90DF90CF90BF9073
:10328000AF9008950F931F93CF93DF931F921F92D8
:10329000CDB7DEB71A82198222E0AE014F5F5F4FD1
:1032A0006AEA8EEE0E9489160AED1EE189819A81F2
:1032B000982789279827F8019183808322E0AE011F
:1032C0004F5F5F4F6CEA8EEE0E94891689819A816A
:1032D000982789279827F8019383828322E0AE01FB
:1032E0004F5F5F4F6EEA8EEE0E94891689819A8148
:1032F000982789279827F8019583848322E0AE01D7
:103300004F5F5F4F60EB8EEE0E94891689819A8134
:10331000982789279827F801938B828B22E0AE01AA
:103320004F5F5F4F62EB8EEE0E94891689819A8112
:10333000982789279827F801958B848B22E0AE0186
:103340004F5F5F4F64EB8EEE0E94891689819A81F0
:10335000982789279827F801978B868B22E0AE0162
:103360004F5F5F4F66EB8EEE0E94891689819A81CE
:10337000982789279827F8019783868322E0AE0152
:103380004F5F5F4F68EB8EEE0E94891689819A81AC
:10339000982789279827F8019187808722E0AE0136
:1033A0004F5F5F4F6AEB8EEE0E94891689819A818A
:1033B000982789279827F8019587848722E0AE010E
:1033C0004F5F5F4F6CEB8EEE0E94891689819A8168
:1033D000982789279827F8019787868722E0AE01EA
:1033E0004F5F5F4F6EEB8EEE0E94891689819A8146
:1033F000982789279827F801918B808B0F900F9041
:10340000DF91CF911F910F9108952F923F924F928C
:103410005F926F927F928F929F92AF92BF92CF9264
:10342000DF92EF92FF920F931F93CF93DF93CDB76D
:10343000DEB769970FB6F894DEBF0FBECDBF182F69
:10344000D62E042F2F8B9E012F5F3F4F790183E0F3
:10345000F90111928A95E9F78091FE1E811105C04C
:103460000E94421981E08093FE1EDD2009F46DC0A8
:103470004EE264EF8EEE0E94791662E174E380E022
:1034800090E00E94C76422E0A70166EF8EEE0E94E2
:10349000891629813A81322723273227A90160E042
:1034A00070E08091F01E9091F11E9A01AB01281BF3
:1034B000390B41095109A091EE1EB091EF1E0E94F7
:1034C0005F926B017C013FE0F594E794D794C79439
:1034D0003A95D1F76091E81E7091E91ECB01770F04
:1034E000AA0BBB0BBC01CD014BE0660F771F881FF9
:1034F000991F4A95D1F72091EA1E3091EB1E4901A0
:10350000330FAA08BB08A50194012C0D3D1D4E1DCB
:103510005F1D0E941A92C20ED31ED092E51EC09269
:10352000E41EF8E0CF0ED11C54E0D594C7945A9510
:10353000E1F70D2C000CEE08FF08C092F21ED092AD
:10354000F31EE092F41EF092F51E812F8295880FF3
:10355000880F807C8C5C8A87212F30E03987288710
:10356000A3E0B0E0012E02C0AA0FBB1F0A94E2F74D
:103570002AE63AE00E9458929B01AC012E5F3F4F31
:103580004F4F5F4F2B873C874D875E8780E593ECDD
:10359000A0E0B0E09C01AD0104C05595479537957A
:1035A00027951A95D2F72B8B3C8B4D8B5E8B10E0B9
:1035B000412C512C320188E090E0AC01E885F9857E
:1035C0004E1B5F0B598F488F101709F439C14A857C
:1035D00064EF8EEE0E9479166B857C858D859E85C5
:1035E0000E94C76423E0AE014F5F5F4F66EF8EEE2F
:1035F0000E9489162090E41E3090E51EF0EA2F1AF2
:10360000FFE03F0A9101D1010E9441926C837D83CA
:103610008E839F83E091DC1EF091DD1EF88BEF8797
:10362000E091DA1EF091DB1EFA8BE98BE091DE1E51
:10363000F091DF1EA091E01EB091E11E9B01AC0154
:103640008CE055954795379527958A95D1F70E9437
:103650006A926C01FF24D7FCF094EF2C9101DF01FA
:103660000E944192DC01CB013DE0B595A79597956D
:1036700087953A95D1F78C0D9D1DAE1DBF1D029605
:10368000A11DB11D42E0B595A795979587954A95DF
:10369000D1F79C01AD0130584F4F5F4FA091EC1E08
:1036A000B091ED1E0E945F924B015C015FE0B69409
:1036B000A794979487945A95D1F78981CA80D12C81
:1036C000E12CF12CFE2CED2CDC2CCC24E82A8B8177
:1036D000C82A088C04C0F594E794D794C7940A9438
:1036E000D2F7A091E21EB091E31E2C813D814E8164
:1036F0005F810E946A929B01AC0177E155954795E5
:10370000379527957A95D1F72C833D834E835F8338
:103710009101AF85B8890E944192DC01CB01EBE0B9
:10372000B595A79597958795EA95D1F72C813D8119
:103730004E815F81820F931FA41FB51FE989FA890B
:10374000AF01FF0F660B770BF2E0440F551F661FAA
:10375000771FFA95D1F7840F951FA61FB71F08840E
:1037600004C0880F991FAA1FBB1F0A94D2F70296A4
:10377000A11DB11D22E0B595A795979587952A952E
:10378000D1F7A7019601281B390B4A0B5B0B6B89FC
:103790007C898D899E890E94B49197FD0BC0660F2C
:1037A000771F881F991FA50194010E94F891490174
:1037B0005A010AC0A50194010E94F89149015A01D9
:1037C000880C991CAA1CBB1C9927B7FC9A958B2DB9
:1037D0007A2D692D9B01AC010E94B4919B01AC0133
:1037E000AEEDBBE00E945F926B017C01A3E4B3EEFF
:1037F000A50194010E946D92BB2797FDB095AB2F58
:103800006701FF24D7FCF094EF2CC80ED91EEA1EE6
:10381000FB1EFFECCF0EFEE0DF1EE11CF11C44E0BE
:10382000F594E794D794C7944A95D1F78C0C9D1CD6
:10383000AE1CBF1C480C591C6A1C7B1C1F5FC4CEED
:10384000112381F0212F30E040E050E0C301B201AC
:103850000E94F8912093F61E3093F71E4093F81EB5
:103860005093F91E2F89222389F16091F61E7091E1
:10387000F71E8091F81E9091F91E61157105810562
:10388000910521F10E94A49520E836EE45EC57E41D
:103890000E94F09421E03EED42E45EE30E9409982C
:1038A0009B01AC0160E070E080E89FE30E940C9413
:1038B0002BE43AE34DEB57E30E94F0946093FA1E39
:1038C0007093FB1E8093FC1E9093FD1E69960FB6AD
:1038D000F894DEBF0FBECDBFDF91CF911F910F9146
:1038E000FF90EF90DF90CF90BF90AF909F908F9020
:1038F0007F906F905F904F903F902F9008950F931F
:103900001F93CF93DF9300D000D0CDB7DEB78E01E9
:103910000F5F1F4F86E0F80111928A95E9F78091B9
:10392000F01D811113C040E061E386EA0E94791620
:103930004AE06CE286EA0E94791681E08093F01DED
:1039400068EF7CE780E090E00E94C76448E06DE2A9
:1039500086EA0E94791668EF7CE780E090E00E949A
:10396000C76426E0A80162E386EA0E94891647E060
:103970006DE286EA0E94791689819A818093EA1D18
:103980009093EB1D2B813C812093EC1D3093ED1D1A
:103990004D815E814093EE1D5093EF1D5F934F93D9
:1039A0003F932F939F938F938BE993E09F938F93F4
:1039B0000E94E79C0FB6F894DEBF0FBECDBF2696DF
:1039C0000FB6F894DEBF0FBECDBFDF91CF911F9130
:1039D0000F9108958F929F92AF92BF92CF92DF92F4
:1039E000EF92FF920F931F93CF93DF9300D000D0FD
:1039F000CDB7DEB78E010F5F1F4F86E0F801119241
:103A00008A95E9F741E062E08CE30E94791648E587
:103A100060E08CE30E94791664E278E680E090E052
:103A20000E94C76426E0A80163E08CE30E94891627
:103A300043E062E08CE30E94791609811A81102725
:103A400001271027EAECFDE111830083EB80FC8065
:103A5000FE24EF24FE24F382E282CD80DE80DC248B
:103A6000CD24DC24D582C482B801012E000C880B41
:103A7000990B0E94A4954B015C01B7010F2C000C1F
:103A8000880B990B0E94A495A50194010E948C9427
:103A900020EE3EE245E652E40E949C9720E030E0B2
:103AA00044E353E40E940D949F938F937F936F930D
:103AB000DF92CF92FF92EF921F930F9389EA93E0E8
:103AC0009F938F930E94E79C0FB6F894DEBF0FBEC2
:103AD000CDBF26960FB6F894DEBF0FBECDBFDF91E7
:103AE000CF911F910F91FF90EF90DF90CF90BF90FB
:103AF000AF909F908F900895CF93DF93EC018881D2
:103B000099810097A9F18C3D924121F01982188288
:103B100083E083C08CE89BE00E94E777892BA1F1CA
:103B20008091C9149091CA14A091CB14B091CC1477
:103B300093FD2CC08091C9149091CA14A091CB140C
:103B4000B091CC1493FD53C08091C9149091CA14C4
:103B5000A091CB14B091CC1494FD51C08091C914A4
:103B60009091CA14A091CB14B091CC1495FD4EC085
:103B700040E850E060E070E08CE89BE00E94C9778C
:103B80008CED92E19983888381E047C08091162E65
:103B900082FFD0CF21E048E061E083E00E94051A77
:103BA0008091FD1E8F938091FC1E8F938091FB1E50
:103BB0008F938091FA1E8F938091F91E8F9380913D
:103BC000F81E8F938091F71E8F938091F61E8F932E
:103BD0008AE693E19F938F930E94FB9C8DB79EB7DB
:103BE0000A960FB6F8949EBF0FBE8DBFA3CF8091EB
:103BF000162E85FFA9CF81E00E944A69A5CF80914A
:103C0000162E86FFABCF0E947F1CA8CF8091162E68
:103C100087FFAECF0E94EA1CABCFDF91CF91089512
:103C2000CF93DF93C82F8CEE0E9445658C2F0E94A6
:103C30004F656AE67AE080E090E00E94C7648DEE0E
:103C40000E9445650E946065D82F0E946A65C82F52
:103C50000E9447658C2F90E09D2BDF91CF910895B6
:103C60001F93CF93DF93C82F8CEE0E9445658C2F56
:103C70000E944F6564E278E680E090E00E94C764AD
:103C80008CEE0E94456580E00E944F656AE67AE00E
:103C900080E090E00E94C7648DEE0E9445650E941E
:103CA0006065182F0E946065C82F0E946A65D82F32
:103CB0000E9447658C2F90E0A0E0B0E0BA2FA92FBA
:103CC000982F8827A12BBC01CD016D2BDF91CF91BF
:103CD0001F9108952F923F924F925F926F927F9221
:103CE0008F929F92AF92BF92CF92DF92EF92FF920C
:103CF0000F931F93CF93DF93CDB7DEB7CE54D10987
:103D00000FB6F894DEBF0FBECDBF80910402909134
:103D10000502892BE1F110920502109204028CEE4B
:103D20000E9445658EE10E944F650E94476566E3EB
:103D30007CE980E090E00E94C76482EA0E94101E45
:103D400090937D0B80937C0B84EA0E94101E9093CD
:103D50007B0B80937A0B86EA0E94101E9093790B5E
:103D60008093780B88EA0E94101E9093770B8093C3
:103D7000760B8AEA0E94101E9093750B8093740B49
:103D80008CEA0E94101E9093730B8093720B88E450
:103D90000E94301E6AAF7BAF8CAF9DAF88E50E945A
:103DA000301E2091740B3091750B4B015C01A90101
:103DB00060E070E080E090E0DC0127962FAF27976D
:103DC00028965FAF289729966FAF29972A967FAFDD
:103DD0002A972B968FAF2B972C969FAF2C972D96CB
:103DE000AFAF2D972E96BFAF2E97AB0160E070E07E
:103DF00080E090E008E00E94A2932A833983B42FE8
:103E0000A52FF62FE72F8C019401A50160E070E04B
:103E100080E090E0AA80B980CB2EDA2EEF2EFE2E25
:103E20000E94EE9329014A016DA37CA389839A83A2
:103E3000315041095F4F6F4F7F4F8F4F9F4F662427
:103E40006394712C21153F4F4F4F5140610571050F
:103E50008105910509F010F4612C712C130140913A
:103E6000720B5091730B52016401EDA0FCA009810B
:103E70001A819A0140E050E060E070E080E090E05C
:103E80000E947292F22E032F142FB52FF62FE72FD8
:103E9000D82EE92EA0E00E94009484F4215031092C
:103EA00040485F4F6F4F7F4F8F4F9F4FF22E032F32
:103EB000142FB52FF62FE72FD82EE92E2F2D302FC8
:103EC000412F5B2F6F2F7E2F8D2D9E2D07E10E949E
:103ED000BB932C8F3D8F4E8F5F8F68A379A38AA3EE
:103EE0009BA32053384F4F4F5F4F6F4F7F4F8F4FE4
:103EF0009F4F2C8B3D8B4E8B5F8B688F798F8A8F7A
:103F00009B8F2056304F4F4F5F4F6F4F7F4F8F4FDC
:103F10009F4F243D304341055105610571058105E1
:103F2000910529F020F01301EFEF2E1A3E0A40917F
:103F3000760B5091770B52016401EDA0FCA0098132
:103F40001A819A0140E050E060E070E080E090E08B
:103F50000E947292F22E032F142FB52FF62FE72F07
:103F6000D82EE92EA0E00E9400945CF4AFE70E94F6
:103F7000E293F22E032F142FB52FF62FE72FD82E12
:103F8000E92E2F2D302F412F5B2F6F2F7E2F8D2D60
:103F90009E2D07E00E94BB932B833C833A01B62FF2
:103FA000A72FF82FE92FA0907A0BB0907B0B9501EB
:103FB00040E050E060E070E080E090E000E10E94CE
:103FC000A29359016A017B018C012B813C81A301E1
:103FD0006B2F7A2F8F2F9E2F0E94D9932B833C8398
:103FE00049875A876B877C878D879E872E5F3F4FD7
:103FF000434051096E4F7F4F8F4F9F4F2230310505
:10400000494F5F4F644071058105910521F018F01B
:104010002FEF221A320A40917C0B50917D0B5E8368
:104020004D834091780B5091790B52016401EDA0C2
:10403000FCA009811A819A0140E050E060E070E044
:1040400080E090E00E947292F22E032F142FB52F81
:10405000F62FE72FD82EE92EA0E00E94009484F4DA
:1040600021503F4F4F4F5F4F6F4F7F4F8F4F9F4FAD
:10407000F22E032F142FB52FF62FE72FD82EE92E6F
:104080002F2D302F412F5B2F6F2F7E2F8D2D9E2DAB
:1040900008E00E94BB932F8338873A01B62FA72FE1
:1040A000F82FE92F6D817E81C12CD12C9B01A601B7
:1040B00060E070E080E090E00FE00E94A293590180
:1040C0006A017B018C012F813885A3016B2F7A2F28
:1040D0008F2F9E2F0E94D9932D833F8348875F8720
:1040E000688B798B8A8B9B8B2F5F3F4F41405109A7
:1040F0006F4F7F4F8F4F9F4F213030484C4F5F475E
:10410000624071058105910521F018F0BFEF2B1A6F
:104110003B0A2C893D894E895F89688D798D8A8D0E
:104120009B8D2F3C37404105510561057105810587
:10413000910511F00CF0D3C152016401EDA0FCA077
:1041400009811A819201A401B701C8010E947292EB
:10415000122F3A834983B52FF62FE72FF82E092F18
:10416000A0E00E94009484F4215031094109504894
:104170006F4F7F4F8F4F9F4F122F3A834983B52F39
:10418000F62FE72FF82E092F212F3A8149815B2F37
:104190006F2F7E2F8F2D902F0FE10E94BB932EAF9C
:1041A0003FAF21964FAF219722965FAF229723967C
:1041B0006FAF239724967FAF249725968FAF2597CF
:1041C00026969FAF269745E0A42EB12CC12CD12C6A
:1041D000E12CF12C00E010E02C8D3D8D4E8D5F8D9B
:1041E00068A179A18AA19BA10E947292AC8CBD8C1E
:1041F000CE8CDF8CE8A0F9A00AA11BA10E947292CC
:10420000122F3BAB4AABB52FF62FE72F7C01922E36
:10421000A32EB42EC52ED62E072F782E8F2CA0E0DD
:104220000E9400945CF4A1E00E94E293922EA32EDF
:10423000B42EC52ED62E072F782E892E292D3A2D55
:104240004B2D5C2D6D2D702F872D982D01E00E9438
:10425000BB932AA73BA74CA75DA76EA77FA788ABF8
:1042600099AB29833A834CA35DA36EA37FA388A750
:1042700099A7212F3BA94AA95B2F6F2F7E2FC7013A
:10428000A0E00E94009454F4A3E00E94E293122F55
:104290003BAB4AABB52FF62FE72F7C01212F3BA973
:1042A0004AA95B2F6F2F7E2FC70102E00E94BB93AC
:1042B0002AAB3BAB4CAB5DAB6EAB7FAB88AF99AF82
:1042C0002F962FAF2F9727963FAF2797B42FA52F65
:1042D000F62FE72F4C012C893D894E895F89688D27
:1042E000798D8A8D9B8D24323A4F4F4F5F4F6F4FA0
:1042F0007F4F8F4F9F4F0CF088C02C8D3D8D4E8D82
:104300005F8D68A179A18AA19BA12455324F4F4F9F
:104310005F4F6F4F7F4F8F4F9F4F29013A014B01E6
:104320008D8F9C8F27E0A22EB12CC12CD12CE12C9B
:10433000F12C00E010E092010E94729252016301A0
:1043400074010D8D1C8D0E947292AAA4BBA4CCA4F2
:10435000DDA4EEA4FFA408A919A90E94D99329837A
:104360003A834CA35DA36EA37FA388A799A73BE0E4
:10437000A32EB12CC12CD12CE12CF12C00E010E0AB
:104380009201A301B4018D8D9C8D0E947292520105
:10439000630174010D8D1C8D0E947292122F3D8F4E
:1043A0004C8FB52FF62FE72FF82E092FA0E00E9493
:1043B00000945CF4A1E00E94E293122F3D8F4C8F99
:1043C000B52FF62FE72FF82E092F212F3D8D4C8D7D
:1043D0005B2F6F2F7E2F8F2D902F01E00E94BB93BC
:1043E000AAA8BBA8CCA8DDA8EEA8FFA808AD19AD67
:1043F0000E94D9932F962FAF2F9727963FAF2797DD
:10440000B42FA52FF62FE72F4C012B813C81498536
:104410005A856B857C858D859E85A980BA80CCA0C8
:10442000DDA0EEA0FFA008A519A50E94EE932B83A6
:104430003C8349875A876B877C878D879E872D8130
:104440003F8148855F85688979898A899B892F960C
:10445000AFAC2F972796BFAC2797CB2EDA2EEF2E37
:10446000FE2E84010E94EE932D833F8348875F8751
:10447000688B798B8A8B9B8B2C893D894E895F89D0
:10448000688D798D8A8D9B8DAEACBFAC2196CFACFB
:1044900021972296DFAC22972396EFAC23972496A0
:1044A000FFAC249725960FAD259726961FAD26972E
:1044B0000E94EE932056304F4F4F5F4F6F4F7F4F0C
:1044C0008F4F9F4F243D30434105510561057105D4
:1044D0008105910521F018F0BFEF2B1A3B0A4AAD78
:1044E0005BAD6CAD7DAD9A01AB0160E070E0CB01DE
:1044F00027962FAF279728963FAF289729964FAF3B
:1045000029972A965FAF2A972B966FAF2B972C96F9
:104510007FAF2C972D968FAF2D972E969FAF2E970E
:10452000AD80BF80C884DF84E888F9880A891B8948
:1045300060E070E080E090E00E947292122F3A8377
:104540004983B52FF62FE72FF82E092FA0E00E9400
:10455000009484F421503109404E5F4F6F4F7F4FDC
:104560008F4F9F4F122F3A834983B52FF62FE72F96
:10457000F82E092F212F3A8149815B2F6F2F7E2F33
:104580008F2D902F05E10E94BB93AB80BC80C98426
:10459000DA84EB84FC840D851E850E94EE93122F35
:1045A0003A834983B52FF62FE72FF82E092FA0E085
:1045B0000E94009484F4215030484F4F5F4F6F4F5A
:1045C0007F4F8F4F9F4F122F3A834983B52FF62F7E
:1045D000E72FF82E092F212F3A8149815B2F6F2F6A
:1045E0007E2F8F2D902F0FE00E94BB9359016A01FF
:1045F0007B018C01722E6B2CB42FAD2DF62F5F2C0E
:104600004C01285E33404109510961097109810952
:104610009109283D304D41405105610571058105E5
:10462000910509F010F4232869F09501A601B7015E
:10463000C8010E945B93722E632EB42FA52FF62F14
:10464000572E4C01272D362D4B2F5A2F6F2F752D9E
:10465000C4010E949C9520E030E048EC52E40E94A6
:10466000F094C25BDF4F0FB6F894DEBF0FBECDBF34
:10467000DF91CF911F910F91FF90EF90DF90CF903E
:10468000BF90AF909F908F907F906F905F904F9072
:104690003F902F9008954F925F926F927F928F92EA
:1046A0009F92AF92BF92CF92DF92EF92FF922B0137
:1046B0003C0169017A0123EC35EF4CE851E4C70174
:1046C000B6010E949C974B015C0128EB3EE143E759
:1046D00053E4C701B6010E940D949B01AC01C501D2
:1046E000B4010E94F0940E946A954B015C0120E0A5
:1046F00030E048EC52E4C301B2010E94F09421E89A
:1047000035E943EC50E40E949C97A50194010E9476
:104710009C974B015C0123E333E948E853E4C7016C
:10472000B6010E940D949B01AC01C501B4010E9429
:10473000F09423E333EB48E553E40E949C97FF9009
:10474000EF90DF90CF90BF90AF909F908F907F9031
:104750006F905F904F9008954F925F926F927F920B
:104760008F929F92AF92BF92CF92DF92EF92FF9281
:1047700069017A010E9410974B015C0123EC35EF2F
:104780004CE851E4C701B6010E949C972B013C0103
:1047900028EB3EE143E753E4C701B6010E940D94C4
:1047A0009B01AC01C301B2010E94F0946B017C013A
:1047B00020E030E040E050E4C501B4010E940C94D8
:1047C00022E93CE54EED5EE30E94F0949B01AC01D2
:1047D000C701B6010E940D946B017C0128EB3EE1FC
:1047E00043E753E40E949C974B015C01A7019601AB
:1047F00063EC75EF8CE891E40E940C949B01AC0192
:10480000C501B4010E94F094FF90EF90DF90CF902B
:10481000BF90AF909F908F907F906F905F904F90E0
:1048200008954F925F926F927F928F929F92AF9274
:10483000BF92CF92DF92EF92FF922B013C01690170
:104840007A0123EC35EF4CE851E4C701B6010E9430
:104850009C974B015C0128EB3EE143E753E4C70121
:10486000B6010E940D949B01AC01C501B4010E94E8
:10487000F0940E946A954B015C0120E030E048EC26
:1048800052E4C301B2010E94F094A50194010E9478
:104890009C9720E030E040E251E40E940C9424EE2A
:1048A00038E34EE05FE30E949C97A70196010E94C7
:1048B0000D94FF90EF90DF90CF90BF90AF909F90BE
:1048C0008F907F906F905F904F90089580E80E9446
:1048D000456581110DC08EEF0E944F65811108C0A2
:1048E00066E37CE980E090E00E94C7640C94476531
:1048F0000E9447658091283290912932A0912A32F6
:10490000B0912B320196A11DB11D80932832909356
:104910002932A0932A32B0932B320895FC01DC0196
:10492000AC014E5F5F4F90E031E38D91982788E0B6
:10493000292F220F97FF03C0922F932701C0922F98
:104940008150B1F7A417B50781F721E030E08281EB
:10495000891711F020E030E0C9010895DF92EF924D
:10496000FF920F931F93CF93DF930E94662480E8FA
:104970000E94456581116DC08AEF0E944F658111CB
:1049800068C08FE00E944F65811163C06AE67AE0DB
:1049900080E090E00E94C76481E80E944565811133
:1049A00058C00E946065D82F0E9460650E946065B3
:1049B000182F0E9460650E946065082F0E94606544
:1049C0000E946A65F82E80E80E944565811141C009
:1049D0008CEF0E944F6581113CC089EC0E944F65AD
:1049E000811137C06AE67AE080E090E00E94C764F7
:1049F00081E80E9445650E946065E82E0E9460651E
:104A0000D82E0E9460650E946065C82F0E946A656A
:104A10001F92DF921F92EF921F92FF921F920F93AD
:104A20001F921F931F92DF931F928F931F92CF931A
:104A30008EEB93E09F938F930E94E79C0E944765C3
:104A40008DB79EB742960FB6F8949EBF0FBE8DBF2E
:104A500017C00E9447658091283290912932A09119
:104A60002A32B0912B320196A11DB11D80932832BC
:104A700090932932A0932A32B0932B320E9466245D
:104A800020E030E040E050E060E070E080E090E066
:104A9000DF91CF911F910F91FF90EF90DF900895DC
:104AA000EF92FF920F931F93CF93DF9300D0CDB778
:104AB000DEB78C0180E80E944565811154C0011564
:104AC000110551F085EE0E944F6581114CC062E0E6
:104AD0007EE281E090E009C083EE0E944F65811183
:104AE00042C062E375E783E090E00E94C76481E81A
:104AF0000E944565811137C00E946065E82E898358
:104B00000E946065F82E8A830E946A658B830E94EA
:104B10004765CE0101960E948E24892B21F16F2DCD
:104B200070E07E296C7F80E090E0012B69F00E94AC
:104B3000A29520E030E04AEF5AE30E949C9720E0E3
:104B400030E040EC50E40CC00E94A29522E538EB26
:104B50004FE25BE30E949C9726E636E64BE352E485
:104B60000E940C941BC00E9447658091283290914E
:104B70002932A0912A32B0912B320196A11DB11D8C
:104B80008093283290932932A0932A32B0932B320B
:104B90000E94662460EF7FEF89E794E40F900F9006
:104BA0000F90DF91CF911F910F91FF90EF9008959B
:104BB0000F931F93CF93DF93729A8091660283FFC6
:104BC00008C08EE40E94EA64811165C0C0E5D0E0AF
:104BD00009C0C0E5D0E08FED97E00E94340E219728
:104BE000D1F7EFCF8FED97E00E94340E2197D1F7E8
:104BF0008FE40E94EA640E946065D82FDF730E94F0
:104C00006065082F0E946065C82F0E946A65182F92
:104C10000E9447658091660283FF72986D2F70E055
:104C2000762F6627600F711D80E090E00E94A295AC
:104C300020E134E048EC5BE30E949C9760930A2AF1
:104C400070930B2A80930C2A90930D2A6C2F70E09E
:104C5000762F6627610F711D769567957695679516
:104C600080E090E00E94A29524EA3CEF44E25CE3FD
:104C70000E949C9720E030E040E252E40E940C94B5
:104C80006093F7367093F8368093F9369093FA363E
:104C900080E090E002C081E090E0DF91CF911F9131
:104CA0000F9108957298729A8EE40E94EA6480EAE5
:104CB0000E944F6580E00E944F6580E00E944F6532
:104CC0008FE40E94EA640E9460658EE40E94EA64B8
:104CD00080E80E944F6580E00E944F6580E00E945E
:104CE0004F650E94476580E090E0089589E992E170
:104CF0009F938F930E94FB9C809180020F900F9056
:104D0000882361F01F928F9386E992E19F938F939E
:104D10000E94FB9C0F900F900F900F90089581E7D9
:104D200092E19F938F930E94FB9C89E492E19F9371
:104D30008F930E94FB9C82E292E19F938F930E944B
:104D4000FB9C87EE91E19F938F930E94FB9C8BEAE3
:104D500091E19F938F930E94FB9C89E791E19F9340
:104D60008F930E94FB9C8DE391E19F938F930E9410
:104D7000FB9C87E191E19F938F930E94FB9C81EEC6
:104D800090E19F938F930E94FB9C8091162E9091AF
:104D9000172E827098702DB73EB72E5E3F4F0FB61C
:104DA000F8943EBF0FBE2DBF892B41F081EB90E1FF
:104DB0009F938F930E94FB9C0F900F9085E890E14A
:104DC0009F938F930E94FB9C89E490E19F938F9324
:104DD0000E94FB9C80E290E19F938F930E94FB9C3A
:104DE00084EF9FE09F938F930E94FB9C85EC9FE054
:104DF0009F938F930E94FB9C83E99FE09F938F93E7
:104E00000E94FB9C82E69FE09F938F930E94FB9CF5
:104E100088E29FE09F938F930E94FB9C82EF9EE02D
:104E20009F938F930E94FB9C82EC9EE09F938F93B5
:104E30000E94FB9C86E99EE09F938F930E94FB9CBF
:104E400087E69EE09F938F930E94FB9C8EE29EE0FC
:104E50009F938F930E94FB9C85EF9DE09F938F9380
:104E60000E94FB9C8EEB9DE09F938F930E94FB9C86
:104E700080E99DE09F938F930E94FB9C8DB79EB726
:104E800080960FB6F8949EBF0FBE8DBF8CE59DE057
:104E90009F938F930E94FB9C8BE29DE09F938F9347
:104EA0000E94FB9C8CEF9CE09F938F930E94FB9C45
:104EB0008DEC9CE09F938F930E94FB9C86EA9CE084
:104EC0009F938F930E94FB9C80E79CE09F938F931E
:104ED0000E94FB9C8AE39CE09F938F930E94FB9C23
:104EE00084E09CE09F938F930E94FB9C8BED9BE062
:104EF0009F938F930E94FB9C83EA9BE09F938F93E9
:104F00000E94FB9C88E79BE09F938F930E94FB9CF1
:104F10002DB73EB72A5E3F4F0FB6F8943EBF0FBE87
:104F20002DBF08958DEE93E00C94239D4F925F92D8
:104F30006F927F928F929F92AF92BF92CF92DF92A9
:104F4000EF92FF92CF93DF93CDB7DEB728970FB6DE
:104F5000F894DEBF0FBECDBF80911C3290911D3200
:104F6000A0911E32B0911F3289839A83AB83BC8398
:104F700040901C3250901D3260901E3270901F3253
:104F800080911C3290911D32A0911E32B0911F323F
:104F90008D839E83AF83B88760911C3270911D32E0
:104FA00080911E3290911F322CE3822E912CA12CE5
:104FB000B12CA50194010E94F8917F936F9330E189
:104FC000C32E3EE0D32EE12CF12C6D817E818F81AA
:104FD0009885A70196010E94F891A50194010E946D
:104FE000F8913F932F9340E8842E41E5942EAA2414
:104FF000A394B12CC301B201A50194010E94F891C0
:10500000A70196010E94F8913F932F9369817A81BD
:105010008B819C81A50194010E94F8913F932F936D
:1050200082E59BE09F938F930E94FB9C0FB6F894C0
:10503000DEBF0FBECDBF28960FB6F894DEBF0FBE01
:10504000CDBFDF91CF91FF90EF90DF90CF90BF90D9
:10505000AF909F908F907F906F905F904F9008954A
:10506000E3E6FBE3808191818234924479F0E35658
:10507000FB43FF93EF9384E39BE09F938F930E9406
:10508000FB9C0F900F900F900F9008953A96E53F7C
:1050900081E8F80738F30895CF93DF93EC018C9AF9
:1050A0000E94A6109F938F937F936F9388E29BE05B
:1050B0009F938F930E94FB9C0F900F900F900F90E7
:1050C0000F900F90209719F084EB92E102C086E2D6
:1050D0009BE09F938F930E94FB9C0F900F9081E029
:1050E0000E945810209185023091860240918702DB
:1050F000509188020E949C979F938F937F936F9308
:105100008AE19BE09F938F930E94FB9C0F900F90EE
:105110000F900F900F900F90209719F084EB92E171
:1051200002C088E19BE09F938F930E94FB9C0F90AD
:105130000F9082E00E9458102091810230918202EB
:1051400040918302509184020E949C979F938F9379
:105150007F936F938CE09BE09F938F930E94FB9CC7
:105160000F900F900F900F900F900F90209719F0C5
:1051700084EB92E102C08AE09BE09F938F930E94B0
:10518000FB9C0F900F9083E00E9458109F938F9389
:105190007F936F938BEF9AE09F938F930E94FB9C7A
:1051A0008C980F900F900F900F900F900F9020976A
:1051B00019F084EB92E102C089EF9AE09F938F93FC
:1051C0000E94FB9C0F900F908091162E9091172EAD
:1051D00092FF88C021E042E161E080ED0E94B1666B
:1051E0009F938F937F936F938CEE9AE09F938F930F
:1051F0000E94FB9C0F900F900F900F900F900F90BC
:10520000209719F084EB92E102C08AEE9AE09F9316
:105210008F930E94FB9C0F900F9021E042E162E08F
:1052200080ED0E94B1669F938F937F936F938DED76
:105230009AE09F938F930E94FB9C0F900F900F908A
:105240000F900F900F90209719F084EB92E102C01D
:105250008BED9AE09F938F930E94FB9C0F900F9091
:1052600021E042E163E080ED0E94B1669F938F935D
:105270007F936F938EEC9AE09F938F930E94FB9C99
:105280000F900F900F900F900F900F90CD2B19F063
:1052900084EB92E102C08CEC9AE09F938F930E9482
:1052A000FB9C0F900F9021E042E164E080ED0E94B2
:1052B000B1669F938F937F936F938FEB9AE09F9349
:1052C0008F930E94FB9C0F900F900F900F900F9068
:1052D0000F9084EB92E19F938F930E94FB9C0F9021
:1052E0000F9002C0CD2BA9F3DF91CF9108950F93BA
:1052F0001F93CF93DF93882389F049E050E06FEF4D
:1053000070E08FED96E30E94319C49E050E06EE042
:1053100070E08FED96E30E94B29F13C0CFEDD6E30D
:105320000AEB1AE089911F928F931F930F930E94AB
:10533000FB9C0F900F900F900F9086E3C73ED8070D
:1053400089F784EB92E19F938F930E94FB9C0F90CF
:105350000F90DF91CF911F910F910895882311F045
:10536000299A089529980895882311F02A9A089572
:105370002A980895CF92DF92EF92FF92CF93DF9316
:105380006B017C0160FF11C08AE294E09F938F93D0
:105390008EEA92E19F938F930E94FB9C0F900F9057
:1053A0000F900F9081E090E002C080E090E0C1FE9D
:1053B00009C0EC01219647EE59E06FE274E00E94CB
:1053C0005916CE01C2FE09C0EC01219647EE59E004
:1053D00067E374E00E945916CE01C3FE09C0EC01D8
:1053E000219647EE59E06FE374E00E945916CE0112
:1053F000C4FE09C0EC01219647EE59E06FEF75E05D
:105400000E945916CE01C5FE09C0EC01219647EE57
:1054100059E063E474E00E945916CE01C6FE09C04B
:10542000EC01219647EE59E067E474E00E945916BA
:10543000CE01C7FE09C0EC01219647EE59E06DE4AC
:1054400074E00E945916CE01D0FE09C0EC012196ED
:1054500047EE59E065E574E00E945916CE01D1FE91
:1054600009C0EC01219647EE59E06DE574E00E9419
:105470005916CE01D2FE09C0EC01219647EE59E043
:1054800061E674E00E945916CE012091162E3091EB
:10549000172E24703071232B59F0D3FE09C0EC0174
:1054A000219647EE59E067E674E00E945916CE0156
:1054B0002091162E26FF0BC0D4FE09C0EC012196C8
:1054C00047EE59E06CE674E00E945916CE01209137
:1054D000162E27FF0BC0D5FE09C0EC01219647EE22
:1054E00059E062E774E00E945916CE01D6FE09C069
:1054F000EC01219647EE59E06AE774E00E945916E4
:10550000CE01D7FE09C0EC01219647EE59E065E8CF
:1055100074E00E945916CE01E0FE0CC047EE59E03F
:1055200066E974E0DF91CF91FF90EF90DF90CF902C
:105530000C945916CD28CE28CF2841F485EB9AE05B
:105540009F938F930E94FB9C0F900F90DF91CF91C0
:10555000FF90EF90DF90CF900895CF92DF92EF927F
:10556000FF92CF93DF93EC01C12CD12C76012097D1
:1055700009F4A3C060EB7AE0CE010E94039C892B62
:1055800011F46894C0F868EA7AE0CE010E94039CA6
:10559000892B11F46894C1F860EA7AE0CE010E9488
:1055A000039C892B11F46894C2F86CE97AE0CE016F
:1055B0000E94039C892B11F46894C3F869E97AE08E
:1055C000CE010E94039C892B11F46894C4F865E90C
:1055D0007AE0CE010E94039C892B11F46894C5F8EF
:1055E0006FE87AE0CE010E94039C892B11F4689445
:1055F000C6F867E87AE0CE010E94039C892B11F47B
:105600006894C7F86FE77AE0CE010E94039C892B6B
:1056100011F46894D0F86BE77AE0CE010E94039C05
:10562000892B11F46894D1F865E77AE0CE010E94E5
:10563000039C892B11F46894D2F860E77AE0CE01DC
:105640000E94039C892B11F46894D3F86AE67AE0EF
:10565000CE010E94039C892B11F46894D4F862E671
:105660007AE0CE010E94039C892B11F46894D5F84E
:1056700067E57AE0CE010E94039C892B11F46894BF
:10568000D6F866E47AE0CE010E94039C892B11F4DF
:105690006894D7F861E47AE0CE010E94039C892BDC
:1056A00011F46894E0F860917E0270917F0280E0CE
:1056B00090E00E94179CEC015ACFC701B601DF9120
:1056C000CF91FF90EF90DF90CF900895AF92BF926F
:1056D000CF92DF92EF92FF920F931F93CF93DF93BE
:1056E000122FD32FC42F052FF62EE72ED82EC92E1A
:1056F000217030E040E050E060E070E080E090E059
:10570000A0E00E94009489F08BE994E09F938F932E
:105710008EEA92E19F938F930E94FB9C0F900F90D3
:105720000F900F90E1E0F0E002C0E0E0F0E0809147
:10573000162E80FF19C0212F247030E040E050E089
:1057400060E070E080E090E0A0E00E94009461F0F2
:105750005F018FEFA81AB80A47EE59E06FE974E0CD
:10576000CF010E945916F501212F227030E040E050
:1057700050E060E070E080E090E0A0E00E940094E3
:1057800061F05F018FEFA81AB80A47EE59E063EAAB
:1057900074E0CF010E945916F501212F287030E0E6
:1057A00040E050E060E070E080E090E0A0E00E9427
:1057B000009461F05F018FEFA81AB80A47EE59E034
:1057C0006BEB74E0CF010E945916F501212F207177
:1057D00030E040E050E060E070E080E090E0A0E089
:1057E0000E94009461F05F018FEFA81AB80A47EE9B
:1057F00059E066EA74E0CF010E945916F501212FA5
:10580000207230E040E050E060E070E080E090E046
:10581000A0E00E94009461F05F018FEFA81AB80A1F
:1058200047EE59E069EA74E0CF010E945916F5018C
:10583000212F207430E040E050E060E070E080E034
:1058400090E0A0E00E94009461F05F018FEFA81A41
:10585000B80A47EE59E06FEA74E0CF010E9459168A
:10586000F501212F207830E040E050E060E070E06A
:1058700080E090E0A0E00E94009461F05F018FEF73
:10588000A81AB80A47EE59E065EB74E0CF010E9410
:105890005916F50120E03D2F317040E050E060E006
:1058A00070E080E090E0A0E00E94009461F05F0171
:1058B0008FEFA81AB80A47EE59E068EB74E0CF0101
:1058C0000E945916F50120E03D2F327040E050E073
:1058D00060E070E080E090E0A0E00E94009461F061
:1058E0005F018FEFA81AB80A47EE59E06DEB74E03C
:1058F000CF010E945916F50120E03D2F347040E0A1
:1059000050E060E070E080E090E0A0E00E94009451
:1059100061F05F018FEFA81AB80A47EE59E064EC16
:1059200074E0CF010E945916F50120E03D2F387038
:1059300040E050E060E070E080E090E0A0E00E9495
:10594000009461F05F018FEFA81AB80A47EE59E0A2
:1059500067EC74E0CF010E945916F50120E03D2F5D
:10596000307140E050E060E070E080E090E0A0E066
:105970000E94009461F05F018FEFA81AB80A47EE09
:1059800059E06CEC74E0CF010E945916F50120E05B
:105990003D2F307240E050E060E070E080E090E049
:1059A000A0E00E94009461F05F018FEFA81AB80A8E
:1059B00047EE59E063ED74E0CF010E945916F501FE
:1059C00020E030E040E050E06F2D647070E080E057
:1059D00090E0A0E00E94009461F05F018FEFA81AB0
:1059E000B80A47EE59E06AED74E0CF010E945916FB
:1059F000F5018091162E81FF19C020E03D2F3074F3
:105A000040E050E060E070E080E090E0A0E00E94C4
:105A1000009461F05F018FEFA81AB80A47EE59E0D1
:105A20006EED74E0CF010E945916F5018091162E9B
:105A30009091172E93FF19C020E030E040E0502FE6
:105A4000507160E070E080E090E0A0E00E9400947F
:105A500061F05F018FEFA81AB80A47EE59E061EED6
:105A600074E0CF010E945916F5018091162E909195
:105A7000172E93FF19C020E030E040E0502F507205
:105A800060E070E080E090E0A0E00E94009461F0AF
:105A90005F018FEFA81AB80A47EE59E064EE74E090
:105AA000CF010E945916F5018091162E9091172E64
:105AB00093FF19C020E030E040E0502F507460E0C8
:105AC00070E080E090E0A0E00E94009461F05F014F
:105AD0008FEFA81AB80A47EE59E06AEE74E0CF01DA
:105AE0000E945916F50120E03D2F307840E050E04B
:105AF00060E070E080E090E0A0E00E94009461F03F
:105B00005F018FEFA81AB80A47EE59E065EF74E01D
:105B1000CF010E945916F50120E030E04C2F417072
:105B200050E060E070E080E090E0A0E00E9400942F
:105B300061F05F018FEFA81AB80A47EE59E06AEFEB
:105B400074E0CF010E945916F50120E030E04C2F9F
:105B5000427050E060E070E080E090E0A0E00E94E1
:105B6000009461F05F018FEFA81AB80A47EE59E080
:105B70006DEF74E0CF010E945916F50120E030E08E
:105B80004C2F447050E060E070E080E090E0A0E0D6
:105B90000E94009461F05F018FEFA81AB80A47EEE7
:105BA00059E060E075E0CF010E945916F50120E050
:105BB00030E040E050E06F2D687070E080E090E0F1
:105BC000A0E00E94009461F05F018FEFA81AB80A6C
:105BD00047EE59E063E075E0CF010E945916F501E8
:105BE00020E030E040E050E06F2D607170E080E038
:105BF00090E0A0E00E94009461F05F018FEFA81A8E
:105C0000B80A47EE59E067E075E0CF010E945916E7
:105C1000F50120E030E040E050E060E07E2D717062
:105C200080E090E0A0E00E94009461F05F018FEFBF
:105C3000A81AB80A47EE59E06BE075E0CF010E9460
:105C40005916F5018091162E9091172E92FF19C0CA
:105C500020E030E04C2F487050E060E070E080E0E1
:105C600090E0A0E00E94009461F05F018FEFA81A1D
:105C7000B80A47EE59E066E175E0CF010E94591677
:105C8000F5018091162E9091172E92FF19C020E0F9
:105C900030E04C2F407150E060E070E080E090E038
:105CA000A0E00E94009461F05F018FEFA81AB80A8B
:105CB00047EE59E06AE175E0CF010E945916F501FF
:105CC0008091162E9091172E92FF19C020E030E09F
:105CD0004C2F407250E060E070E080E090E0A0E087
:105CE0000E94009461F05F018FEFA81AB80A47EE96
:105CF00059E06EE175E0CF010E945916F5018091DF
:105D0000162E9091172E92FF19C020E030E04C2FF4
:105D1000407450E060E070E080E090E0A0E00E941D
:105D2000009461F05F018FEFA81AB80A47EE59E0BE
:105D300062E275E0CF010E945916F5018091162E9E
:105D400082FF19C020E030E04C2F407850E060E046
:105D500070E080E090E0A0E00E94009461F05F01BC
:105D60008FEFA81AB80A47EE59E063E976E0CF0151
:105D70000E945916F5018091162E82FF19C020E06D
:105D800030E040E0502F517060E070E080E090E043
:105D9000A0E00E94009461F05F018FEFA81AB80A9A
:105DA00047EE59E066E275E0CF010E945916F50111
:105DB0008091162E9091172E93FF19C020E030E0AD
:105DC00040E0502F527060E070E080E090E0A0E092
:105DD0000E94009461F05F018FEFA81AB80A47EEA5
:105DE00059E069E275E0CF010E945916F5018091F2
:105DF000162E9091172E93FF19C020E030E040E05E
:105E0000502F547060E070E080E090E0A0E00E94CD
:105E1000009461F05F018FEFA81AB80A47EE59E0CD
:105E200061E375E0CF010E945916F5018091162EAD
:105E30009091172E94FF19C020E030E040E0502FE1
:105E4000587060E070E080E090E0A0E00E94009474
:105E500061F05F018FEFA81AB80A47EE59E06AE3D4
:105E600075E0CF010E945916F5018091162E85FF2D
:105E700019C020E030E040E050E06F2D607270E02B
:105E800080E090E0A0E00E94009461F05F018FEF5D
:105E9000A81AB80A47EE59E063E475E0CF010E9402
:105EA0005916F5018091162E85FF19C020E030E0CB
:105EB00040E050E06F2D607470E080E090E0A0E082
:105EC0000E94009461F05F018FEFA81AB80A47EEB4
:105ED00059E06CE475E0CF010E945916F5018091FC
:105EE000162E85FF1EC020E030E040E050E06F2D10
:105EF000607870E080E090E0A0E00E94009489F07B
:105F000047EE59E066E575E0CF01DF91CF911F9133
:105F10000F91FF90EF90DF90CF90BF90AF900C94D7
:105F20005916212F3D2F4C2F502F6F2D7E2D8D2D4B
:105F30009C2DA0E00E94009441F48CE39AE09F9392
:105F40008F930E94FB9C0F900F90DF91CF911F9138
:105F50000F91FF90EF90DF90CF90BF90AF9008959A
:105F60001F93CF93DF938091162ED0E082FF02C063
:105F700010E801C010E081FDD0E427E04AE250E0E3
:105F80006BE270E089E290E00E94956280E090E030
:105F90000E944F11882311F0CDE001C0C5E026E03A
:105FA0004AE250E06BE270E089E290E00E94956284
:105FB00081E090E00E944F112C2F882311F0206186
:105FC00001C02F7E50E060E08091162E9091172E38
:105FD000FC01E072FF2785FF02C0277F60E293FF8C
:105FE00002C0277F56E094FD5860EF2B09F0606CEB
:105FF0003D2F412F70E080E090E0DF91CF911F9125
:1060000008950E94B02FE9EFFDE1208331834283A0
:10601000538364837583868397838CE390E09187B1
:10602000808725E4228720E8238727E024871586B8
:1060300016861786108A118A938B828B85E0848B53
:1060400080E2858B168A178A108E81E0818F128EEE
:10605000138E88E592E0958F848F168E178E10A28E
:1060600011A212A213A214A215A217A216A248E20C
:1060700050E062E270E0CF010C94B29FCF92DF92C9
:10608000EF92FF920F931F93CF93DF93EC018B015D
:10609000FB0110826AE37AE00E94039C892B61F481
:1060A00081E0F801808360917E0270917F0280E040
:1060B00090E00E94179CEC0168E37AE0CE010E9418
:1060C000039C892B61F48FEFF801808360917E023D
:1060D00070917F0280E090E00E94179CEC01F12C0F
:1060E00000E010E0E12CD12CC12C209709F466C10E
:1060F00064E37AE0CE010E94039C892B19F4FF2D02
:10610000F160FF2E60E37AE0CE010E94039C892BB0
:1061100019F48F2D8460F82E6DE27AE0CE010E9492
:10612000039C892B19F4EF2DE260FE2E6BE27AE0DE
:10613000CE010E94039C892B19F4FF2DF860FF2EDD
:1061400068E27AE0CE010E94039C892B19F48F2D1E
:106150008061F82E62E27AE0CE010E94039C892BD6
:1061600019F4EF2DE062FE2E6CE17AE0CE010E9480
:10617000039C892B19F4FF2DF064FF2E69E17AE06E
:10618000CE010E94039C892B19F48F2D8068F82E74
:1061900064E17AE0CE010E94039C892B09F401603E
:1061A0006DE07AE0CE010E94039C892B09F4026025
:1061B0006AE07AE0CE010E94039C892B09F4046016
:1061C00065E07AE0CE010E94039C892B09F4086007
:1061D0006EEF79E0CE010E94039C892B09F40061E7
:1061E00067EF79E0CE010E94039C892B09F40062DD
:1061F00063EF79E0CE010E94039C892B19F4ED2D09
:10620000E460DE2E60EF79E0CE010E94039C892BD2
:1062100009F400646BEE79E0CE010E94039C892BA7
:1062200009F4006868EE79E0CE010E94039C892B96
:1062300009F4116065EE79E0CE010E94039C892B80
:1062400009F4126062EE79E0CE010E94039C892B72
:1062500009F414606EED79E0CE010E94039C892B55
:1062600009F418606AED79E0CE010E94039C892B45
:1062700009F4106166ED79E0CE010E94039C892B40
:1062800009F4106262ED79E0CE010E94039C892B33
:1062900009F4106460ED79E0CE010E94039C892B23
:1062A00009F410686DEC79E0CE010E94039C892B03
:1062B00019F4FE2DF160EF2E65EC79E0CE010E941D
:1062C000039C892B19F48E2D8260E82E6CEB79E00B
:1062D000CE010E94039C892B19F4EE2DE460EE2E72
:1062E00063EB79E0CE010E94039C892B19F4FE2D0B
:1062F000F860EF2E60EB79E0CE010E94039C892BC1
:1063000019F48E2D8061E82E6AEA79E0CE010E94B0
:10631000039C892B19F4EE2DE062EE2E6FE979E0F3
:10632000CE010E94039C892B19F4FE2DF064EF2E00
:106330006BE979E0CE010E94039C892B19F48D2D25
:106340008860D82E67E979E0CE010E94039C892BF2
:1063500019F4ED2DE061DE2E6EE879E0CE010E94A9
:10636000039C892B19F4FD2DF062DF2E64E879E09F
:10637000CE010E94039C892B19F48D2D8064D82EA8
:106380006BE779E0CE010E94039C892B19F4ED2D77
:10639000E068DE2E60E779E0CE010E94039C892B45
:1063A00019F4FC2DF160CF2E60917E0270917F0276
:1063B00080E090E00E94179CEC0197CE2F2D302FAB
:1063C000412F5E2D6D2D7C2D80E090E0DF91CF91EF
:1063D0001F910F91FF90EF90DF90CF9008953F9223
:1063E0004F925F926F927F928F929F92AF92BF92E5
:1063F000CF92DF92EF92FF920F931F93CF93DF9391
:10640000582EC9EFDDE100E010E08AE6E82E89E0D1
:10641000F82E852D8170382E852D8270482E95E5B9
:10642000C92E99E0D92E2DE5A22E29E0B22E3BE50A
:10643000832E39E0932E44EB642E42E1742E5520D6
:1064400051F01F930F93FF92EF920E94FB9C0F90CD
:106450000F900F900F903320A1F089858F9388853E
:106460008F93BF92AF920E94FB9C0F900F900F9062
:106470000F904420C1F09F928F920E94FB9C0F903E
:106480000F90442081F0DF92CF920E94FB9C2881E4
:1064900039814A815B816C817D818E819F810E94DF
:1064A000662B0F900F907F926F920E94FB9C0F5F64
:1064B0001F4F2A960F900F900430110509F0BFCF9F
:1064C000DF91CF911F910F91FF90EF90DF90CF90D0
:1064D000BF90AF909F908F907F906F905F904F9004
:1064E0003F90089580E599E09F938F930E94FB9CD5
:1064F0008091062A9091072AA091082AB091092A32
:106500000F900F90813027EA92072EE1A207B10584
:1065100019F482E499E01DC0823026EA92072EE148
:10652000A207B10519F485E399E013C0823027EA88
:1065300092072EE1A207B10519F487E299E009C09C
:10654000823028EA92072EE1A207B10549F489E1D9
:1065500099E09F938F930E94FB9C0F900F9008955A
:10656000BF93AF939F938F9383E199E09F938F9312
:106570000E94FB9C0F900F900F900F900F900F9028
:10658000089583E099E09F938F930E94FB9C0E9463
:1065900092270E94723284EB92E19F938F930E9424
:1065A000FB9C8EB390E00E94C16C80EE9DE19F93B6
:1065B0008F938BEF98E09F938F930E94FB9C609149
:1065C000600270916102809162029091630228EEF4
:1065D00033E040E050E00E94F8915F934F933F9387
:1065E0002F938BEE98E09F938F930E94FB9C82EEFB
:1065F00098E09F938F930E94FB9C0E94C31680910A
:10660000162E2DB73EB7205F3F4F0FB6F8943EBF12
:106610000FBE2DBF80FF05C041E061E081E00E9418
:106620009F188EED98E09F938F930E94FB9C80E0D3
:106630000E9477290E949627809165021F928F936E
:1066400085ED98E09F938F930E94FB9C8091C614E8
:106650001F928F938CEC98E09F938F930E94FB9CEA
:10666000809190028F9380918F028F9380918E0200
:106670008F9380918D028F938EEB98E09F938F93F1
:106680000E94FB9C1F9280E48F9386EA98E09F9380
:106690008F930E94FB9C809142391F928F9380912F
:1066A00041391F928F9383E998E09F938F930E94C3
:1066B000FB9C809164021F928F938AE898E09F93DD
:1066C0008F930E94FB9C8091660290916702A0913B
:1066D0006802B09169022DB73EB7225E3F4F0FB6F8
:1066E000F8943EBF0FBE2DBF96FD03C08FE595E029
:1066F00002C083E99AE09F938F9380E898E09F938C
:106700008F930E94FB9C83E00E94EF310F900F90CB
:106710000F900F901D9903C08FE595E002C083E9AB
:106720009AE09F938F9384E798E09F938F930E94C2
:10673000FB9C8AE698E09F938F930E94FB9C80913C
:1067400066020F900F900F900F900F900F9081FFA7
:1067500009C084E698E09F938F930E94FB9C0F9062
:106760000F9013C080FD03C08FE595E002C083E960
:106770009AE09F938F9380E698E09F938F930E9477
:10678000FB9C0F900F900F900F908091660290915C
:106790006702A0916802B091690297FD03C08FE57E
:1067A00095E002C083E99AE09F938F9387E598E094
:1067B0009F938F930E94FB9C80E598E09F938F931B
:1067C0000E94FB9C6091C9147091CA148091CB14F3
:1067D0009091CC140E94BA2984EB92E19F938F93FD
:1067E0000E94FB9C8DB79EB708960FB6F8949EBF8B
:1067F0000FBE8DBF779B03C08FE595E002C083E994
:106800009AE09F938F9387E498E09F938F930E94E1
:10681000FB9C0E943A0E0E940B119F938F937F93D3
:106820006F9389E398E09F938F930E94FB9C0E9453
:10683000BA109F938F937F936F938BE298E09F930F
:106840008F930E94FB9C81E090E00E944C288091F5
:10685000C5369091C636A091C736B091C836BF9361
:10686000AF939F938F938DE198E09F938F930E94B6
:10687000FB9C8091DA368F938091D9368F938091EB
:10688000D8368F938091D7368F9389E098E09F9385
:106890008F930E94FB9C8091C9369091CA36A0913B
:1068A000CB36B091CC36BF93AF939F938F938BEF42
:1068B00097E09F938F930E94FB9C2DB73EB72E5D70
:1068C0003F4F0FB6F8943EBF0FBE2DBF8091DE360E
:1068D0008F938091DD368F938091DC368F938091FA
:1068E000DB368F9387EE97E09F938F930E94FB9CFC
:1068F00061E070E080E090E00E94BE1161E070E035
:1069000081E090E00E94BE110F900F900F900F90C9
:106910000F900F90299903C08FE595E002C083E99D
:106920009AE09F938F938FED97E09F938F930E94B0
:10693000FB9C0F900F900F900F902A9903C08FE54A
:1069400095E002C083E99AE09F938F9387ED97E0EB
:106950009F938F930E94FB9C8091660290916702A7
:10696000A0916802B09169020F900F900F900F9064
:1069700094FD03C08FE595E002C083E99AE09F9300
:106980008F938FEC97E09F938F930E94FB9C809155
:10699000162E0F900F900F900F9085FF5FC081E033
:1069A0000E944A696091EA367091EB368091EC362C
:1069B0009091ED360E94A49520E030E048EC52E43E
:1069C0000E94F0949F938F937F936F9383E695E05B
:1069D0009F938F930E94E79C6091EE367091EF3603
:1069E0008091F0369091F1360E94A29520E030E03F
:1069F00040E85AE30E949C979F938F937F936F93F5
:106A000082E795E09F938F930E94E79C6091F23616
:106A10007091F3368091F4369091F5360E94A295EC
:106A200020E030E040E85BE30E949C979F938F93C7
:106A30007F936F9383E895E09F938F930E94E79CE9
:106A400084EB92E19F938F930E94FB9C8DB79EB73E
:106A500044960FB6F8949EBF0FBE8DBF0895F8946C
:106A600091E2E0E0F0E0909357008491E2E0F0E002
:106A7000909357002491E4E0F0E090935700E49164
:106A800090E0A0E0B0E0BC0155274427822F90E0C1
:106A9000A0E0B0E0BA2FA92F982F8827840F951F68
:106AA000A61FB71F8E0F911DA11DB11D8093062A31
:106AB0009093072AA093082AB093092A78940895FE
:106AC000CF93DF93CDB7DEB761970FB6F894DEBFF3
:106AD0000FBECDBF48E250E062E270E089EF9DE179
:106AE0000E94949F2091F91D3091FA1D4091FB1D49
:106AF0005091FC1D6091FD1D7091FE1D8091FF1D48
:106B00009091001EAFEF0E94009411F40E9401309A
:106B100044E050E06EE170E0CE010B960E94949F3D
:106B20008B859C85AD85BE858F3F2FEF9207A20791
:106B3000B207A9F48AE090E4A0E0B0E08093660296
:106B400090936702A0936802B093690244E050E01A
:106B50006EE170E086E692E00E94B29F08C08093EA
:106B6000660290936702A0936802B09369028091D5
:106B7000660290916702A0916802B0916902A2FF3B
:106B800002C02A9A03C080E00E94B42944E050E089
:106B90006AE570E0CE010B960E94949F8B859C85E0
:106BA000AD85BE858F3F2FEF9207A207B20789F40C
:106BB0001092C9141092CA141092CB141092CC14D3
:106BC00044E050E06AE570E089EC94E10E94B29FF5
:106BD00008C08093C9149093CA14A093CB14B093A7
:106BE000CC1449E050E06EE070E08FED96E30E9437
:106BF000949F0E94051344E050E06EE470E0CE01E3
:106C00000B960E94949F8B859C85AD85BE8544E044
:106C100050E06EE470E08F3F9F4FAF4FBF4F29F4BD
:106C200085E892E00E94B29F04C085E892E00E944D
:106C3000949F44E050E06AE470E0CE010B960E941D
:106C4000949F8B859C85AD85BE8544E050E06AE4C9
:106C500070E08F3F9F4FAF4FBF4F29F481E892E024
:106C60000E94B29F04C081E892E00E94949F44E099
:106C700050E062E570E0CE010B960E94949F8B85F8
:106C80009C85AD85BE8544E050E062E570E08F3FB5
:106C90009F4FAF4FBF4F29F489E892E00E94B29F07
:106CA00004C089E892E00E94949F41E050E06DE1C9
:106CB00070E0CE0141960E94949F898941E050E0A6
:106CC0006DE170E08F3F29F486EC94E10E94B29F61
:106CD00004C086EC94E10E94949F41E050E06CE196
:106CE00070E0CE0141960E94949F898941E050E076
:106CF0006CE170E08F3F29F485E692E00E94B29F3C
:106D000004C085E692E00E94949F41E050E06BE170
:106D100070E0CE0141960E94949F898941E050E045
:106D20006BE170E08F3F29F484E692E00E94B29F0D
:106D300004C084E692E00E94949F4AE050E064E040
:106D400070E0CE0101960E94949F89814AE050E054
:106D500064E070E08F3F29F480EE9DE10E94B29FD5
:106D600004C080EE9DE10E94949F44E050E066E5FF
:106D700070E0CE010B960E94949F8B859C85AD851B
:106D8000BE8544E050E066E570E08F3F9F4FAF4F17
:106D9000BF4F29F48DE892E00E94B29F04C08DE8B5
:106DA00092E00E94949F44E050E067E170E0CE01E1
:106DB0000B960E94949F8B859C85AD85BE8544E093
:106DC00050E067E170E08F3F9F4FAF4FBF4F29F416
:106DD00080E692E00E94B29F04C080E692E00E94AA
:106DE000949F8091600290916102A0916202B091A3
:106DF000630281389A41A640B105A0F088E394E08F
:106E00009F938F930E94FB9C80E197E2A0E0B0E00B
:106E10008093600290936102A0936202B093630238
:106E20000F900F90609160027091610280916202F8
:106E3000909163020E94D46442E050E062E070E00E
:106E4000CE010F960E94949F8F85988942E050E072
:106E500062E070E08F3F910529F48FEB94E10E948E
:106E6000B29F04C08FEB94E10E94949F42E050E0F7
:106E700060E070E0CE010F960E94949F8F85988904
:106E800042E050E060E070E08F3F910529F48DEB27
:106E900094E10E94B29F04C08DEB94E10E94949F04
:106EA00061960FB6F894DEBF0FBECDBFDF91CF91D4
:106EB0000895CF92DF92EF92FF920E9401308AE014
:106EC00090E4A0E0B0E08093660290936702A09304
:106ED0006802B093690244E050E06EE170E086E63B
:106EE00092E00E94B29F1092C9141092CA1410929C
:106EF000CB141092CC1444E050E06AE570E089ECC9
:106F000094E10E94B29F82E2C82EDD24DA948CECD8
:106F1000E82E8BE3F82EC0928502D0928602E09292
:106F20008702F092880244E050E06EE470E085E869
:106F300092E00E94B29FC0928102D0928202E092BF
:106F40008302F092840244E050E06AE470E081E859
:106F500092E00E94B29F87ED94E3AFEEBCE3809392
:106F6000890290938A02A0938B02B0938C0244E032
:106F700050E062E570E089E892E00E94B29F8AE901
:106F800099E9A9E1B0E480938D0290938E02A093D9
:106F90008F02B093900244E050E066E570E08DE827
:106FA00092E00E94B29F1092C61480E00E946A7420
:106FB00041E050E06DE170E086EC94E10E94B29F08
:106FC0008AE1809365020E94577341E050E06CE1D2
:106FD00070E085E692E00E94B29F8FE080936402A9
:106FE00041E050E06BE170E084E692E00E94B29FE5
:106FF0008AE0E0EEFDE1DF011D928A95E9F74AE0C3
:1070000050E064E070E0CF010E94B29F80E197E21F
:10701000A0E0B0E08093600290936102A0936202CE
:10702000B093630244E050E067E170E080E692E0F4
:107030000E94B29F1092C0141092BF1442E050E020
:1070400062E070E08FEB94E10E94B29F1092BE1458
:107050001092BD1442E050E060E070E08DEB94E1EE
:107060000E94B29F81E00E94772980E090E0FF902B
:10707000EF90DF90CF900C941A130E9478706C9A66
:107080006B9A6A9A6F9A729A749A739A779A80989E
:1070900080B3897F80BB8398849887E080937E004B
:1070A000549A0E942F350E9460358091660290911B
:1070B0006702A0916802B091690294FD0E948770F6
:1070C0000E94A80E80E090E00E941A136091600276
:1070D0007091610280916202909163020E94D46477
:1070E0000E94BA10609318327093193280931A324A
:1070F00090931B328091660286FD239A219A229AF0
:10710000239A0E94BD0E1D9B05C01092C8141092B8
:10711000C714089581E090E09093C8148093C71439
:107120000895CF93DF9390E04091C9145091CA1411
:107130006091CB147091CC1441FD08C0209166027F
:1071400020FD04C021FF92C01D9B90C02DE8289F08
:10715000E001299FD00D1124CE018A5F904E9F93AC
:107160008F9383E995E09F938F930E94E79CFE01A4
:10717000E150F14EDF01AA57BF4F2C910F900F90B5
:107180000F900F90438154816581768180911C32EC
:1071900090911D32A0911E32B0911F32841B950B2D
:1071A000A60BB70B2223D1F1BF93AF939F938F937D
:1071B000DF01A257BF4F11968C9111978F938C913D
:1071C0008F93129711968C9111978F938C918F9327
:1071D00013978C911F928F9311978C911F928F937D
:1071E00013968C911F928F9311978C911F928F936E
:1071F000E957FF4F80811F928F931F922F9389E948
:1072000095E09F938F930E94E79C8DB79EB746961B
:107210000FB6F8949EBF0FBE8DBF10C0BF93AF9343
:107220009F938F9380EE95E09F938F930E94E79CAE
:107230000F900F900F900F900F900F9084EB92E1B2
:107240009F938F930E94FB9C809180020F900F90E0
:10725000882361F01F928F9385E394E09F938F932F
:107260000E94FB9C0F900F900F900F90DF91CF9199
:1072700008958091FF1E882341F08091001F90E0C7
:107280000E9491380E94AE0FF4CF0895CF93DF9300
:10729000EC01888199818E362FE09207F1F018F485
:1072A000892BC1F04BC086372FE0920709F44CC000
:1072B0008A379F4009F042C080E89BE00E94E77750
:1072C000892B09F43FC080E89BE00E94D37780E0DF
:1072D0000E94AE298EE69FE02EC0623199F5299A70
:1072E0004091BD145091BE145695542F4427579584
:1072F000479560E070E080E89BE00E94C97780914C
:10730000C9149091CA14A091CB14B091CC14A0FFD1
:1073100010C08091BE148F938091BD148F9383E52C
:1073200093E19F938F930E94FB9C0F900F900F907F
:107330000F9086E79FE09983888304C019821882A2
:1073400083E019C081E017C080E89BE00E94E777E6
:10735000892BC1F380E89BE00E94D3770E943939E2
:1073600040E250E060E070E080E89BE00E94C97776
:107370008AE79FE0E0CFDF91CF9108952F923F926F
:107380004F925F926F927F928F929F92AF92BF9235
:10739000CF92DF92EF92FF920F931F93CF93DF93E1
:1073A000CDB7DEB72B970FB6F894DEBF0FBECDBFBB
:1073B0009B878A873A01FC0180819181892B11F09A
:1073C0000C94074F60917E0270917F02CA010E9467
:1073D000179C60E870E0C3010E94579C009759F425
:1073E00060915D3B70915E3B8AE090E00E94AB9CB7
:1073F00081E00C940C4F8130910561F4F301108110
:10740000912E990C9908892CE92CF92C092D492CDD
:10741000592CC0C082309105B9F4F3018081082E47
:10742000000C990B982F88272181820F911D27FD31
:107430009A95182F992E892E880C8808E82CF82CFC
:10744000082D482C582CA6C083309105C1F5F301B6
:107450002081922F990F990B392F492F592F692F7E
:10746000792F892F00E10E94A29329014A01B62FAA
:10747000A72F382E292E2181922F990F990B392F62
:10748000492F592F692F792F892F08E00E94A29345
:1074900059016A017B018C019201A4016B2F7A2FA3
:1074A000832D922D0E94D993A2801A2D110F110BBA
:1074B000B12EC12ED12EE12EF12E012F59C00497ED
:1074C0000CF460C0F3012081922F990F990B392F92
:1074D000492F592F692F792F892F08E10E94A293F4
:1074E00029014A01B62FA72F382E292E2181922F4C
:1074F000990F990B392F492F592F692F792F892FE0
:1075000000E10E94A29359016A017B018C01920162
:10751000A4016B2F7A2F832D922D0E94D993A380E3
:107520001A2D110F110BB12EC12ED12EE12EF12EDD
:10753000012F0E94D99329014A01B62FA72F382E77
:10754000292E2281922F990F990B392F492F592FCC
:10755000692F792F892F08E00E94A29359016A01AF
:107560007B018C019201A4016B2F7A2F832D922D28
:107570000E94D993122F932E842EE52EF62E072FDC
:107580002C0108C01AE0912C812CE12CF12C00E098
:10759000412C512C34EB232E32E1332E3F922F928B
:1075A0000E94FB9C0F900F90212F392D482D5E2DAE
:1075B0006F2D702FC2012537F3E63F07FDE64F0719
:1075C0005105610571058105910511F40C9421495E
:1075D0002537E3E63E07EDE64E07510561057105E7
:1075E0008105910511F008F0B9C12337F2E73F0793
:1075F00041055105610571058105910511F40C9452
:10760000EB4B2337E2E73E07410551056105710564
:107610008105910511F008F0BCC02536F4E63F075E
:1076200041055105610571058105910509F4FAC708
:107630002536E4E63E0741055105610571058105E2
:10764000910511F008F042C0A6E70E94009411F4E1
:107650000C94A0450E94009409F070F4A8E60E94E2
:10766000009411F40C946F43A5E70E94009411F468
:107670000C948A450C94054F212F392D482D5E2DF1
:107680006F2D702FC2012436F1E63F0741055105E9
:10769000610571058105910511F40C94134C253792
:1076A000E2E63E0741055105610571058105910539
:1076B00009F448C52A333642410551056105710573
:1076C0008105910509F43EC30C94054F212F392DF6
:1076D000482D5E2D6F2D702FC2012737EFE63E0734
:1076E00041055105610571058105910511F40C9461
:1076F0008B492737FFE63F074105510561057105B5
:107700008105910509F0C8F42436E9E63E074105F4
:107710005105610571058105910511F40C946345CE
:1077200025363E46410551056105710581059105E6
:1077300011F40C94C3490C94054F212F392D482D79
:107740005E2D6F2D702FC2012536E2E73E07410501
:107750005105610571058105910511F40C949E4A4E
:107760002936F2E73F07410551056105710581059D
:10777000910511F40C949A4B23333147410551057F
:10778000610571058105910511F00C94054F0C946C
:10779000134C212F392D482D5E2D6F2D702FC201D6
:1077A0002236F5E63F07F4E64F07510561057105FE
:1077B0008105910509F436C72236E5E63E07E4E681
:1077C0004E075105610571058105910511F008F01D
:1077D0005CC02133F4E63F07F1E64F075105610530
:1077E00071058105910509F4C1C22133E4E63E0724
:1077F000E1E64E075105610571058105910509F026
:10780000C0F42337F3E73F074105510561057105D2
:107810008105910511F40C94FF4B2837344741053D
:107820005105610571058105910509F48BC20C9420
:10783000054F212F392D482D5E2D6F2D702FC20140
:107840002837F4E63F07F1E64F075105610571055A
:107850008105910509F486C22C36E5E73E07E2E68C
:107860004E075105610571058105910509F46AC44A
:107870002336344641465105610571058105910560
:1078800011F00C94054F0C94134C212F392D482DD9
:107890005E2D6F2D702FC2012D36E5E73E07E8E61D
:1078A0004E075105610571058105910511F40C9490
:1078B000294C2D36F5E73F07F8E64F0751056105DE
:1078C00071058105910509F0E0F42237E2E73E07F2
:1078D000E5E64E075105610571058105910511F435
:1078E0000C94CE4823363D46484651056105710546
:1078F0008105910511F00C94054F0E94EA1C0C942F
:10790000074F212F392D482D5E2D6F2D702FC2016D
:107910002436E3E63E07ECE64E07510561057105A6
:107920008105910511F40C9431482736FFE63F0795
:10793000FCE64F075105610571058105910511F4BC
:107940000C9434482336324349465105610571058C
:107950008105910511F00C94054F28C2212F392D76
:10796000482D5E2D6F2D702FC2012037FCE63F079A
:10797000F5E64F07F8E65F0761057105810591059A
:1079800009F4ADC62037ECE63E07E5E64E07E8E62B
:107990005E07610571058105910511F008F0E3C0EE
:1079A0002437F8E73F07F4E74F07510561057105F4
:1079B0008105910511F40C940C462437E8E73E0745
:1079C000E4E74E075105610571058105910511F048
:1079D00008F05EC02033F1E33F07F1E74F075105A0
:1079E000610571058105910511F40C94CE48203391
:1079F000E1E33E07E1E74E075105610571058105A9
:107A0000910509F0C0F42133F2E63F07F0E74F0794
:107A10005105610571058105910509F4A8C222335C
:107A2000324640475105610571058105910509F40C
:107A3000F3C20C94054F212F392D482D5E2D6F2D4B
:107A4000702FC2012037F5E63F07F2E74F075105D7
:107A5000610571058105910511F40C949E4A2C363F
:107A6000E4E73E074E075105610571058105910563
:107A700011F40C941C4E21333143414751056105EB
:107A800071058105910511F00C94054F0C94214965
:107A9000212F392D482D5E2D6F2D702FC2012B36D1
:107AA000ECE63E07E5E74E07E2E65E076105710595
:107AB0008105910509F446C32B36FCE63F07F5E73F
:107AC0004F07F2E65F07610571058105910509F031
:107AD000E0F42437E4E63E07E7E74E075105610589
:107AE00071058105910511F40C94704E24373F46C1
:107AF0004F465246610571058105910511F00C94C0
:107B0000054F0C9400000C94074F212F392D482D60
:107B10005E2D6F2D702FC2012E36E1E63E07E8E69E
:107B20004E07E3E65E07610571058105910511F4D5
:107B30000C94E0452633F9E63F07F5E74F07F5E6F5
:107B40005F07610571058105910509F4CCC52936EA
:107B50003C4641465346610571058105910511F08A
:107B60000C94054F99C3212F392D482D5E2D6F2D73
:107B7000702FC2012437F3E73F07F5E64F07F2E71E
:107B80005F07610571058105910511F40C943F4A69
:107B90002437E3E73E07E5E64E07E2E75E076105C7
:107BA00071058105910511F008F063C02337F5E6F2
:107BB0003F07F2E74F07F0E75F07610571058105B1
:107BC000910511F40C94E54C2337E5E63E07E2E716
:107BD0004E07E0E75E07610571058105910509F033
:107BE000D0F42136FDE63F07F5E74F07F8E65F07DB
:107BF000610571058105910511F40C94A94922379D
:107C0000374740475047610571058105910509F4E3
:107C100068C20C94054F212F392D482D5E2D6F2DF4
:107C2000702FC2012436FDE63F07F3E64F07F2E767
:107C30005F07610571058105910509F45FC621366D
:107C4000ECE63E07E5E64E07E2E75E0761057105F3
:107C50008105910509F464C52337324747475047EA
:107C6000610571058105910511F00C94054F0C9487
:107C7000514A212F392D482D5E2D6F2D702FC201B5
:107C80002437E2E73E07E1E64E07E5E75E076105D8
:107C900071058105910509F48CC62437F2E73F0789
:107CA000F1E64F07F5E75F0761057105810591056D
:107CB00009F0C8F42437E3E73E07E5E64E07E4E7BA
:107CC0005E07610571058105910509F4D0C7273765
:107CD000304748475447610571058105910509F40E
:107CE00045C70C94054F212F392D482D5E2D6F2D42
:107CF000702FC2012F36ECE63E07EFE54E07E6E7B0
:107D00005E07610571058105910509F4A2C52C3650
:107D1000F1E63F07F4E74F07F8E75F0761057105F4
:107D20008105910511F40C94E34D22373746404705
:107D30005547610571058105910511F00C94054FBA
:107D40000C940D4883E08093CD361092CF3610927C
:107D5000CE364DEC56E362E182E492E00E94167A60
:107D60000C94074F0E947F1C0C94074F21E042E1C6
:107D700061E080ED0E94B16621E042E161E080EDCA
:107D80000E94B16621E042E161E080ED0E94B166AF
:107D900021E042E161E080ED0E94B16621E042E134
:107DA00061E080ED0E94B1660C94074F60917E0205
:107DB00070917F0280E090E00E94179C6CEE75E06D
:107DC0000E94389C892B09F0CEC060917E02709190
:107DD0007F0280E090E00E94179C8C01009709F4DC
:107DE0009DC060E873E00E94389C892BE1F488EE26
:107DF00093E0A0E0B0E08093600290936102A093D2
:107E00006202B093630268EE73E080E090E00E944B
:107E1000D46444E050E067E170E080E692E00E94C4
:107E2000B29F0C94074F62EF75E0C8010E94389C26
:107E3000892BE1F480E197E2A0E0B0E0809360025A
:107E400090936102A0936202B093630260E177E2D3
:107E500080E090E00E94D46444E050E067E170E08C
:107E600080E692E00E94B29F0C94074F65EF75E0A8
:107E7000C8010E94389C892BE1F480EA96E8A1E0D1
:107E8000B0E08093600290936102A0936202B0938D
:107E9000630260EA76E881E090E00E94D46444E006
:107EA00050E067E170E080E692E00E94B29F0C949F
:107EB000074F69EF75E0C8010E94389C892BE1F4F7
:107EC00080E89AE1A6E0B0E08093600290936102BE
:107ED000A0936202B093630260E87AE186E090E0EA
:107EE0000E94D46444E050E067E170E080E692E0F4
:107EF0000E94B29F0C94074F84EF95E09F938F935D
:107F00000E94FB9C84EB92E19F938F930E94FB9CC9
:107F10000F900F900F900F900C94074F609160029C
:107F200070916102809162029091630228EE33E0C9
:107F300040E050E00E94F8915F934F933F932F935E
:107F400080EF95E09F938F930E94FB9C84EB92E1DE
:107F50009F938F930E94FB9C0FB6F894DEBF0FBED9
:107F6000CDBF0C94074F0E94C3160C94074F60912D
:107F70007E0270917F0280E090E00E94179C8C014D
:107F800063E97AE00E94389C892BA1F48091660213
:107F900090916702A0916802B0916902A2608093FB
:107FA000660290936702A0936802B0936902299ACF
:107FB0000C94074F6FE575E0C8010E94389C892B2F
:107FC000B1F48091660290916702A0916802B0912D
:107FD0006902AD7F8093660290936702A093680266
:107FE000B093690280E00E94AE290C94074F299B50
:107FF00003C083E99AE002C08FE595E09F938F93D9
:1080000088EE95E09F938F930E94FB9C0F900F90BA
:108010000F900F900C94074F60917E0270917F0239
:1080200080E090E00E94179C8C0163E97AE00E9456
:10803000389C892BE1F48091660290916702A091AF
:108040006802B0916902A46080936602909367020F
:10805000A0936802B09369022A9A44E050E06EE16E
:1080600070E086E692E00E94B29F0C94074F6FE5A5
:1080700075E0C8010E94389C892BF1F4809166025A
:1080800090916702A0916802B0916902AB7F8093E2
:10809000660290936702A0936802B093690280E041
:1080A0000E94B42944E050E06EE170E086E692E080
:1080B0000E94B29F0C94074F2A9B03C083E99AE069
:1080C00002C08FE595E09F938F9380EE95E09F939C
:1080D0008F930E94FB9C0F900F900F900F900C9429
:1080E000074F60917E0270917F0280E090E00E94D5
:1080F000179C8C0163E97AE00E94389C892B19F463
:1081000077980C94074F6FE575E0C8010E94389C82
:10811000892B19F4779A0C94074F779903C083E958
:108120009AE002C08FE595E09F938F9389EB97E0EB
:108130009F938F930E94FB9C0F900F900F900F9036
:108140000C94074F60917E0270917F0280E090E076
:108150000E94179C8C016DEF75E00E94389C892B62
:10816000D1F48091FF1E1F928F938091011F1F9267
:108170008F938091001F1F928F931F9284E18F93A2
:1081800086EB95E09F938F930E94FB9C0FB6F8942B
:10819000DEBF0FBECDBF62E076E0C8010E94389C12
:1081A000892B19F40E9439396DC061E77AE0C80162
:1081B0000E94389C892BF9F560917E0270917F02B4
:1081C00080E090E00E94179C009709F45BC00E9439
:1081D000049B8531910530F59093C0148093BF14B2
:1081E00042E050E062E070E08FEB94E10E94B29FC9
:1081F00060917E0270917F0280E090E00E94179C67
:10820000009709F43FC00E94049B9093BE14809392
:10821000BD1442E050E060E070E08DEB94E10E941C
:10822000B29F30C084EA95E09F938F930E94FB9C9D
:108230000F900F9027C08091C0148F938091BF142E
:108240008F938BE995E09F938F930E94FB9C04EBA7
:1082500012E11F930F930E94FB9C8091BE148F9399
:108260008091BD148F938CE895E09F938F930E942B
:10827000FB9C1F930F930E94FB9C0FB6F894DEBFEC
:108280000FBECDBF84EB92E19F938F930E94FB9C26
:108290000F900F900C94074F60917E0270917F02B7
:1082A00080E090E00E94179C8C016AEF74E00E94CD
:1082B000389C892B09F077C060917E0270917F0213
:1082C00080E090E00E94179C8C01009711F40C94C0
:1082D000074F6FE67AE00E94389C892BB1F482E266
:1082E0009FEFACECBBE38093850290938602A09352
:1082F0008702B093880244E050E06EE470E085E8C5
:1083000092E00E94B29F0C94074F68E076E0C801AB
:108310000E94389C892BB1F482E29FEFACECBAE367
:108320008093850290938602A0938702B09388027F
:1083300044E050E06EE470E085E892E00E94B29F75
:108340000C94074FC8010E94009B2B013C0120E0C8
:1083500030E0A9010E94EB948823D9F081E00E94CB
:1083600058109B01AC01C301B2010E94F0946093CC
:10837000850270938602809387029093880244E07E
:1083800050E06EE470E085E892E00E94B29F0C94A9
:10839000074F8FE795E09F938F930E94FB9C0F9070
:1083A0000F900C94074F6DEF74E0C8010E94389C49
:1083B000892B09F077C060917E0270917F0280E086
:1083C00090E00E94179C8C01009711F40C94074FC9
:1083D0006FE67AE00E94389C892BB1F482E29FEF2D
:1083E000ACECBBE38093810290938202A093830262
:1083F000B093840244E050E06AE470E081E892E0E7
:108400000E94B29F0C94074F68E076E0C8010E947A
:10841000389C892BB1F482E29FEFACECBAE38093F5
:10842000810290938202A0938302B093840244E07D
:1084300050E06AE470E081E892E00E94B29F0C9400
:10844000074FC8010E94009B2B013C0120E030E057
:10845000A9010E94EB948823D9F082E00E94581071
:108460009B01AC01C301B2010E94F09460938102B0
:1084700070938202809383029093840244E050E0E0
:108480006AE470E081E892E00E94B29F0C94074F8A
:1084900082E795E09F938F930E94FB9C0F900F9033
:1084A0000C94074F65EF74E0C8010E94389C892B3B
:1084B00009F073C060917E0270917F0280E090E0CD
:1084C0000E94179C8C01009711F40C94074F6FE6E3
:1084D0007AE00E94389C892BB1F487ED94E3AFEEEB
:1084E000BCE38093890290938A02A0938B02B0939D
:1084F0008C0244E050E062E570E089E892E00E947E
:10850000B29F0C94074F68E076E0C8010E94389C47
:10851000892B51F483E695E09F938F930E94FB9CF7
:108520000F900F900C94074FC8010E94009B2B01E5
:108530003C0120E030E0A9010E94EB94882319F16E
:1085400080E00E9458104B015C0121EE3AE744E9BB
:108550005EE3C301B2010E940C94A50194010E9444
:10856000F0946093890270938A0280938B029093B7
:108570008C0244E050E062E570E089E892E00E94FD
:10858000B29F0C94074F86E595E09F938F930E94CE
:10859000FB9C0F900F900C94074F0E94A6109F9386
:1085A0008F937F936F938FE495E09F938F930E94B7
:1085B000FB9C82E00E94581020918102309182023F
:1085C00040918302509184020E949C97162F072F9E
:1085D000F82EE92E81E00E945810EF92FF920F933F
:1085E0001F9320918502309186024091870250911D
:1085F00088020E949C979F938F937F936F9383E44D
:1086000095E09F938F930E94FB9C84EB92E19F9354
:108610008F930E94FB9C0FB6F894DEBF0FBECDBFB8
:108620000C94074F60917E0270917F0280E090E091
:108630000E94179C009711F10E94AD2A0091C91465
:108640001091CA142091CB143091CC14601771078B
:108650008207930769F16093C9147093CA148093D9
:10866000CB149093CC1444E050E06AE570E089ECC0
:1086700094E10E94B29F82EB97E002C08BEA97E000
:108680009F938F930E94FB9C6091C9147091CA14B0
:108690008091CB149091CC140E94BA2984EB92E182
:1086A0009F938F930E94FB9C0F900F900F900F90C1
:1086B00080EA97E09F938F930E94FB9C6FEF7FEF80
:1086C000CB010E94BA2984EB92E19F938F930E9481
:1086D000FB9C0F900F900F900F900C94074F0E94EF
:1086E0008F260C94074FF3018481843329F440E0F2
:1086F00061E080E00E949F1880918002882311F43D
:108700000C94074F1F928F938DE997E09F938F935F
:108710000E94FB9C0F900F900F900F900C94074FAE
:10872000F3018481893709F080C060917E027091E5
:108730007F0280E090E00E94179C8C0163E97AE060
:108740000E94389C892B51F48091660290916702B7
:10875000A0916802B0916902906410C06FE575E065
:10876000C8010E94389C892BD1F4809166029091B7
:108770006702A0916802B09169029F7B80936602B4
:1087800090936702A0936802B093690244E050E0BE
:108790006EE170E086E692E00E94B29F46C06DE016
:1087A00076E0C8010E94389C892B21F58091F81D44
:1087B0008F938091F71D8F938091F61D8F938091F9
:1087C000F51D8F938091F41D8F938091F31D8F93EE
:1087D0008091F21D8F938091F11D8F9388E195E038
:1087E0009F938F930E94FB9C0FB6F894DEBF0FBE41
:1087F000CDBF1BC08091660290916702A091680274
:10880000B091690296FF03C083E99AE002C08FE548
:1088100095E09F938F9384E195E09F938F930E94BF
:10882000FB9C0F900F900F900F90809180028823F7
:1088300011F40C94074F1F928F938AE997E09F934E
:108840008F930E94FB9C0F900F900F900F900C94B1
:10885000074FF30184818737E9F560917E027091BB
:108860007F0280E090E00E94179C0097D9F00E9460
:10887000009B2B013C0120E030E0A9010E94EB9419
:10888000882381F040928D0250928E0260928F0276
:108890007092900244E050E066E570E08DE892E06E
:1088A0000E94B29F809190028F9380918F028F934C
:1088B00080918E028F9380918D028F9386E095E058
:1088C0009F938F930E94FB9C0F900F900F900F909F
:1088D0000F900F9080918002882311F40C94074F21
:1088E0001F928F9387E997E09F938F930E94FB9C41
:1088F0000F900F900F900F900C94074F60917E0295
:1089000070917F0280E090E00E94179C8C0163E9E7
:108910007AE00E94389C4090660250906702609016
:10892000680270906902892B19F4689457F809C09D
:108930006FE575E0C8010E94389C892B99F4E89492
:1089400057F84092660250926702609268027092F5
:10895000690244E050E06EE170E086E692E00E9439
:10896000B29F13C057FE03C083E99AE002C08FE5AF
:1089700095E09F938F9382E095E09F938F930E9461
:10898000FB9C0F900F900F900F9080918002882396
:1089900011F40C94074F1F928F9384E997E09F93F3
:1089A0008F930E94FB9C0F900F900F900F900C9450
:1089B000074F60917E0270917F0280E090E00E94FC
:1089C000179C8C0163E176E00E94389C892B11F49E
:1089D00089E108C067E176E0C8010E94389C892BD4
:1089E00049F480E18093C4001092C50082E0809336
:1089F000C00055C06BE176E0C8010E94389C892B0D
:108A000011F488E0EFCF60E276E0C8010E94389C64
:108A1000892B39F065E276E0C8010E94389C892BE9
:108A200011F483E0DFCF8091C400893141F48DEFF0
:108A300094E09F938F930E94FB9C0F900F908091E6
:108A4000C400803141F488EF94E09F938F930E949B
:108A5000FB9C0F900F908091C400883041F482EF0E
:108A600094E09F938F930E94FB9C0F900F908091B6
:108A7000C400833041F48CEE94E09F938F930E9466
:108A8000FB9C0F900F908091C400883041F486EEDB
:108A900094E09F938F930E94FB9C0F900F90809186
:108AA0008002882311F40C94074F1F928F9381E961
:108AB00097E09F938F930E94FB9C0F900F900F90D5
:108AC0000F900C94074F60917E0270917F0280E0BE
:108AD00090E00E94179C6FE67AE00E94389C892BF8
:108AE00011F481E001C080E00E947729809180022A
:108AF000882311F40C94074F1F928F938EE897E010
:108B00009F938F930E94FB9C0F900F900F900F905C
:108B10000C94074F0E94962780918002882311F4BD
:108B20000C94074F1F928F938BE897E09F938F933E
:108B30000E94FB9C0F900F900F900F900C94074F8A
:108B40000E94922780918002882311F40C94074F91
:108B50001F928F9388E897E09F938F930E94FB9CCE
:108B60000F900F900F900F900C94074F60917E0222
:108B700070917F0280E090E00E94179C0E94049B0D
:108B8000803170F48093C6140E946A7441E050E012
:108B90006DE170E086EC94E10E94B29F0C94074F67
:108BA0008091C6141F928F938CED94E09F938F93C6
:108BB0000E94FB9C0F900F900F900F900C94074F0A
:108BC00060917E0270917F0280E090E00E94179C8D
:108BD0000E94049B95EF980F903170F4809365028A
:108BE0000E94577341E050E06CE170E085E692E04E
:108BF0000E94B29F0C94074F809165021F928F9341
:108C000083ED94E09F938F930E94FB9C0F900F90B5
:108C10000F900F900C94074F60917E0270917F022D
:108C200080E090E00E94179C009789F04AE050E0B5
:108C3000BC0180EE9DE10E94489C4AE050E064E067
:108C400070E080EE9DE10E94B29F0C94074F80EE91
:108C50009DE19F938F938AE296E09F938F930E946A
:108C6000E79C0F900F900F900F900C94074F60911E
:108C70007E0270917F0280E090E00E94179C8C0140
:108C800060E873E00E94389C892BE1F4219A80917E
:108C9000660290916702A0916802B09169028061BA
:108CA0008093660290936702A0936802B093690272
:108CB00044E050E06EE170E086E692E00E94B29FF0
:108CC0000C94074F6EEF74E0C8010E94389C892B0A
:108CD000E1F4229A8091660290916702A091680265
:108CE000B091690280628093660290936702A093BC
:108CF0006802B093690244E050E06EE170E086E6FD
:108D000092E00E94B29F0C94074F62E673E0C801A4
:108D10000E94389C892BE1F4239A809166029091FD
:108D20006702A0916802B091690280648093660234
:108D300090936702A0936802B093690244E050E008
:108D40006EE170E086E692E00E94B29F0C94074FBD
:108D500061EA74E0C8010E94389C892BE1F4239AEF
:108D60008091660290916702A0916802B0916902B9
:108D700080688093660290936702A0936802B09324
:108D8000690244E050E06EE170E086E692E00E9405
:108D9000B29F0C94074F6AE573E0C8010E94389CAB
:108DA000892B79F581E08093313289EF9DE19093B1
:108DB00033328093323210923532109234328091B5
:108DC000660290916702A0916802B0916902916079
:108DD0008093660290936702A0936802B093690241
:108DE00044E050E06EE170E086E692E00E94B29FBF
:108DF00041E352E362E182E492E00E94167A0C942D
:108E0000074F69E873E0C8010E94389C892B21F55F
:108E1000E9E2FEE189E49EE1119211928E179F072B
:108E2000D9F78091660290916702A0916802B09193
:108E3000690292608093660290936702A093680231
:108E4000B093690244E050E06EE170E086E692E0A3
:108E50000E94B29F0C94074F6FE575E0C8010E9415
:108E6000389C40916602509167026091680270914F
:108E70006902892BC1F44F705C7F40936602509366
:108E8000670260936802709369022B9A44E050E095
:108E90006EE170E086E692E00E94B29F8091D63645
:108EA0000E946573B4C744FF03C083E99AE002C01F
:108EB0008FE595E09F938F9388EC94E09F938F9339
:108EC0000E94FB9C809166020F900F900F900F9074
:108ED00085FF03C083E99AE002C08FE595E09F9388
:108EE0008F938DEB94E09F938F930E94FB9C8091D6
:108EF00066020F900F900F900F9086FF03C083E9DA
:108F00009AE002C08FE595E09F938F9382EB94E007
:108F10009F938F930E94FB9C809166020F900F900D
:108F20000F900F9087FF03C083E99AE002C08FE59E
:108F300095E09F938F9387EA94E09F938F930E948D
:108F4000FB9C8091660290916702A0916802B091AB
:108F500069020F900F900F900F9090FF03C083E96C
:108F60009AE002C08FE595E09F938F938CE994E09F
:108F70009F938F930E94FB9C809166029091670261
:108F8000A0916802B09169020F900F900F900F901E
:108F900091FF03C083E99AE002C08FE595E09F93BB
:108FA0008F9381E994E09F938F930E94FB9C809123
:108FB000660290916702A0916802B09169020F90D9
:108FC0000F900F900F9091FF22C782E396E00E94CE
:108FD000239D99E2E92E9EE1F92E0BE010E02AE3B1
:108FE000822E26E0922EF70180819181F2E0EF0E31
:108FF000F11C9F938F931F930F939F928F920E94C8
:10900000E79C0F5F1F4F0F900F900F900F900F90E6
:109010000F900B31110539F7FAC684E897E09F935A
:109020008F930E94FB9C809180020F900F90882369
:1090300061F01F928F9381E897E09F938F930E9436
:10904000FB9C0F900F900F900F90F89498E088E1A0
:109050000FB6F894A895809360000FBE90936000BF
:10906000FFCF0E946266D3C660917E0270917F023C
:1090700080E090E00E94179C8C0163E97AE00E94F6
:10908000389C892BE9F40E945B7280916602909172
:109090006702A0916802B09169028D7F8160809320
:1090A000660290936702A0936802B093690244E05D
:1090B00050E06EE170E086E692E00E94B29FA7C6A3
:1090C0006FE575E0C8010E94389C892BE1F40E948D
:1090D00092718091660290916702A0916802B091AE
:1090E00069028C7F8093660290936702A093680266
:1090F000B093690244E050E06EE170E086E692E0F1
:109100000E94B29F84C665E476E0C8010E94389C44
:10911000892BE9F40E949271809166029091670216
:10912000A0916802B09169028E7F8260809366028E
:1091300090936702A0936802B093690244E050E004
:109140006EE170E086E692E00E94B29F60C6809178
:10915000660281FF0FC085E496E09F938F938DE8B0
:1091600094E09F938F930E94FB9C0F900F900F9021
:109170000F904DC680FF03C083E99AE002C08FE5DF
:1091800095E09F938F9389E894E09F938F930E943B
:10919000FB9C0F900F900F900F9039C680912F324B
:1091A0008F9380912E328F9380912D328F93809167
:1091B0002C328F9380912B328F9380912A328F9310
:1091C000809129328F93809128328F93809127321A
:1091D0008F93809126328F93809125328F93809147
:1091E00024328F93809123328F93809122328F93F8
:1091F000809121328F93809120328F9385E597E083
:109200009F938F930E94FB9C84EB92E19F938F939B
:109210000E94FB9C809180020FB6F894DEBF0FBEC7
:10922000CDBF882309F4F3C51F928F9382E597E0A1
:109230009F938F930E94FB9C0F900F900F900F9025
:10924000E6C5F89489E021E030E0F9018093570009
:10925000C895E02C20E030E0F90180935700C895D4
:10926000F02C7894F89423E030E0F90180935700D3
:10927000C895002D22E030E0F90180935700C89591
:10928000102D78948091092A8F938091082A8F93CA
:109290008091072A8F938091062A8F9388E497E024
:1092A0009F938F930E94FB9C1F92EF921F92FF92BD
:1092B0001F920F931F921F9381E297E09F938F93CA
:1092C0000E94FB9C0E943028809166001F928F9321
:1092D00085E197E09F938F930E94FB9C84EB92E142
:1092E0009F938F930E94FB9C809180020FB6F8940D
:1092F000DEBF0FBECDBF882309F489C51F928F93AF
:1093000082E197E09F938F930E94FB9C0F900F90B8
:109310000F900F907CC560E070E080E090E00E94CC
:10932000BE1160E070E081E090E00E94BE1180918B
:109330008002882309F46BC51F928F938FE097E01A
:109340009F938F930E94FB9C0F900F900F900F9014
:109350005EC50E9452263F922F920E94FB9C8091F4
:1093600080020F900F90882309F451C51F928F93AC
:109370008CE097E09F938F930E94FB9C0F900F903F
:109380000F900F9044C560917E0270917F0280E043
:1093900090E00E94179C62E076E00E94389C892B46
:1093A00031F5F8948BEB9BE00E94ED7A8C01892BD0
:1093B00069F0C8010F960E94CE78B80188E092E06B
:1093C0000E94687CC8010E944E7BF0CF8BEB9BE033
:1093D0000E94417B892B29F08BEB9BE00E94017B53
:1093E000F5CF8BEB9BE00E94E97A789436C08BEB4B
:1093F0009BE00E94ED7A8C018AE4E82E86E0F82E4C
:109400000115110551F1F80186811F928F93808516
:109410001F928F9385811F928F9381851F928F93C7
:1094200087811F928F9384811F928F9383811F92D4
:109430008F9382811F928F9382851F928F93FF92C9
:10944000EF920E94E79CC8010E944E7B8C010FB6F0
:10945000F894DEBF0FBECDBFD3CF809180028823AA
:1094600009F4D5C41F928F9389E097E09F938F935F
:109470000E94FB9C0F900F900F900F90C8C46091BA
:109480007E0270917F0280E090E00E94179C69E864
:1094900076E00E94389C892B09F0B9C40E945937A4
:1094A000B6C460917E0270917F0280E090E00E94DD
:1094B000179C8C0160E976E00E94389C892BD1F4DE
:1094C0008091660290916702A0916802B091690252
:1094D000977F8093660290936702A0936802B0938F
:1094E000690244E050E06EE170E086E692E00E949E
:1094F000B29F8DC468E076E0C8010E94389C892B39
:10950000D1F48091660290916702A0916802B091B7
:10951000690298608093660290936702A093680244
:10952000B093690244E050E06EE170E086E692E0BC
:109530000E94B29F6CC40E943A0E69C460917E0280
:1095400070917F0280E090E00E94179C8C0164E0A3
:1095500077E00E94039C892B19F40E94013057C4C4
:10956000F80180818332D1F44AE050E060E070E09D
:10957000C80101960E94C5987B836A8360917E0230
:1095800070917F0280E090E00E94179C8C012A81FC
:109590003B81243031050CF09EC002C01B821A8230
:1095A0000115110509F497C01982BE016F5F7F4F45
:1095B000C8010E943E3019013A014B01B82FA92F72
:1095C0008AE02A813B81829FF001839FF00D112464
:1095D000E750F24E4080518032813C8383818D83FD
:1095E00094819E8325812F8336813887878189875F
:1095F0009101A301B4018B2F9A2F5201CC80DD8001
:10960000EE80FF80088519850E94F79309F466C0F3
:109610008981811103C0208231822AC0181684F406
:10962000422853289C81692A2D81722A3E81832AEF
:109630008F81982A9885B92B2985A22B408217C043
:10964000209430946094709480949094B095A095F8
:10965000242053203C8163228D8178229E8189229F
:109660002F8192223885B3238985A82320825182B5
:109670006282738284829582B683A78348E250E037
:1096800062E270E089EF9DE10E94B29F8CEF96E06C
:109690009F938F930E94FB9C8AE02A813B81829F4B
:1096A000F001839FF00D1124E750F24E20813181AB
:1096B0004281538164817581868197810E94662BE6
:1096C00084EB92E19F938F930E94FB9C0F900F90ED
:1096D0000F900F9003C082E00E94EF3180EF96E080
:1096E0009F938F930E94FB9C2FEF3FEF4FEF5FEF15
:1096F0006FEF7FEF8FEF9FEF0E94662B84EB92E17D
:109700009F938F930E94FB9C809180020F900F90FB
:109710000F900F90882309F47AC31F928F938DEED8
:1097200096E09F938F930E94FB9C0F900F900F9059
:109730000F906DC360917E0270917F0280E090E097
:109740000E94179CFC0120812332A1F44AE050E0E2
:1097500060E070E001960E94C5988B0160917E02E6
:1097600070917F0280E090E00E94179C0430110508
:10977000ECF402C000E010E00097C1F04AE050E0D5
:1097800060E070E00E94F3992AE0209FF001219FA1
:10979000F00D1124E750F24E7187608748E250E0E7
:1097A00062E270E089EF9DE10E94B29F81E00E9439
:1097B000EF3180918002882309F429C31F928F938F
:1097C0008AEE96E09F938F930E94FB9C0F900F90E0
:1097D0000F900F901CC30E94577B809180028823BA
:1097E00009F415C31F928F9387EE96E09F938F9392
:1097F0000E94FB9C0F900F900F900F9008C30E9447
:10980000C13280918002882309F401C31F928F9393
:1098100084EE96E09F938F930E94FB9C0F900F9095
:109820000F900F90F4C280E090E00E944C2880914D
:109830008002882309F4EBC21F928F9381EE96E099
:109840009F938F930E94FB9C0F900F900F900F900F
:10985000DEC28091162E81FF2DC00E94D825892B53
:1098600049F580910D2A8F9380910C2A8F938091D6
:109870000B2A8F9380910A2A8F9386ED96E09F930F
:109880008F930E94FB9C8091FA368F938091F936DA
:109890008F938091F8368F938091F7368F9389EC70
:1098A00096E09F938F930E94FB9C0FB6F894DEBFC7
:1098B0000FBECDBF84EB92E19F938F930E94FB9CE0
:1098C0008091162E9091172E0F900F9093FF63C0EA
:1098D00081E090E00E9450251B012C0180E090E087
:1098E0000E9450257B018C010E94AE245F924F9212
:1098F0003F922F9288EB96E09F938F930E94FB9C60
:109900001F930F93FF92EF9288EA96E09F938F93B5
:109910000E94FB9C370148019701A8017101820157
:10992000B101C2010E944B239F938F937F936F934A
:109930008DE996E09F938F930E94FB9C262D372DF7
:10994000482D592D622D7F2D842D912F0E94AC23FF
:109950009F938F937F936F938FE896E09F938F935E
:109960000E94FB9C262D372D482D592D622D7F2DD1
:10997000842D912F0E9411249F938F937F936F9337
:109980008CE796E09F938F930E94FB9C0FB6F89410
:10999000DEBF0FBECDBF84EB92E19F938F930E94F9
:1099A000FB9C809180020F900F90882309F42FC2B6
:1099B0001F928F9389E796E09F938F930E94FB9C61
:1099C0000F900F900F900F9022C28091162E82FF61
:1099D00043C021E048E061E083E00E94051A8091E5
:1099E000FD1E8F938091FC1E8F938091FB1E8F93A1
:1099F0008091FA1E8F938091F91E8F938091F81EAB
:109A00008F938091F71E8F938091F61E8F9382E63D
:109A100096E09F938F930E94FB9C3F922F920E940F
:109A2000FB9C8091F51E8F938091F41E8F93809103
:109A3000F31E8F938091F21E8F9384E596E09F939F
:109A40008F930E94FB9C3F922F920E94FB9C0FB62B
:109A5000F894DEBF0FBECDBF8091162E85FF5CC08F
:109A600081E00E944A696091EA367091EB368091FC
:109A7000EC369091ED360E94A49520E030E048EC61
:109A800052E40E94F0949F938F937F936F9383E6A9
:109A900095E09F938F930E94E79C6091EE367091C2
:109AA000EF368091F0369091F1360E94A29520E039
:109AB00030E040E85AE30E949C979F938F937F93F6
:109AC0006F9382E795E09F938F930E94E79C60914C
:109AD000F2367091F3368091F4369091F5360E940B
:109AE000A29520E030E040E85BE30E949C979F93C2
:109AF0008F937F936F9383E895E09F938F930E945A
:109B0000E79C84EB92E19F938F930E94FB9C0FB69E
:109B1000F894DEBF0FBECDBF8091162E9091172E08
:109B200094FF3FC00E946A1E20E030E048EC52E4FF
:109B3000162F072FF82EE92E0E949C9720E836EE6C
:109B400045EC57E40E94F09421E03EED42E45EE3F0
:109B50000E9409989B01AC0160E070E080E89FE3FF
:109B60000E940C942BE43AE34DEB57E30E94F094EF
:109B70009F938F937F936F93EF92FF920F931F9317
:109B80008BE396E09F938F930E94FB9C84EB92E182
:109B90009F938F930E94FB9C0FB6F894DEBF0FBE7D
:109BA000CDBF80918002882309F431C11F928F9329
:109BB00088E396E09F938F930E94FB9C0F900F90F9
:109BC0000F900F9024C160917E0270917F0280E01F
:109BD00090E00E94179C65E976E00E94389C892BF2
:109BE00099F460917E0270917F0280E090E00E9483
:109BF000179C009709F40BC10E94049B909152019D
:109C0000892B8093520103C1809152018F701F9262
:109C10008F938CE794E09F938F930E94FB9C84EB3F
:109C200092E19F938F930E94FB9C0F900F900F9057
:109C30000F900F900F90EBC060917E0270917F02A9
:109C400080E090E00E94179C009711F14AE050E0FC
:109C500060E070E00E94C598603198F460936402FF
:109C60001F926F938BE296E09F938F930E94FB9CD1
:109C700041E050E06BE170E084E692E00E94B29F28
:109C800011C0809164021F928F9382E296E006C019
:109C9000809164021F928F9389E196E09F938F9346
:109CA0000E94FB9C0F900F900F900F9084EB92E11D
:109CB0009F938F930E94FB9C809180020F900F9046
:109CC000882309F4A4C01F928F9386E196E09F93A6
:109CD0008F930E94FB9C0F900F900F900F9097C056
:109CE00060917E0270917F0280E090E00E94179C5C
:109CF0008C0163E97AE00E94389C892BE1F40E9490
:109D000087708091660290916702A0916802B0917D
:109D1000690290618093660290936702A093680243
:109D2000B093690244E050E06EE170E086E692E0B4
:109D30000E94B29F6CC06FE575E0C8010E94389C1C
:109D4000892B99F5F8940E9494700FB6F894A89511
:109D500080916000886180936000109260000FBE67
:109D600084B7877F84BF80916000886180936000A2
:109D70001092600078948091660290916702A091A1
:109D80006802B09169029F7E809366029093670299
:109D9000A0936802B093690244E050E06EE170E085
:109DA00086E692E00E94B29F32C06AE976E0C8017E
:109DB0000E94389C4091660250916702609168024F
:109DC00070916902892B69F454FF02C0F894FFCFA7
:109DD0008BE694E09F938F930E94FB9C0F900F90D3
:109DE00016C054FF03C083E99AE002C08FE595E0F6
:109DF0009F938F9387E694E09F938F930E94FB9CA1
:109E00000F900F900F900F9002C00E947626EA8567
:109E1000FB851182108283E02B960FB6F894DEBF8B
:109E20000FBECDBFDF91CF911F910F91FF90EF90AB
:109E3000DF90CF90BF90AF909F908F907F906F906A
:109E40005F904F903F902F900895CF93DF93EC0158
:109E500088819981009741F0853B924109F4A0C027
:109E60001982188283E0A7C00E943D388091660263
:109E700080FD05C081FF01C01D9B0E9492718091F1
:109E800070008C7F809370008091B6008062809318
:109E9000B6001092B20082E08093B1008091B600CB
:109EA0008770E1F78091700081608093700068E5B1
:109EB0007EE080E090E00E9461700E94922780E046
:109EC0000E94772981E993E19F938F930E94FB9CE5
:109ED0000E94C3160F900F90809104379091053720
:109EE000892B51F48FE793E19F938F930E94FB9C02
:109EF0000E9459370F900F908091162E9091172E37
:109F000091FD0E940E668091162E9091172E93FD62
:109F10000E9466248091162E9091172E92FF06C003
:109F200021E04CE061E080ED0E94B1668091C614B2
:109F30000E946A74809165020E9457730E94547354
:109F40008093AB0B809165020E9457738091C61479
:109F50001F928F938091AB0B1F928F938FE996E0A6
:109F60009F938F930E94E79C1092AD0B1092AC0BC5
:109F70000F900F900F900F900F900F9086E592E04A
:109F80009093E9368093E83683E290E09093C21490
:109F90008093C11485EB92E19983888381E00BC0A3
:109FA0006332E1F745E452E360E070E08CEA9BE065
:109FB0000E94BE39E3CFDF91CF9108950F931F9395
:109FC000CF93DF93EC018A0188819981009711F189
:109FD0008A3C924121F01982188283E020C06231CC
:109FE000E9F4A80162E170E08CEA9BE00E94BE39CE
:109FF00084E08093CD361092CF361092CE361093F7
:10A00000D1360093D0364DEC56E362E182E492E023
:10A010000E94167A8AEC92E19983888381E0DF912D
:10A02000CF911F910F9108958436910514F19F935C
:10A030008F9385EF96E09F938F930E94E79C80918A
:10A04000203290912132A0912232B0912332019698
:10A05000A11DB11D8093203290932132A093223212
:10A06000B09323320F900F900F900F9081E090E00B
:10A07000089580E090E008952F923F924F925F9272
:10A080006F927F928F929F92AF92BF92CF92DF9208
:10A09000EF92FF920F931F93CF93DF93CDB7DEB76D
:10A0A000C959D1090FB6F894DEBF0FBECDBFCD564A
:10A0B000DF4F99838883C359D040F62E8A0123E865
:10A0C000621304C080EB9BE00E94957FCD56DF4F6A
:10A0D000A881B981C359D0408D919C918C35B2E152
:10A0E0009B0711F40C94B05F38F4009781F08E3424
:10A0F000904109F4FCC4F0C48E3622E1920709F4C1
:10A10000CAC48537924111F40C94B85FE5C449EE96
:10A1100059E061E870E080EB9BE00E947A7F8EE47A
:10A1200090E1B0C48C010F5F1F4FE3E0F0E0EC0F53
:10A13000FD1FE00FF11F1082C8010E941450892BEF
:10A1400071F720E030E040E050E0C157DF4F688118
:10A15000CF58D040627070E080E090E0A0E00E94B4
:10A16000009409F0C6C7C557DF4F2881CB58D040AF
:10A17000287030E040E050E060E070E080E090E087
:10A18000A0E00E94009499F127E04AE250E06BE2DF
:10A1900070E089E290E00E9495628FED96E30E9464
:10A1A0005B64BC01990F880B990B0E94A49520E079
:10A1B00030E048EC52E40E94F0949F938F937F9399
:10A1C0006F9388E397E09F938F931F9287E78F9316
:10A1D000CE01800F911F03969F938F930E94539DF2
:10A1E000080F191F0FB6F894DEBF0FBECDBFC557BD
:10A1F000DF4F2881CB58D040207130E040E050E064
:10A2000060E070E080E090E0A0E00E940094E9F15E
:10A2100026E04AE250E06BE270E089E290E00E94C2
:10A22000956281E090E00E944F118093C51482E511
:10A230009EE10E945B64BC01990F880B990B0E9400
:10A24000A49520E030E048EC52E40E94F0949F9303
:10A250008F937F936F9382E497E09F938F931F92E6
:10A2600087E78F93C801029621E030E02C0F3D1F55
:10A27000820F931F9F938F930E94539D080F191F66
:10A280000FB6F894DEBF0FBECDBF2E2D30E040E0FC
:10A2900050E060E070E080E090E0A0E00E94009478
:10A2A00001F10E940B119F938F937F936F938DE425
:10A2B00097E09F938F931F9287E78F93C801029631
:10A2C000A1E0B0E0AC0FBD1F8A0F9B1F9F938F933F
:10A2D0000E94539D080F191F0FB6F894DEBF0FBEE2
:10A2E000CDBFC557DF4F2881CB58D040207430E018
:10A2F00040E050E060E070E080E090E0A0E00E948C
:10A30000009431F180911B328F9380911A328F9398
:10A31000809119328F93809118328F938BE597E05B
:10A320009F938F931F9287E78F93C801029621E036
:10A3300030E02C0F3D1F820F931F9F938F930E943D
:10A34000539D080F191F0FB6F894DEBF0FBECDBF87
:10A35000C557DF4F2881CB58D040207830E040E00F
:10A3600050E060E070E080E090E0A0E00E940094A7
:10A3700041F1F8948091C5369091C636A091C736C8
:10A38000B091C8367894BF93AF939F938F9389E62B
:10A3900097E09F938F931F9287E78F93C801029650
:10A3A000A1E0B0E0AC0FBD1F8A0F9B1F9F938F935E
:10A3B0000E94539D080F191F0FB6F894DEBF0FBE01
:10A3C000CDBF20E0C457DF4F3881CC58D04031702A
:10A3D00040E050E060E070E080E090E0A0E00E94AB
:10A3E000009409F098C620E0C457DF4F3881CC585C
:10A3F000D040327040E050E060E070E080E090E0FB
:10A40000A0E00E94009409F0E6C620E0C457DF4FA8
:10A410003881CC58D040347040E050E060E070E0CB
:10A4200080E090E0A0E00E94009409F005C720E0E1
:10A43000C457DF4F3881CC58D040387040E050E0EE
:10A4400060E070E080E090E0A0E00E94009409F0FD
:10A4500023C720E0C457DF4F3881CC58D04030713B
:10A4600040E050E060E070E080E090E0A0E00E941A
:10A47000009409F071C720E0C457DF4F3881CC58F1
:10A48000D040307240E050E060E070E080E090E06A
:10A49000A0E00E94009409F08FC720E030E040E087
:10A4A00050E0C157DF4F6881CF58D040647070E0F2
:10A4B00080E090E0A0E00E94009409F0ABC720E0AB
:10A4C000C956DF4F3881C759D04040E050E060E0C6
:10A4D00070E080E090E0A0E00E94009411F00C9405
:10A4E000785A20E0C856DF4F3881C859D04040E044
:10A4F00050E060E070E080E090E0A0E00E94009416
:10A5000011F00C94A75AC357DF4F5881CD58D04053
:10A510005170E52E20E030E0452F50E060E070E023
:10A5200080E090E0A0E00E94009411F00C94D65AD4
:10A5300020E030E0C357DF4F4881CD58D040427013
:10A5400050E060E070E080E090E0A0E00E940094C5
:10A5500011F00C940A5B20E030E04F2D50E060E0F9
:10A5600070E080E090E0A0E00E94009411F00C9474
:10A570003E5B20E030E040E050E0C157DF4F6881B3
:10A58000CF58D040687070E080E090E0A0E00E947A
:10A59000009411F00C94695B20E030E040E050E062
:10A5A000C157DF4F6881CF58D040607170E080E0C4
:10A5B00090E0A0E00E94009411F00C94955B20E0E4
:10A5C00030E040E050E060E0CE56DF4F7881C25985
:10A5D000D040717080E090E0A0E00E94009411F003
:10A5E0000C94C15B20E030E0C357DF4F4881CD5869
:10A5F000D040487050E060E070E080E090E0A0E083
:10A600000E94009411F00C94E75B20E030E0C35707
:10A61000DF4F4881CD58D040407150E060E070E09D
:10A6200080E090E0A0E00E94009411F00C941C5C8B
:10A6300020E030E0C357DF4F4881CD58D040407212
:10A6400050E060E070E080E090E0A0E00E940094C4
:10A6500011F00C94515C20E030E0C357DF4F48818B
:10A66000CD58D040407450E060E070E080E090E071
:10A67000A0E00E94009411F00C94865CC357DF4F59
:10A680005881CD58D0405078D52E20E030E0452F6D
:10A6900050E060E070E080E090E0A0E00E94009474
:10A6A00011F00C94BB5CC257DF4F8881CE58D0406C
:10A6B0008170C82E20E030E040E0582F60E070E06C
:10A6C00080E090E0A0E00E94009411F40C94CB5F35
:10A6D0008091162E82FF06C021E046E061E083E013
:10A6E0000E94051A20E030E04D2D50E060E070E05F
:10A6F00080E090E0A0E00E94009411F40C94035DCF
:10A700008091162E82FF02C00C94C85C20E030E0DD
:10A7100040E0C257DF4F5881CE58D040527060E0C1
:10A7200070E080E090E0A0E00E94009411F00C94B2
:10A73000385D20E030E040E0C257DF4F5881CE580E
:10A74000D040547060E070E080E090E0A0E00E94B3
:10A75000009411F00C946B5D20E030E040E0C257B3
:10A76000DF4F5881CE58D040507160E070E080E0FB
:10A7700090E0A0E00E94009411F00C949E5D20E017
:10A7800030E040E0C257DF4F5881CE58D040507281
:10A7900060E070E080E090E0A0E00E94009411F0A2
:10A7A0000C94DD5D20E030E040E0C257DF4F58817F
:10A7B000CE58D040507460E070E080E090E0A0E0BF
:10A7C0000E94009411F00C941C5E20E030E040E008
:10A7D000C257DF4F5881CE58D040587060E070E0CB
:10A7E00080E090E0A0E00E94009411F00C945B5E89
:10A7F00020E030E040E050E0C157DF4F6881CF58A3
:10A80000D040607270E080E090E0A0E00E94009490
:10A8100011F40C948C5E8091162E85FD02C00C9470
:10A820008C5E81E00E944A696091EA367091EB3655
:10A830008091EC369091ED360E94A49520E030E0B6
:10A8400048EC52E40E94F0949F938F937F936F9310
:10A8500081E099E09F938F931F9287E78F93C801C0
:10A860000296A1E0B0E0AC0FBD1F8A0F9B1F9F9323
:10A870008F930E94539D080F191FC8010E94145006
:10A880000FB6F894DEBF0FBECDBF892B09F047CCC1
:10A89000E1E020E030E040E050E0C157DF4F688168
:10A8A000CF58D040607470E080E090E0A0E00E945B
:10A8B000009411F00C948F5E20E030E040E050E016
:10A8C000C157DF4F6881CF58D040607870E080E09A
:10A8D00090E0A0E00E94009411F00C94D25E20E081
:10A8E00030E040E0C756DF4F5881C959D04060E0A2
:10A8F00070E080E090E0A0E00E94009411F00C94E1
:10A90000145F20E030E04E2D50E060E070E080E029
:10A9100090E0A0E00E94009411F00C94505FC557A5
:10A92000DF4F2881CB58D040C457DF4F3881CC58F7
:10A93000D040C357DF4F4881CD58D040C257DF4F7A
:10A940005881CE58D040C157DF4F6881CF58D04092
:10A95000CE56DF4F7881C259D040CB56DF4F888129
:10A96000C559D040CA56DF4F9881C659D040A0E0A3
:10A970000E94009411F00C947D5F809164028061CC
:10A9800089838091A40B8A83FE01E00FF11F13825B
:10A990008091C9149091CA14A091CB14B091CC1499
:10A9A000A8014D5F5F4F7A0180FF0CC0FF924F936B
:10A9B0008CE499E09F938F930E94E79C0F900F90F7
:10A9C0000F900F90B701CE0101960E94DA8080911E
:10A9D000660282FF0AC025EC32E3A701BE016F5F69
:10A9E0007F4F8EE692E00E9474658091C914909129
:10A9F000CA14A091CB14B091CC1482FD73980E941C
:10AA00005B7280EB9BE00E94977F80916602909141
:10AA10006702A0916802B091690290FD02C00C9497
:10AA2000615F0F5F1F4F0E945473E82E89E10E94FF
:10AA300065738091660290916702A0916802B0915F
:10AA4000690290FD02C00C945D5F73988091A40B25
:10AA50008F5F8093A40B8A83B8016F5F7F4FCE0115
:10AA600001960E94DA8080EB9BE00E94977F40E095
:10AA700050E065E880913316909134160E94167A62
:10AA80008CE592E1CD56DF4FA881B981C359D04002
:10AA90008D939C931EC088E99BE00E94E777892BE9
:10AAA000C1F00E945B728091660287FD2B9840E4A2
:10AAB00050E060E070E088E99BE00E94C97785E79C
:10AAC00092E1CD56DF4FE881F981C359D04091839F
:10AAD000808381E00C94DB5FCD56DF4FA881B98184
:10AAE000C359D0401D921C9283E00C94DB5FB2E10D
:10AAF000FB1669F080910A37F81211CBBAE00639DB
:10AB00001B0709F00CCB89E097E00E94239D809001
:10AB1000660290906702A0906802B090690291FC72
:10AB2000FECAF80180818130E1F50180F281E02DDB
:10AB30002081C557DF4F2883CB58D0403181C4577F
:10AB4000DF4F3883CC58D0404281C357DF4F488312
:10AB5000CD58D0405381C257DF4F5883CE58D04094
:10AB60008481C157DF4F8883CF58D0409581CE561E
:10AB7000DF4F9883C259D040A681CB56DF4FA883C0
:10AB8000C559D040B781CA56DF4FB883C659D040A7
:10AB900060847184C057DF4F19821882C059D04039
:10ABA00085C0823041F5F8010380F481E02DC05763
:10ABB000DF4FF983E883C059D040612C712CF1E05C
:10ABC000C557DF4FF883CB58D040C457DF4F1882AA
:10ABD000CC58D040C357DF4F1882CD58D04020E822
:10ABE000C257DF4F2883CE58D040C157DF4F18825D
:10ABF000CF58D0404CC0833039F1843009F08FCA2F
:10AC0000612C712CC057DF4F19821882C059D04077
:10AC100035E0C557DF4F3883CB58D040C457DF4F9E
:10AC20001882CC58D040C357DF4F1882CD58D0403F
:10AC3000C257DF4F1882CE58D04042E0C157DF4F95
:10AC40004883CF58D04023C0612C712CC057DF4FB0
:10AC500019821882C059D04055E0C557DF4F58833C
:10AC6000CB58D040C457DF4F1882CC58D040C35780
:10AC7000DF4F1882CD58D040C257DF4F1882CE58D0
:10AC8000D04081E0C157DF4F8883CF58D040CE56A7
:10AC9000DF4F1882C259D040CB56DF4F1882C559BA
:10ACA000D040CA56DF4F1882C659D04020908D023E
:10ACB00030908E0240908F0250909002C0901832D7
:10ACC000D0901932E0901A32F0901B322DEC3CEC0F
:10ACD0004CE45EE3C201B1010E940D94A70196010C
:10ACE0000E94EB9418165CF0E894A0F8809266023B
:10ACF00090926702A0926802B092690253C0A701C5
:10AD00009601C201B1010E94C99618160CF04AC002
:10AD10008091243290912532A0912632B091273231
:10AD20000196A11DB11D8093243290932532A093EA
:10AD30002632B0932732A0FCF2C96894A0F8809222
:10AD4000660290926702A0926802B092690295E44E
:10AD5000C557DF4F9883CB58D040A0E2C457DF4F90
:10AD6000A883CC58D040C357DF4F1882CD58D0406D
:10AD7000C257DF4F1882CE58D040B4E0C157DF4FE2
:10AD8000B883CF58D040CE56DF4F1882C259D0403A
:10AD9000CB56DF4F1882C559D040CA56DF4F1882B4
:10ADA000C659D040C357DF4FE881CD58D040E4703A
:10ADB000FE2E20E030E04E2F50E060E070E080E0BA
:10ADC00090E0A0E00E94009409F08C9AC557DF4FF4
:10ADD000F881CB58D040F072EF2E2F2F30E040E0BA
:10ADE00050E060E070E080E090E0A0E00E9400941D
:10ADF00011F00E940B11C457DF4F2881CC58D0406E
:10AE00002074C956DF4F2883C759D04020E0C95667
:10AE1000DF4F3881C759D04040E050E060E070E03B
:10AE200080E090E0A0E00E94009411F00E94D825FC
:10AE3000C457DF4F3881CC58D0403078C856DF4FE8
:10AE40003883C859D04020E040E050E060E070E036
:10AE500080E090E0A0E00E94009451F00E94A610D3
:10AE60006093D2367093D3368093D4369093D53690
:10AE7000C557DF4F2881CB58D040217030E040E0EB
:10AE800050E060E070E080E090E0A0E00E9400947C
:10AE9000F1F080EE9DE19F938F9388E197E09F937F
:10AEA0008F931F9287E78F93CE0103969F938F9383
:10AEB0000E94539D6C010E9414500FB6F894DEBF9F
:10AEC0000FBECDBF892B09F02AC9860102C000E060
:10AED00010E0C557DF4F2881CB58D040227030E0BA
:10AEE00040E050E060E070E080E090E0A0E00E9490
:10AEF0000094D9F1C801029660E277E0A1E0B0E0E9
:10AF0000AC0FBD1F8A0F9B1F0E94419C0D5F1F4FFE
:10AF10003FEDC32E36E3D32E47EE842E46E3942E28
:10AF200052E9A52E53E0B52E67E7562EF601819122
:10AF30006F011F928F93BF92AF921F925F92C801D1
:10AF4000029621E030E02C0F3D1F820F931F9F934C
:10AF50008F930E94539D080F191F0FB6F894DEBF00
:10AF60000FBECDBF8C149D0409F7C557DF4F288154
:10AF7000CB58D040247030E040E050E060E070E01A
:10AF800080E090E0A0E00E94009409F446C0C8016F
:10AF9000029664E277E0A1E0B0E0AC0FBD1F8A0F3B
:10AFA0009B1F0E94419C0C5F1F4F6E01BAE7CB0EA6
:10AFB000D11C80E1F60111928A95E9F728E0A601FB
:10AFC00068E980EB0E9489164601F8E08F0E911C1B
:10AFD00092E9A92E93E0B92E27E7522ED6018D9142
:10AFE0006D011F928F93BF92AF921F925F92C80123
:10AFF0000296E1E0F0E0EC0FFD1F8E0F9F1F9F9384
:10B000008F930E94539D080F191F0FB6F894DEBF4F
:10B010000FBECDBFC814D90409F7C257DF4F38811E
:10B02000CE58D0403078C756DF4F3883C959D0400A
:10B0300020E030E040E0C756DF4F5881C959D0408A
:10B0400060E070E080E090E0A0E00E940094E1F415
:10B050008091C7149091C8149F938F9389E297E0D1
:10B060009F938F931F9287E78F93CE01800F911F3D
:10B0700003969F938F930E94539D080F191F0FB63D
:10B08000F894DEBF0FBECDBF20E030E040E050E0DE
:10B09000C157DF4F6881CF58D040617070E080E0C9
:10B0A00090E0A0E00E94009409F44BC8E3E0F0E0D7
:10B0B000EC0FFD1FE00FF11F80E28083DE01A00F87
:10B0C000B11FBD016C5F7F4FE5E4F2E3055412430D
:10B0D0009F012D5F3F4FC8018E0F9F1F4381319607
:10B0E000442309F41FC8D9018C91DB018D93BD0164
:10B0F000EFCFCE01800F911F60E377E003960E94AF
:10B10000419C095F1F4FC8010E941450892B11F008
:10B110000C948F5028C86114710409F464C9F89420
:10B120002090C5363090C6364090C7365090C8360D
:10B13000789480914A1E90914B1EA0914C1EB09124
:10B140004D1EA2019101281B390B4A0B5B0BCA0152
:10B15000B9010E94A2954B015C01B30180E090E02F
:10B160000E94A2959B01AC01C501B4010E94F0941C
:10B17000B62EC72ED82EE92E9F938F937F936F9371
:10B1800084E797E09F938F931F9287E78F93CE0179
:10B19000800F911F03969F938F930E94539D080FDA
:10B1A000191F8B2D9C2DAD2DBE2D8093D7369093DE
:10B1B000D836A093D936B093DA3620924A1E309210
:10B1C0004B1E40924C1E50924D1E0FB6F894DEBF9F
:10B1D0000FBECDBF08C96114710409F416C9F894F3
:10B1E0008091211E9091221EA091231EB091241EB9
:10B1F00078949F938F9380916D028F9380916C02CE
:10B200008F9381E897E09F938F931F9287E78F93A7
:10B21000C8010296A1E0B0E0AC0FBD1F8A0F9B1FD2
:10B220009F938F930E94539D080F191F0FB6F89498
:10B23000DEBF0FBECDBFE9C8F8948091C9369091AA
:10B24000CA36A091CB36B091CC367894BF93AF93E9
:10B250009F938F9381E997E09F938F931F9287E746
:10B260008F93C801029621E030E02C0F3D1F820F22
:10B27000931F9F938F930E94539D080F191FC8011E
:10B280000E9414500FB6F894DEBF0FBECDBF892BBD
:10B2900011F00C948F50CBC86114710409F4D9C813
:10B2A000F8942090C9363090CA364090CB365090F2
:10B2B000CC36789480914E1E90914F1EA091501ED6
:10B2C000B091511EA2019101281B390B4A0B5B0B57
:10B2D000CA01B9010E94A2954B015C01B30180E053
:10B2E00090E00E94A2959B01AC01C501B4010E94AF
:10B2F000F094B62EC72ED82EE92E9F938F937F936E
:10B300006F938CE997E09F938F931F9287E78F93BA
:10B31000CE01800F911F03969F938F930E94539DA0
:10B32000080F191F8B2D9C2DAD2DBE2D8093DB3664
:10B330009093DC36A093DD36B093DE3620924E1E1D
:10B3400030924F1E4092501E5092511E0FB6F894EC
:10B35000DEBF0FBECDBF7DC8672809F48CC8F89446
:10B360008091251E9091261EA091271EB091281E27
:10B3700078949F938F9380916B028F9380916A0250
:10B380008F9389EA97E09F938F931F9287E78F931C
:10B39000C8010296A1E0B0E0AC0FBD1F8A0F9B1F51
:10B3A0009F938F930E94539D080F191F0FB6F89417
:10B3B000DEBF0FBECDBF5FC880911C3290911D32A1
:10B3C000A0911E32B0911F32BF93AF939F938F9382
:10B3D00089EB97E09F938F931F9287E78F93C80124
:10B3E000029621E030E02C0F3D1F820F931F9F93A8
:10B3F0008F930E94539D080F191FC8010E9414507B
:10B400000FB6F894DEBF0FBECDBF892B11F00C94A0
:10B410008F5043C8809127328F93809126328F932B
:10B42000809125328F93809124328F9380912332A3
:10B430008F93809122328F93809121328F938091CC
:10B4400020328F9384EC97E09F938F931F9287E72E
:10B45000E82EEF92C8010296A1E0B0E0AC0FBD1F4C
:10B460008A0F9B1F9F938F930E94539D080F191F54
:10B47000C8010E9414500FB6F894DEBF0FBECDBFB6
:10B48000892B11F00C948F508091162E9091172ECD
:10B4900093FF15C880912B328F9380912A328F931E
:10B4A000809129328F93809128328F9388EE97E094
:10B4B0009F938F931F92EF92C801029621E030E094
:10B4C0002C0F3D1F820F931F9F938F930E94539DBC
:10B4D000080F191FC8010E9414500FB6F894DEBF60
:10B4E0000FBECDBF892B11F00C948F500C945F527E
:10B4F00080910D2A8F9380910C2A8F9380910B2A33
:10B500008F9380910A2A8F938AEF97E09F938F936E
:10B510001F9287E78F93C8010296A1E0B0E0AC0FBD
:10B52000BD1F8A0F9B1F9F938F930E94539D080FEF
:10B53000191FC8010E9414500FB6F894DEBF0FBE49
:10B54000CDBF892B11F00C948F500C9471528091C7
:10B55000D5368F938091D4368F938091D3368F9345
:10B560008091D2368F9385E098E09F938F931F92BE
:10B5700087E78F93C801029621E030E02C0F3D1F32
:10B58000820F931F9F938F930E94539D080F191F43
:10B59000C8010E9414500FB6F894DEBF0FBECDBF95
:10B5A000892B11F00C948F500C94835281E00E94EF
:10B5B0005810209185023091860240918702509167
:10B5C00088020E949C979F938F937F936F9382E151
:10B5D00098E09F938F931F9287E78F93C8010296FD
:10B5E000A1E0B0E0AC0FBD1F8A0F9B1F9F938F930C
:10B5F0000E94539D080F191FC8010E9414500FB6D6
:10B60000F894DEBF0FBECDBF892B11F00C948F5084
:10B610000C94985282E00E9458102091810230913F
:10B62000820240918302509184020E949C979F93D2
:10B630008F937F936F938FE198E09F938F931F92E7
:10B6400087E78F93C801029621E030E02C0F3D1F61
:10B65000820F931F9F938F930E94539D080F191F72
:10B66000C8010E9414500FB6F894DEBF0FBECDBFC4
:10B67000892B11F00C948F500C94AB5283E00E94F4
:10B6800058109F938F937F936F938CE298E09F93D2
:10B690008F931F9287E78F93C8010296A1E0B0E0D5
:10B6A000AC0FBD1F8A0F9B1F9F938F930E94539DCA
:10B6B000080F191F8C98C8010E9414500FB6F894F7
:10B6C000DEBF0FBECDBF892B11F00C948F500C94B0
:10B6D000B952299903C08FE595E002C083E99AE049
:10B6E0009F938F9389E398E09F938F931F9287E7AF
:10B6F0008F93C801029621E030E02C0F3D1F820F8E
:10B70000931F9F938F930E94539D080F191FC80189
:10B710000E9414500FB6F894DEBF0FBECDBF892B28
:10B7200011F00C948F500C94CC522A9903C08FE5E1
:10B7300095E002C083E99AE09F938F9381E498E0BB
:10B740009F938F931F9287E78F93C8010296A1E082
:10B75000B0E0AC0FBD1F8A0F9B1F9F938F930E9479
:10B76000539D080F191FC8010E9414500FB6F8947A
:10B77000DEBF0FBECDBF892B11F00C948F500C94FF
:10B78000DF528EB31F928F9389E498E09F938F933B
:10B790001F9287E78F93C801029621E030E02C0FBB
:10B7A0003D1F820F931F9F938F930E94539D080FFD
:10B7B000191FC8010E9414500FB6F894DEBF0FBEC7
:10B7C000CDBF892B11F00C948F500C94F2528091C4
:10B7D000162E9091172E92FD02C00C94055321E075
:10B7E00042E161E080ED0E94B1669F938F937F9369
:10B7F0006F9388E598E09F938F931F9287E78F93CD
:10B80000C8010296A1E0B0E0AC0FBD1F8A0F9B1FDC
:10B810009F938F930E94539D080F191FC8010E9488
:10B8200014500FB6F894DEBF0FBECDBF892B11F0B8
:10B830000C948F500C9405538091162E9091172ED6
:10B8400092FD02C00C94185321E042E162E080EDC9
:10B850000E94B1669F938F937F936F9386E698E0E3
:10B860009F938F931F9287E78F93C801029621E0E1
:10B8700030E02C0F3D1F820F931F9F938F930E94E8
:10B88000539D080F191FC8010E9414500FB6F89459
:10B89000DEBF0FBECDBF892B11F00C948F500C94DE
:10B8A00018538091162E9091172E92FD02C00C9481
:10B8B0002B5321E042E163E080ED0E94B1669F934B
:10B8C0008F937F936F9384E798E09F938F931F925A
:10B8D00087E78F93C8010296A1E0B0E0AC0FBD1FCF
:10B8E0008A0F9B1F9F938F930E94539D080F191FD0
:10B8F000C8010E9414500FB6F894DEBF0FBECDBF32
:10B90000892B11F00C948F500C942B538091162E90
:10B910009091172E92FD02C00C943E5321E042E11B
:10B9200064E080ED0E94B1669F938F937F936F9345
:10B9300082E898E09F938F931F9287E78F93C801C7
:10B94000029621E030E02C0F3D1F820F931F9F9342
:10B950008F930E94539D080F191FC8010E94145015
:10B960000FB6F894DEBF0FBECDBF892B11F00C943B
:10B970008F500C943E538091162E82FD02C00C9481
:10B98000535346E061E083E00E94051A0C94535340
:10B990008091F91E8F938091F81E8F938091F71EEE
:10B9A0008F938091F61E8F9380E998E09F938F93F9
:10B9B0001F9287E78F93C8010296A1E0B0E0AC0F19
:10B9C000BD1F8A0F9B1F9F938F930E94539D080F4B
:10B9D000191FC8010E9414500FB6F894DEBF0FBEA5
:10B9E000CDBF892B11F00C948F5020E030E040E067
:10B9F0005C2D60E070E080E090E0A0E00E940094A8
:10BA000011F40C9486538091162E82FD02C00C9482
:10BA100086538091FD1E8F938091FC1E8F938091A1
:10BA2000FB1E8F938091FA1E8F9388E998E09F9375
:10BA30008F931F9287E78F93C801029621E030E031
:10BA40002C0F3D1F820F931F9F938F930E94539D36
:10BA5000080F191FC8010E9414500FB6F894DEBFDA
:10BA60000FBECDBF892B11F00C948F500C948653D0
:10BA70008091162E9091172E93FD02C00C9499532D
:10BA800080E090E00E9450259F938F937F936F9367
:10BA900083EA98E09F938F931F9287E78F93C80163
:10BAA0000296A1E0B0E0AC0FBD1F8A0F9B1F9F93D1
:10BAB0008F930E94539D080F191FC8010E941450B4
:10BAC0000FB6F894DEBF0FBECDBF892B11F00C94DA
:10BAD0008F500C9499538091162E9091172E93FDB0
:10BAE00002C00C94AC5381E090E00E9450259F93DB
:10BAF0008F937F936F9383EB98E09F938F931F9225
:10BB000087E78F93C801029621E030E02C0F3D1F9C
:10BB1000820F931F9F938F930E94539D080F191FAD
:10BB2000C8010E9414500FB6F894DEBF0FBECDBFFF
:10BB3000892B11F00C948F500C94AC538091162EDD
:10BB40009091172E93FD02C00C94BF5381E090E0BA
:10BB50000E9450254B015C0180E090E00E9450253E
:10BB60009B01AC01C501B4010E944B239F938F93AD
:10BB70007F936F9384EC98E09F938F931F9287E756
:10BB80008F93C8010296A1E0B0E0AC0FBD1F8A0FF1
:10BB90009B1F9F938F930E94539D080F191FC801ED
:10BBA0000E9414500FB6F894DEBF0FBECDBF892B94
:10BBB00011F00C948F500C94BF538091162E9091DD
:10BBC000172E93FD02C00C94D25381E090E00E94A6
:10BBD00050254B015C0180E090E00E9450259B01C4
:10BBE000AC01C501B4010E94AC239F938F937F9356
:10BBF0006F938FEC98E09F938F931F9287E78F93BB
:10BC0000C801029621E030E02C0F3D1F820F931FE8
:10BC10009F938F930E94539D080F191FC8010E9484
:10BC200014500FB6F894DEBF0FBECDBF892B11F0B4
:10BC30000C948F500C94D2538091162E9091172E05
:10BC400093FD02C00C94E55381E090E00E945025E2
:10BC50004B015C0180E090E00E9450259B01AC010B
:10BC6000C501B4010E9411249F938F937F936F931A
:10BC70008DED98E09F938F931F9287E78F93C80174
:10BC80000296A1E0B0E0AC0FBD1F8A0F9B1F9F93EF
:10BC90008F930E94539D080F191FC8010E941450D2
:10BCA0000FB6F894DEBF0FBECDBF892B11F00C94F8
:10BCB0008F500C94E5538091162E9091172E94FD81
:10BCC00002C00C94F8530E946A1E9F938F937F9337
:10BCD0006F9380EF98E09F938F931F9287E78F93E6
:10BCE000C801029621E030E02C0F3D1F820F931F08
:10BCF0009F938F930E94539D080F191FC8010E94A4
:10BD000014500FB6F894DEBF0FBECDBF892B11F0D3
:10BD10000C948F500C94F853E0E00C9449548091AB
:10BD2000162E85FD02C00C945C54E11103C081E025
:10BD30000E944A696091EE367091EF368091F0363C
:10BD40009091F1360E94A29520E030E040E85AE35D
:10BD50000E949C979F938F937F936F9382E199E0CA
:10BD60009F938F931F9287E78F93C801029621E0DC
:10BD700030E02C0F3D1F820F931F9F938F930E94E3
:10BD8000539D080F191FC8010E9414500FB6F89454
:10BD9000DEBF0FBECDBF892B11F00C948F50E1E0B8
:10BDA0000C945C548091162E85FD02C00C946F5447
:10BDB000E11103C081E00E944A696091F2367091FE
:10BDC000F3368091F4369091F5360E94A29520E0EA
:10BDD00030E040E85BE30E949C979F938F937F93B2
:10BDE0006F9384E299E09F938F931F9287E78F93DD
:10BDF000C8010296A1E0B0E0AC0FBD1F8A0F9B1FE7
:10BE00009F938F930E94539D080F191FC8010E9492
:10BE100014500FB6F894DEBF0FBECDBF892B11F0C2
:10BE20000C948F500C946F54C057DF4FA881B98188
:10BE3000C059D04016968C9116971F928F931596E5
:10BE40008C9115971F928F9313968C9113971F9235
:10BE50008F9312968C911F928F9385E399E09F9315
:10BE60008F931F9287E78F93C8010296E1E0F0E07D
:10BE7000EC0FFD1F8E0F9F1F9F938F930E94539D6A
:10BE8000080F191FC8010E9414500FB6F894DEBFA6
:10BE90000FBECDBF892B11F00C948F500C948154A0
:10BEA000779A8091C9149091CA14A091CB14B09143
:10BEB000CC1492FF22C0749A20C08E2D0E9465730C
:10BEC000739A8091C7149091C814892B11F00E9425
:10BED00092718091A40B8F5F8093A40B8091C91401
:10BEE0009091CA14A091CB14B091CC1482FD02C0E1
:10BEF0000C948F50739A0C948F508091C914909128
:10BF0000CA14A091CB14B091CC1482FD0CC08091C6
:10BF1000660280FD08C081FD02C00C94BD541D99CD
:10BF200002C00C94BD5440E050E060E070E0CE01EF
:10BF300001960E94C30E8091FF1E90E02091BF14D5
:10BF40003091C0148217930710F40C94BD5440E054
:10BF500050E062E180E192E00E94167A0C94BD54B8
:10BF6000E5E8FE120C94695500E010E00C941955B8
:10BF700088E99BE00E94E777892B11F40C946955BE
:10BF80000E9492718091660287FD02C00C948F50CE
:10BF90002B9A0C948F5020E030E04D2D50E060E063
:10BFA00070E080E090E0A0E00E94009411F00C941A
:10BFB00080530C948653C756DF4F0FB6F894DEBFFC
:10BFC0000FBECDBFDF91CF911F910F91FF90EF90EA
:10BFD000DF90CF90BF90AF909F908F907F906F90A9
:10BFE0005F904F903F902F9008950C947D7E4F92DC
:10BFF0005F926F927F929F92AF92BF92CF92DF92A9
:10C00000EF92FF920F931F93CF93DF93CDB7DEB7DD
:10C0100060970FB6F894DEBF0FBECDBF5B010E94E4
:10C020005473E82FF0E0EE0FFF1FED5EF14E8081BC
:10C0300091810196918380838091C9149091CA1453
:10C04000A091CB14B091CC1481FD749840906602FD
:10C050005090670260906802709069020E9431807F
:10C060006C01FC018081982F92959F70913099F41A
:10C070008F7051F48091F71D9091F81D0196909367
:10C08000F81D8093F71D3EC1B50181E499E30E943C
:10C090004E81892B51F08091F51D9091F61D0196EE
:10C0A0009093F61D8093F51D2DC1D301C2013EE092
:10C0B000B695A795979587953A95D1F7F82FF17092
:10C0C0009F2E8BEB9BE00E94ED7A7C01892B09F47B
:10C0D0004BC0B501C70102960E944E81892B09F41D
:10C0E0003FC0870122E73EE040E054E660E070E0B8
:10C0F000C7010F960E949678F6019181F70184811D
:10C10000981321C082858F5F82878091F31D909163
:10C11000F41D01969093F41D8093F31D84E00E941A
:10C120001A81F701208530E02817390708F07AC115
:10C1300084E00E941A81F7018087F60180818F7068
:10C14000F7018187DFC0F701128684E00E941A811F
:10C15000F7018087F60180818F70F701818763C1C5
:10C16000C7010E944E7BB1CF88E092E00E94437CE1
:10C170007C01892B09F4C6C0B501C70102960E9453
:10C180004781F60181818150F701848380E091E04D
:10C19000A0E0B0E083879487A587B687128684E005
:10C1A0000E941A81F7018087F60180818F70F70164
:10C1B0008187B7018BEB9BE00E94287B870122E7F8
:10C1C0003EE040E054E660E070E0C7010F960E9458
:10C1D000967811E0F6018181F7018483F601808170
:10C1E0008F70F701878384E00E941A81F7018583AD
:10C1F00083E00E941A81F701868387818F3009F0DE
:10C2000010E0F6014180F7018481481A512C612C1D
:10C21000712C86E0440C551C661C771C8A95D1F75E
:10C220002385348545855685A0ECB0E00E945F9259
:10C23000BB27A92F982F872F480E591E6A1E7B1ED9
:10C240004386548665867686A501B701C6010E949D
:10C25000C30E8091FF1E90E02091BF143091C01456
:10C260008217930738F040E050E062E180E192E00D
:10C270000E94167A8091BF149091C014029708F41E
:10C280004DC08091162E9091172E91FF2AC00E94CA
:10C290000066C60105960E94CC65F60181811F9259
:10C2A0008F93F70186811F928F9385811F928F93C1
:10C2B0008DE599E09F938F931F9280E18F93CE013C
:10C2C00001965C019F938F930E94539D82E00E9490
:10C2D000E665C5010E94CC650FB6F894DEBF0FBEBF
:10C2E000CDBF8091660290916702A0916802B091E3
:10C2F000690297FD4DC08091BF149091C0140297C0
:10C3000008F47AC08091C9149091CA14A091CB14FA
:10C31000B091CC1481FF89C0749A87C08091660265
:10C3200090916702A0916802B091690296FFA9CF2F
:10C33000992009F4A6CFF6019081892F8F70823061
:10C34000E8F0907F8150892B808380EB9BE00E94F6
:10C35000F55F8091F11D9091F21D01969093F21D71
:10C360008093F11D8091C9149091CA14A091CB14AF
:10C37000B091CC1496FF85CF739883CF8091F71D31
:10C380009091F81D01969093F81D8093F71D79CF39
:10C3900080EE9DE12091E01D222309F4ACCF9F9314
:10C3A0008F9380E799E09F938F93CE0101963C0194
:10C3B0009F938F930E94909D5C01B301C6010296EA
:10C3C0000E94629C0F900F900F900F900F900F9013
:10C3D000009709F490CFEFEFAE1ABE0A8A0D9B1DAD
:10C3E000AC010196FA0120812032D1F362E18AE1A9
:10C3F00092E00E94167A7FCF112309F483CF82E066
:10C40000809331321092333210923232F0923532C0
:10C41000E092343241E352E362E182E492E00E942E
:10C42000167A70CF912C10E0D5CE60960FB6F894A6
:10C43000DEBF0FBECDBFDF91CF911F910F91FF9057
:10C44000EF90DF90CF90BF90AF909F907F906F90D4
:10C450005F904F9008958115910511F00197F1F7C4
:10C460000895E091FE36F091FF3690818091FD367F
:10C4700089230895E091FB36F091FC3690818091FC
:10C48000FD36892B8083E0910037F0910137908150
:10C490008091FD36892B808308951F93CF93DF937E
:10C4A000E091FB36F091FC3690818091FD368095CD
:10C4B00089238083E0910037F0910137908180914A
:10C4C000FD36892B80838FE897E00E942B621FB78F
:10C4D000F894E0910037F091013790818091FD361A
:10C4E00080958923808389E091E00E942B62E0910E
:10C4F000FE36F091FF36D081C091FD361FBF789493
:10C5000085E896E00E942B62E091FE36F091FF36BE
:10C5100090818091FD36892319F08D2F8C2301C0E5
:10C5200081E0DF91CF911F9108955093013740939F
:10C5300000377093FC366093FB369093FF36809300
:10C54000FE3681E001C0880F2A95EAF78093FD3618
:10C550000C944D62CF93DF93C82FDFB7F894E0912E
:10C560000037F091013790818091FD36892B8083CF
:10C5700087E090E00E942B62CC2351F0E0910037DD
:10C58000F091013790818091FD36809589238083D9
:10C5900084E390E00E942B62E091FE36F091FF363A
:10C5A00090818091FD36892309F4C0E085EB90E00D
:10C5B0000E942B62E0910037F091013790818091C9
:10C5C000FD36809589238083DFBF88E790E00E9455
:10C5D0002B628C2FDF91CF910895CF93DF93C82FDB
:10C5E000D8E08C2F81700E94AA62C6958111C06824
:10C5F000D150B9F78C2FDF91CF9108958FEF0C9424
:10C60000ED62DF92EF92FF920F931F93CF93DF9330
:10C61000E82E8B010E944D62811135C080EF0E948F
:10C62000ED62D0E0C0E488EFD82EDC0E81E00E94FD
:10C63000AA62F82E81E00E94AA62882319F0FF20E6
:10C6400071F023C0F1100BC0CE1530F0F8018081DD
:10C6500080FF05C0CE1519F0DC2FFF24F3948F2D39
:10C660000E94AA62F80180818695FF2011F08068FF
:10C67000F8018083C150CD11D9CF0F5F1F4FC11179
:10C68000D2CF8D2F03C08FEF01C08EEFDF91CF91FE
:10C690001F910F91FF90EF90DF900895EF92FF921E
:10C6A0001F93CF93DF93182FEB010E944D622097C9
:10C6B00071F085E50E94ED627E0188E0E80EF11CD4
:10C6C00089910E94ED62CE15DF05D1F703C08CEC95
:10C6D0000E94ED62812FDF91CF911F91FF90EF902B
:10C6E0000C94ED620F931F93CF93DF93DB01ED91D9
:10C6F000FC911197803161F4EE7F63E0EE0FFF1F34
:10C700006A95E1F716969C911697E91BF1093C96FC
:10C71000F7FF07C091E0EA019883F195E195F109EF
:10C7200002C0EA011882883279F414968C91982F0D
:10C730009076903649F086FF02C0EE7F05C085FFF7
:10C7400002C0EC7F01C0E87FCF0144E09695879559
:10C750004A95E1F7D9018C93EF70E801E88380E016
:10C76000DF91CF911F910F9108950F931F93CF9356
:10C77000DF93EC018B01B80188810E9401638883FB
:10C7800081508D3F30F4F8018081883211F0803182
:10C7900091F7DF91CF911F910F910895CF93DF9380
:10C7A000EC010E944D62BE0184EB0E944E6381E069
:10C7B0000E94AA62C82F0E944D6281E0C11101C08F
:10C7C00080E0DF91CF9108950F931F93CF93C82FEF
:10C7D0008B010E944D620E943162882349F0B801AA
:10C7E00084E40E944E63C13029F00E943A6202C084
:10C7F00082E001C080E0CF911F910F9108954F9288
:10C800005F926F927F928F929F92AF92BF92CF92E0
:10C81000DF92EF92FF920F931F93CF93DF93CDB7E9
:10C82000DEB729970FB6F894DEBF0FBECDBF6C01FF
:10C830003B015A0189010E944D62B6018EEB0E94B4
:10C840004E63CE0101967C014E019AE0890E911C47
:10C8500027010E94FE62F70181937F01E815F90527
:10C86000C1F769E070E0C2010E949584F82E811141
:10C8700008C09501A301B201F60180810E94726394
:10C8800002C083E0F82E8F2D29960FB6F894DEBFF4
:10C890000FBECDBFDF91CF911F910F91FF90EF9011
:10C8A000DF90CF90BF90AF909F908F907F906F90D0
:10C8B0005F904F900895EF92FF920F931F93CF9345
:10C8C000DF93CDB7DEB72B970FB6F894DEBF0FBE60
:10C8D000CDBF182F092F682F792F88E0810F0E9474
:10C8E000E463882319F084E391E244C06CE872E8C1
:10C8F0008EE190E00E94C7647E0189E0E80EF11CA1
:10C900009701AE01465F5F4FBE01655F7F4F812F8C
:10C91000902F0E94FF638111E6CF88E0EFEEF2E0F6
:10C92000DE01119601900D928A95E1F7298541E784
:10C9300052E0249FC001259F900D112464E670E011
:10C940000E94E4918A8594E6899F600D711D1124EF
:10C95000FE0131968191281303C06F5F7F4F03C0A2
:10C96000EE15FF05B9F78B85882319F07195619550
:10C970007109CB012B960FB6F894DEBF0FBECDBF69
:10C98000DF91CF911F910F91FF90EF900895DC01FF
:10C99000CB0181159105A105B10529F08150904089
:10C9A000A040B040D9F708959B01AC011092B900A6
:10C9B00060E074E284EF90E00E94F891DA01C9012E
:10C9C0004097A109B109B695A7959795879580934A
:10C9D000B800089594EA9093BC0040EA56E861E0FC
:10C9E00070E09091BC0097FD07C04150510961096A
:10C9F0007109B9F781E008959091B900987F983056
:10CA000011F09031B9F78093BB0084E88093BC00AB
:10CA100080EA96E8A1E0B0E02091BC0027FD05C0C7
:10CA20000197A109B109C1F7E5CF8091B900887FCD
:10CA3000883111F08034F1F680E0089524EA34E87A
:10CA400044E92093BC009091BC0097FFFCCF9091EB
:10CA5000B900987F983011F0903199F78093BB001E
:10CA60003093BC009091BC0097FFFCCF9091B9002F
:10CA7000987F903211F0983539F44093BC00909132
:10CA8000BC0094FDFCCFDDCF08950C94EA6484E9EA
:10CA90008093BC008091BC0084FDFCCF08958093FE
:10CAA000BB0084E88093BC008091BC0087FFFCCF72
:10CAB0009091B900987F81E0983209F480E0089560
:10CAC00084EC8093BC008091BC0087FFFCCF8091F8
:10CAD000BB00089584E88093BC008091BC0087FF70
:10CAE000FCCF8091BB000895CF93DF93FC0170963B
:10CAF000EC01A991CE01A0933F01EC17FD07C1F70E
:10CB000080913C018F7D80933C0180913C01877F27
:10CB100080933C01DB015096FB01819180933E01A3
:10CB2000EA17FB07D1F780913C01806880933C01B4
:10CB300080913D0180FFFCCF4051510980913C0123
:10CB4000806280933C0180913C01877F80933C010F
:10CB5000141615069CF4FB01819180933E01AE17DB
:10CB6000BF07D1F780913C01806880933C018091A0
:10CB70003D0180FFFCCF40515109EACFF901C901C5
:10CB8000409620913E0121938E179F07D1F781E0B7
:10CB900090E0DF91CF9108950F931F93CF93DF9390
:10CBA000EC018CE70E941E658CE70E944F658E01A8
:10CBB000005F1F4F89910E944F65C017D107D1F7C1
:10CBC000DF91CF911F910F910C944765813019F43B
:10CBD00040E050E002C040EC50E060E070E08CE7E4
:10CBE00090E00C947916813019F44EE050E002C0C8
:10CBF00048E050E060E070E08CE790E00C9479163B
:10CC000041E050E060E070E08CE790E00E9479162F
:10CC100064ED74E180E090E00C94C76448E350E078
:10CC200060E070E08CE790E00E94791649E350E004
:10CC300060E070E08CE790E00E94791644E150E0FB
:10CC400060E070E08CE790E00E94791648E750E0E1
:10CC500060E070E08CE790E00E9479164EE550E0CD
:10CC600060E070E08CE790E00E9479164DE650E0BD
:10CC700060E070E08CE790E00E94791668E374E36E
:10CC80008CE090E00E94C7644CE050E060E070E00F
:10CC90008CE790E00E94791641E050E060E070E09F
:10CCA0008CE790E00E94791646E050E060E070E08A
:10CCB0008CE790E00E94791664ED74E180E090E0EA
:10CCC0000C94C764CF93DF93CDB7DEB7A2970FB6AE
:10CCD000F894DEBF0FBECDBF81E1EFEFF9E0DE01DA
:10CCE000529601900D928A95E1F781E1E0E1FAE038
:10CCF000DE01119601900D928A95E1F70E940E6671
:10CD0000CE0142960E94CC6582E00E94E66564ED09
:10CD100074E180E090E00E94C764CE0101960E9419
:10CD2000CC6560E27CE581E590E00E94C76480E02C
:10CD30000E94F36560E27CE581E590E00E94C764B3
:10CD40004EE050E060E070E08CE790E00E947916E1
:10CD5000A2960FB6F894DEBF0FBECDBFDF91CF9184
:10CD60000895CF92DF92EF92FF920F931F93CF938C
:10CD7000DF9300D0CDB7DEB7042F122F213031F072
:10CD8000223031F0243031F0283031F090E005C00D
:10CD900091E003C092E001C093E0E82FF0E08160F1
:10CDA000F82E0C3009F4E1C00E3011F49460DDC0AF
:10CDB000003111F49860D9C0023109F0D6C0292F92
:10CDC0002C60613009F4B6C0623011F4206207C0F3
:10CDD000633011F4206403C0643009F420662068D5
:10CDE000622F70E023E030E0AE014F5F5F4FCF0174
:10CDF0000E94891662E174E380E090E00E94C764BB
:10CE00008F2D0E94EA640E94606589830E9460659C
:10CE10008A83023119F40E9460658B830E946065E9
:10CE200087FDF1CF0E946A650E94476562E174E365
:10CE300080E090E00E94C7648F2D0E94EA640E9407
:10CE4000606589830E9460658A83023119F40E94BB
:10CE50006A658B830E946A650E94476569812A81A1
:10CE6000023139F5862F90E0A0E0B0E04B8130E050
:10CE7000322F2227DC0199278827820F931FA11DBB
:10CE8000B11D61FF09C0840F911DA11DB11DBC0121
:10CE9000CD018C6F9F6F06C0BC01CD01640F711D69
:10CEA000811D911D0E94A49520E83FEF4FEF57E4AC
:10CEB0001FC070E0762F6627620F711D072E000CD1
:10CEC000880B990B0E94A4950C3029F420E030EED9
:10CED0004FEF54E40DC00E3029F420E038EF4FEF4F
:10CEE00055E406C0003131F420E03EEF4FEF56E448
:10CEF0000E94F0942FE632E143E050E40E949C97B8
:10CF00006B017C01612F70E080E090E00E94A495AD
:10CF10009B01AC01C701B6010E94F0940F900F90E5
:10CF20000F90DF91CF911F910F91FF90EF90DF90C5
:10CF3000CF9008959C68692F70E023E030E0AE0147
:10CF40004F5F5F4FCF010E94891662E174E380E07A
:10CF500090E00E94C7648F2D0E94EA640E94606581
:10CF600089830E9460658A8356CF6130D9F49068C6
:10CF7000692F70E023E030E0AE014F5F5F4FCF01DB
:10CF80000E94891662E174E380E090E00E94C76429
:10CF90008F2D0E94EA640E94606589830E9460650B
:10CFA0008A833CCF292F10CF8F929F92AF92BF924E
:10CFB000CF92DF92EF92FF920F931F93EDECF4E18B
:10CFC0000081118120E030E06B017C0144E0F594A8
:10CFD000E794D794C7944A95D1F7C01AD10AE20AC8
:10CFE000F30ADC01CB0153E0B595A795979587959A
:10CFF0005A95D1F7000F111F221F331F4C015D01FD
:10D00000801A910AA20AB30AA5019401A281B381F0
:10D010000E946A924B015C017BE0B594A7949794BF
:10D0200087947A95D1F7A7019601C701B6010E94AE
:10D03000B4919B01AC01ACE0559547953795279588
:10D04000AA95D1F7A481B5810E946A92DC01CB0137
:10D050001EE0B595A795979587951A95D1F7A501E7
:10D060009401280F391F4A1F5B1F21A332A343A33A
:10D0700054A3A5E0B0E00E945F92DC01CB01805890
:10D080009F4FAF4FBF4F692F7A2F8B2F992787FD67
:10D090009A951F910F91FF90EF90DF90CF90BF90E6
:10D0A000AF909F908F900895CF92DF92EF92FF9272
:10D0B0001F93CF93DF93CDB7DEB76A970FB6F8947F
:10D0C000DEBF0FBECDBF182F21E030E0CE010196AC
:10D0D0007C01AC0160ED70E08EEE90E00E9489165C
:10D0E0008981803609F0C8C046EB50E060EE70E000
:10D0F0008EEE90E00E9479163CE2C32EDD24D3949C
:10D1000088EE93E00E94386F91E0C91AD108C1F708
:10D110008AE1F70111928A95E9F72AE130E0A70147
:10D1200068E870E08EEE90E00E94891689819A810D
:10D130009093CE148093CD148C8190E0982F882703
:10D140002B81822B9093D0148093CF148E8190E00A
:10D15000982F88272D81822B9093D2148093D114FD
:10D160008F8198859093D4148093D3148A8590E00E
:10D17000982F88272985822B9093D6148093D514D5
:10D180008C8590E0982F88272B85822B9093D8143C
:10D190008093D7148E8590E0982F88272D85822B39
:10D1A0009093DA148093D914888990E0982F882777
:10D1B0002F85822B9093DC148093DB148A8990E076
:10D1C000982F88272989822B9093DE148093DD1471
:10D1D0008C8990E0982F88272B89822B9093E014DC
:10D1E0008093DF148E8990E0982F88272D89822BD9
:10D1F0009093E2148093E114888D90E0982F882713
:10D200002F89822B9093E4148093E3148A8D80936A
:10D21000E51428E030E0A70161EE70E08EEE90E0CA
:10D220000E9489168A8190E0982F88272981822B75
:10D230009093E7148093E6148B818093E8148D819A
:10D240002C81F0E12F9F90011124982F9F70292BA2
:10D250003093EA142093E9142E812F7030E1839FDC
:10D26000C0011124822B9093EC148093EB148F81D6
:10D270008093ED141093F2146A960FB6F894DEBF03
:10D280000FBECDBFDF91CF911F91FF90EF90DF9048
:10D29000CF9008952F923F924F925F926F927F921C
:10D2A0008F929F92AF92BF92CF92DF92EF92FF92B6
:10D2B0000F931F93CF93DF93CDB7DEB7A4970FB62D
:10D2C000F894DEBF0FBECDBF9E012F5F3F4F7901A7
:10D2D00098E0D9011D929A95E9F7813009F015C3BC
:10D2E0008091F214813009F010C341E050E062EF08
:10D2F00070E08EEE90E00E94791640E050E065EF1D
:10D3000070E08EEE90E00E94791646E250E064EF05
:10D3100070E08EEE90E00E94791600E416E088EE50
:10D3200093E00E94386F01501109C9F70CE211E037
:10D3300021E030E0AE01475F5F4F63EF70E08EEEBB
:10D3400090E00E948916898589708987882341F039
:10D3500088EE93E00E94386F0150110949F7D5C259
:10D3600028E030E0A70167EF70E08EEE90E00E94C9
:10D370008916F981FAA32A812BA33B813CA3CF8094
:10D38000D884DC24CD24DC24E12CF12C6C81862F84
:10D3900090E0A0E0B0E0AC01BD01ECE0440F551F0F
:10D3A000661F771FEA95D1F78D8190E0A0E0B0E08D
:10D3B000F4E0880F991FAA1FBB1FFA95D1F7842BA1
:10D3C000952BA62BB72B2E8122952F70BC01CD015A
:10D3D000622B0E94D4676093EA367093EB36809399
:10D3E000EC369093ED368090EE149090EF14A09070
:10D3F000F014B090F114D501C4019C52A140B109C0
:10D400008A879B87AC87BD87AEE0CC0CDD1CEE1C09
:10D41000FF1CAA95D1F78091E9149091EA14092E86
:10D42000000CAA0BBB0B14E1880F991FAA1FBB1F8E
:10D430001A95D1F7C81AD90AEA0AFB0AA091EB1487
:10D44000B091EC142A853B854C855D850E946A92DB
:10D45000C61AD70AE80AF90A90E4D90EE11CF11CB1
:10D460000FE0F594E794D794C7940A95D1F7A0916B
:10D47000E814B0E00E945F922B013C018BE07594B0
:10D480006794579447948A95D1F7A0E85A0E611C87
:10D49000711CA091ED140A2E000CBB0B0E946A9225
:10D4A0002AE095958795779567952A95D1F7A301F9
:10D4B00092010E94B491DC01CB013AE0B595A795A9
:10D4C000979587953A95D1F79C01AD01405E5F4FE6
:10D4D000A091E614B091E7140E946A92DC01CB019E
:10D4E000905EAF4FBF4FBC01CD014EE09595879543
:10D4F000779567954A95D1F7A70196010E94B49157
:10D500006B017C015FE095958795779567955A95B6
:10D51000D1F79B01AC010E94B4919B01AC0167E083
:10D5200055954795379527956A95D1F7A091E514BC
:10D53000B0E00E945F92DC01CB0174E0B595A79545
:10D54000979587957A95D1F7A7019601281B390BF6
:10D550004A0B5B0BDA01C90157FF03C080E090E082
:10D56000DC0181309105A10539E1B30724F080E0A9
:10D5700090E0A0E0B9E12CE0B595A7959795879547
:10D580002A95D1F78093EE369093EF36A093F0363C
:10D59000B093F13675016401FF0CCC08DC2C7601E8
:10D5A0009401A5016C2D7C2D8C2D9C2D345F414068
:10D5B000510961097109810991092A873E874F87BD
:10D5C000588B698B7A8B8B8B9C8B59016A017B0101
:10D5D0008C010E9472922D8B3E8B4F8B5D8F6E8FD4
:10D5E0007F8F88A399A33091D6142091D514932FBF
:10D5F000990F990B492F592F692F792F892F0E9445
:10D6000072920CE00E94A293922E832E742E652EAD
:10D61000562E472E382E292E3091D8142091D7140B
:10D62000932F990F990BAD88BE88CF88DD8CEE8C37
:10D63000FF8C08A119A1492F592F692F792F892F04
:10D640000E94729208E00E94BB93A92CB82CC72CB0
:10D65000D62CE52CF42C032D122D0E94D993705852
:10D660008F4F9F4F2090D3143090D4145101C12C70
:10D67000D12CE12CF12C00E010E00E94729201E22A
:10D680000E94BB93288F398F4A8F5B8F6C8F272E18
:10D69000382E492EA0E00E94009409F42AC130914E
:10D6A000DE142091DD14932F990F990BAD88BE885D
:10D6B000CF88DD8CEE8CFF8C08A119A1492F592F42
:10D6C000692F792F892F0E9472922D8B3E8B4F8B61
:10D6D000552E3B014C013091DC142091DB14932F2B
:10D6E000990F990BAA84BE84CF84D888E988FA88D8
:10D6F0000B891C89492F592F692F792F892F0E9457
:10D70000729201E10E94A293AD88BE88CF88D52C89
:10D71000730184010E94D99359016A017B01582E3B
:10D72000192FBBA14B2F50E060E070E0E4E0440F04
:10D73000551F661F771FEA95D1F78CA182958F70D0
:10D74000482BEAA18E2F90E0A0E0B0E0FCE0880F2B
:10D75000991FAA1FBB1FFA95D1F7482B592B6A2B8B
:10D760007B2B80E090E0A0E1B0E0841B950BA60B42
:10D77000B70B3C014D01990C6608762C43019C01C6
:10D78000AD01662D762D862D962D0FE10E94A29378
:10D7900039014A01B62FA72FF82FE92F3091DA145B
:10D7A0002091D914932F990F990B492F592F692F35
:10D7B000792F892F03E20E94A293052D0E94D9930D
:10D7C00059016A017B018C019301A4016B2F7A2F0F
:10D7D0008F2F9E2F0E94EE93E5E3AE2EFCE0BF2E2E
:10D7E000C12CD12CE12CF12C00E010E00E947292AF
:10D7F000A88CB98CCA8CDB8CEC8CF22C032D142DEC
:10D800000E94CD922A873E874F87588B698B7A8BEF
:10D810008B8B9C8B0DE00E94BB93922E832E742EDB
:10D82000652E562E472E382E292E3091E414209145
:10D83000E314932F990F990BA92CB82CC72CD62C35
:10D84000E52CF42C032D122D492F592F692F792FF8
:10D85000892F0E9472920E94729209E10E94BB93EA
:10D86000AA84BE84CF84D888E988FA880B891C8969
:10D870000E94D99319012A013B014C013091E21415
:10D880002091E114932F990F990B492F592F692F4C
:10D89000792F892F0E94729203E10E94BB93590154
:10D8A0006A017B018C019101A201B301C4010E94B4
:10D8B000D99308E00E94BB9359016A017B01E82FCC
:10D8C000192F3091E0142091DF14932F990F990BA9
:10D8D000492F592F692F792F892F04E00E94A29395
:10D8E0000E2F0E94D993722F632F942F852F9B01A7
:10D8F00004C030E020E090E080E03093F2362093E6
:10D90000F3369093F4368093F536A4960FB6F894D8
:10D91000DEBF0FBECDBFDF91CF911F910F91FF9062
:10D92000EF90DF90CF90BF90AF909F908F907F90BF
:10D930006F905F904F903F902F900895CF93E6E4C3
:10D94000F1E0C081908180812081C07C2295269564
:10D9500026952370C20F969596959073C90F829560
:10D960008C70C80F1F92CF938AE094E19F938F939E
:10D970000E94FB9C0F900F900F900F908C2FCF91D7
:10D980000895CF93C82F81E29AE09F938F930E94CE
:10D99000E79C0F900F90C0FF04C08EE29AE00E94B7
:10D9A000239DC1FF04C08DE39AE00E94239DC2FF26
:10D9B00004C08CE49AE00E94239DC3FF04C08BE561
:10D9C0009AE00E94239DC4FF05C08AE69AE0CF91A9
:10D9D0000C94239DCF9108951F93CF93DF9383B130
:10D9E00081708093043746E069E180E00E941A70FC
:10D9F00080E00E946F700E94F46E85E79AE09F932A
:10DA00008F938FEE93E19F938F930E94FB9C8EB335
:10DA10000E94C16C0E946F7A0E94A67960E070E05B
:10DA200089EB92E00E94427A0E948A78E091D00AC3
:10DA3000F091D10A19950E949E6C90E00E94A0700E
:10DA40000E94338182E080934139809342390E9461
:10DA5000456E41E459E3BC018DEC9BEA0E946A7378
:10DA60000E94B76D0E9457730E94496E0E946A74AB
:10DA70000E94BC7FE0914A0BF0914B0B1995E0910D
:10DA8000220BF091230B1995E091060BF091070BF7
:10DA900019950E946C74182FC091560BD091570B9A
:10DAA000FE0119950F900F900F900F90892B49F060
:10DAB000FE011995BC0180E890E00E94D091EB0135
:10DAC00002C0C0E8D0E00E9454731F921F93DF93FE
:10DAD000CF931F928F938091490B8F938091480B26
:10DAE0008F938091210B8F938091200B8F938DEBDF
:10DAF00093E19F938F930E94FB9C80EB93E19F9314
:10DB00008F930E94FB9C8FE993E19F938F930E94D8
:10DB1000FB9C60E070E085EE92E00E94427A60E05B
:10DB200070E087E992E00E94427A8DEE99E00E94CF
:10DB3000A77687E993E19F938F930E94FB9C8DB713
:10DB40009EB742960FB6F8949EBF0FBE8DBFDF9171
:10DB5000CF911F91089580E8809361001092610039
:10DB60000E94EC6C0E94B6790E949270FBCFEF92FB
:10DB7000FF920F931F93CF93DF93CDB7DEB7A0979C
:10DB80000FB6F894DEBF0FBECDBF83E690E00E94D3
:10DB9000AC9F182F282F35EF380F303108F0982F11
:10DBA0009095291709F463C089E194E19F938F93BD
:10DBB0000E94FB9CEEE5F4E18E010F5F1F4FCE014A
:10DBC00009960F900F90D801780124912D933196EA
:10DBD000A817B907D1F7F89448E050E06FE770E074
:10DBE000C8010E94B29FE0E5F4E1CE010F96D80192
:10DBF00024912D933196A817B907D1F74EE050E044
:10DC000061E770E0C8010E94B29FE6E4F4E1CE0152
:10DC10000B962491D8012D938D013196A817B90741
:10DC2000C1F74AE050E067E670E0C7010E94B29F8A
:10DC30006DEC7BEA81E690E00E94CA9F60E070E0B4
:10DC40008FE590E00E94CA9F60E08EE590E00E9420
:10DC5000BC9F60E070E085E690E00E94CA9F1AE1F8
:10DC60006AE175EE83E690E00E94CA9F7894812F66
:10DC7000A0960FB6F894DEBF0FBECDBFDF91CF9157
:10DC80001F910F91FF90EF9008958FE590E00C9415
:10DC9000AC9F8EE590E00C94A49F83B1817090E0DE
:10DCA0000895209880E090E0089580E090E0089545
:10DCB000CF93DF93EC01888199818737910509F42F
:10DCC00057C08E37910509F470C0892B09F084C0C4
:10DCD0000E949F7980930A371092F6141092F514DF
:10DCE0008091F5149091F614FC01EE0FFF1FED5694
:10DCF000FD4F0190F081E02D3097B1F0DC01A85F7D
:10DD0000B84C1C920480F581E02D60E070E080E862
:10DD100090E019958091F5149091F61401969093E6
:10DD2000F6148093F514DCCF8093F71487E790E026
:10DD300039C0FC01E85FF84C208127FD22C08091AA
:10DD4000F5149091F61401969093F6148093F514BF
:10DD50008091F5149091F6142091F71430E0821719
:10DD600093073CF38091F3149091F414892BF1F212
:10DD70001092F4141092F3141092F6141092F514F9
:10DD8000E7CF880F991FFC01ED56FD4F408151816F
:10DD900060910A3780E090E00E94167A892B49F45E
:10DDA0008EE790E0998388831BC080910A378613A1
:10DDB00017C0E091F514F091F614E85FF84C8081FB
:10DDC0008F7780838091F3149091F414019690934F
:10DDD000F4148093F314B3CF1982188283E001C046
:10DDE00081E0DF91CF910895F8941092B60016BCAF
:10DDF00089E787BD82E084BD95E095BD95B395BB6D
:10DE000080936E00789408950F931F936091FA1495
:10DE10007091FB148091FC149091FD140091FA1400
:10DE20001091FB142091FC143091FD1460177107C0
:10DE30008207930759F71F910F9108950F931F932E
:10DE40006091133770911437809115379091163780
:10DE500000911337109114372091153730911637F0
:10DE6000601771078207930759F71F910F91089563
:10DE7000009731F0880F991F880F991F0197F1F7CC
:10DE800008951F920F920FB60F9211240BB60F92A6
:10DE90002F933F934F935F936F937F938F939F93B2
:10DEA000AF93BF93EF93FF938091FA149091FB147B
:10DEB000A091FC14B091FD140196A11DB11D809399
:10DEC000FA149093FB14A093FC14B093FD1480916A
:10DED000F9148F5F8093F91487FF15C01092F9141D
:10DEE0008091133790911437A0911537B091163760
:10DEF0000196A11DB11D8093133790931437A09301
:10DF00001537B09316378091B2388823E1F08091AD
:10DF1000F8148F5F8093F81487FF15C01092F814DF
:10DF200080910B3790910C37A0910D37B0910E373F
:10DF30000196A11DB11D80930B3790930C37A093D0
:10DF40000D37B0930E370E94F277892B11F00E94A3
:10DF50001377FF91EF91BF91AF919F918F917F9137
:10DF60006F915F914F913F912F910F900BBE0F904A
:10DF70000FBE0F901F9018951F920F920FB60F9221
:10DF800011240BB60F922F933F934F935F936F9390
:10DF90007F938F939F93AF93BF93EF93FF93809162
:10DFA000C600E0911937F0911A37309709F01995AA
:10DFB000FF91EF91BF91AF919F918F917F916F9161
:10DFC0005F914F913F912F910F900BBE0F900FBE1D
:10DFD0000F901F9018951F920F920FB60F92112459
:10DFE0000BB60F922F933F934F935F936F937F9353
:10DFF0008F939F93AF93BF93EF93FF938091CE0046
:10E00000E0911737F0911837309709F01995FF9183
:10E01000EF91BF91AF919F918F917F916F915F91A0
:10E020004F913F912F910F900BBE0F900FBE0F900D
:10E030001F90189581110EC01092C5006093C40006
:10E0400088E98093C1004093C20010921A37109261
:10E0500019370895813069F41092CD006093CC0097
:10E0600088E98093C9004093CA0010921837109233
:10E0700017370895811107C08091C00085FFFCCF3C
:10E080006093C6000895813031F48091C80085FF07
:10E09000FCCF6093CE000895CF93C82F8A3031F41F
:10E0A0006DE08091FE140E943A7002C08D3029F01C
:10E0B0006C2F8091FE140E943A7080E090E0CF9126
:10E0C0000895811105C070931A3760931937089528
:10E0D000813021F470931837609317370895809337
:10E0E000FE1481EA92E090935E3B80935D3B08953D
:10E0F00084B7877F84BF0FB6F894A895809160009D
:10E10000886180936000109260000FBE08959FE0C8
:10E1100088E10FB6F894A895809360000FBE9093A5
:10E1200060000895A89508950FB6F894A895809179
:10E130006000886180936000109260000FBE0895B7
:10E140000C94BA980C94B6988091203790E008957A
:10E150008091390181FF09C0809139018D7F8093C1
:10E16000390189E190E00197F1F723E040E06FE1A8
:10E1700082E491E00E94C77585E090E00197F1F795
:10E1800008959091390191FD0AC0282F803108F03F
:10E190002FE040E06FE085E491E00C94C7750895AE
:10E1A0008091390181FD09C040E06FE181E491E097
:10E1B0000E94BC758F7E813019F080E090E0089558
:10E1C00081E090E008958091390181FF02C081E0F3
:10E1D000089540E06FE181E491E00E94BC758F31C9
:10E1E00021F08F7E8150823090F780E008958091F9
:10E1F000390181FD04C00E94E3708823C1F30895B2
:10E200001092B2388091390181FD8BC00E94F77065
:10E210008091390181FD85C00E94A87080913901EB
:10E220008260809339018091EA388823D9F1809106
:10E230009400909195004091FB385091FC388417E0
:10E240009507A0F48091C7389091C838A091C9383B
:10E25000B091CA38875F924CAF4FBF4F8093C73899
:10E260009093C838A093C938B093CA3820919400CD
:10E2700030919500241B350B8091C7389091C83898
:10E28000A091C938B091CA38820F931FA11DB11D4A
:10E290008093C7389093C838A093C938B093CA38D0
:10E2A0001092EA388091EC388823D9F1809194005B
:10E2B000909195004091FF3850910039841795074F
:10E2C000A0F48091CF389091D038A091D138B091FE
:10E2D000D238875F924CAF4FBF4F8093CF38909327
:10E2E000D038A093D138B093D23820919400309197
:10E2F0009500241B350B8091CF389091D038A09198
:10E30000D138B091D238820F931FA11DB11D8093D7
:10E31000CF389093D038A093D138B093D2381092A0
:10E32000EC3808958091B238882321F00E94E37080
:10E330000E94007180E090E0089522E0260F27FF00
:10E340000CC08091B0389091B13801969093B1385B
:10E350008093B0388FEF9FEF0895AB01BC018FEF32
:10E3600094E10E94289C80E090E0089540E06FE1F5
:10E3700081E491E00C94BC75282F40E06FEF86E5B6
:10E3800091E00E94C7750895CF93DF9398EF980F9F
:10E39000923038F0982F9F7E963019F0893109F02D
:10E3A0004BC09091390191FD4AC0C82F0E94F7706F
:10E3B0000E94B671D82FC81709F43BC0C83029F4A1
:10E3C000809139010E94A87027C0C93119F48631A3
:10E3D00081F404C0C63169F4893159F429E040E080
:10E3E0006FE182E491E00E94C77585E090E00197BB
:10E3F000F1F72C2F40E06FE182E491E00E94C775B5
:10E40000D83031F48FEF0E94BC7181ED92E002C0F0
:10E4100085E090E00197F1F70E94B671C81749F0C6
:10E42000C63019F4813071F404C0C63159F4813119
:10E4300049F480E490E008C082E490E005C084E400
:10E4400090E002C083E490E0DF91CF910895809145
:10E45000940090919500909300398093FF3881E06B
:10E460008093EC388093B2389091390191FF1EC0AF
:10E4700020919400309195003093FC382093FB3824
:10E480008093EA388093AD382FB778948091390122
:10E49000809139018D7F8093390180E197E230913D
:10E4A000AD38332311F00197D1F72FBF86E10E94D9
:10E4B000C4710C94F7708091B238811102C00E942F
:10E4C000277281E090E008950F931F93CF93DF931D
:10E4D0001F92CDB7DEB78091B238882361F080916A
:10E4E000390181FF02C080E07BC00E94E370882375
:10E4F000D1F300E003C00E945B7201E080919400C0
:10E50000909195009093FA388093F93811E0109328
:10E51000E93880E88093550186E00E94C471109329
:10E5200021378FB7898378941092470180912137E2
:10E530008111FCCF89818FBF8091470111E08E301E
:10E5400008F010E0119586E10E94C4711092550107
:10E550008091E9388823D9F18091940090919500B9
:10E560004091F9385091FA3884179507A0F48091BA
:10E57000C3389091C438A091C538B091C638875F30
:10E58000924CAF4FBF4F8093C3389093C438A09341
:10E59000C538B093C6382091940030919500241B63
:10E5A000350B8091C3389091C438A091C538B09193
:10E5B000C638820F931FA11DB11D8093C33890935D
:10E5C000C438A093C538B093C6381092E938011109
:10E5D0000E949271812F82958695869583708170B5
:10E5E00090E00F90DF91CF911F910F9108958FEFE1
:10E5F00080934E0121E044E060EF8CE691E00E94C0
:10E60000C77525E041E06EE08CE691E00E94C77599
:10E6100080E880936F018091460180936D0121E035
:10E6200045E060E284E491E00C94C775CF93DF93FA
:10E63000C9EFD7E0CE010197F1F70E94BB751092A8
:10E6400027371092A93710922B3810922637109244
:10E650002537E9E3F1E080818E7F808380818D7FA3
:10E66000808381EC93E00197F1F780818160808362
:10E6700023E040E06FE182E491E00E94C7752197BA
:10E68000F1F780915D0180915E010E94F77260E078
:10E6900070E08FEA92E00E94427A0E94277281E045
:10E6A00090E0DF91CF910895809180150895CF93E8
:10E6B000C82F0E94F770C09380152C2F40E06FE1A7
:10E6C00088E491E0CF910C94C7750E94577386E05F
:10E6D0000C94C471EF92FF920F931F93CF93DF932B
:10E6E0007C018B01EA011F936F93FF928F9386EA5F
:10E6F0009AE09F938F930E94E79CE0926201F092D0
:10E70000630100936001109361010F900F900F90CF
:10E710000F900F900F902097C1F0888180936B012C
:10E72000898180936A018A81809369018B818093BA
:10E7300068018C81809367018D81809366018E8151
:10E74000809365018F8180936401DF91CF911F9148
:10E750000F91FF90EF9008958FEA92E00E94637A04
:10E7600081E0809320378091223790912337019662
:10E77000909323378093223781E090E008950F93A0
:10E780001F93CF9320912637C2E8C29F9001112496
:10E79000F901E95DF84C4081442309F44FC047FD7D
:10E7A00009C0433038F050E08A0102501109601767
:10E7B000710710F4108242C0B901685D784C0E9464
:10E7C000289C80912637C89FF0011124E95DF84C00
:10E7D000DF01A058BF4F9C9190931B3710828F5F31
:10E7E000833018F48093263702C010922637E091C8
:10E7F000263782E8E89FF0011124E95DF84C80811A
:10E80000882319F00E94AC7302C0109220376091E7
:10E81000470160931C3780911F37882311F06817D8
:10E8200010F460931F3770E084E00E940F816091C4
:10E830001B3770E083E00E940F8102C000E010E00F
:10E84000C801CF911F910F9108950F931F93CF93FC
:10E85000DF931F92CDB7DEB78C01FC0180819181DF
:10E86000009709F18334954029F0F8011182108254
:10E8700083E02AC06238E1F40E94C7808FB78983A1
:10E88000F8940E94318060E870E00E94BF73298193
:10E890002FBF1816190674F40E942C80E091500BBB
:10E8A000F091510B199583E495E0F80191838083F1
:10E8B00081E00AC080911D3790911E370196909398
:10E8C0001E3780931D37EFCF0F90DF91CF911F91AF
:10E8D0000F9108950C94C1708091390181FD06C09B
:10E8E00040E06FE085E491E00C94BC7580E1089510
:10E8F000EF92FF921F93CF93DF931F92CDB7DEB7B6
:10E90000182F8091390181FD07C00E94F770809116
:10E91000B23881111CC05AC080919400909195002A
:10E920009093FC388093FB3881E08093EA388093A1
:10E93000AD38809139018D7F8093390180E197E274
:10E940002091AD38222309F30197D1F7DECF8091D2
:10E95000EC388823D9F180919400909195004091F2
:10E96000FF385091003984179507A0F48091CF3873
:10E970009091D038A091D138B091D238875F924C25
:10E98000AF4FBF4F8093CF389093D038A093D138FA
:10E99000B093D2382091940030919500241B350B10
:10E9A0008091CF389091D038A091D138B091D238A1
:10E9B000820F931FA11DB11D8093CF389093D03843
:10E9C000A093D138B093D2381092EC3889E10E94EC
:10E9D000C47186E00E941A81892B51F00E946C74E8
:10E9E000E82E86E00E941A8181500E94C17002C008
:10E9F000E12CF12C80919400909195009093FE3839
:10EA00008093FD3881E08093EB388FB78983F89449
:10EA100080913901826080933901809139018D7F25
:10EA20008093390162E0610F8FEF94E10E940D76CF
:10EA300089818FBF8091AE389091AF3801969093C5
:10EA4000AF388093AE380E94F77045E060EE82E404
:10EA500091E00E94BC75182F86E00E941A81892BD4
:10EA600019F08E2D0E94C1708091EB388823D9F166
:10EA700080919400909195004091FD385091FE381E
:10EA800084179507A0F48091CB389091CC38A09151
:10EA9000CD38B091CE38875F924CAF4FBF4F809347
:10EAA000CB389093CC38A093CD38B093CE3820910A
:10EAB000940030919500241B350B8091CB389091B8
:10EAC000CC38A091CD38B091CE38820F931FA11DC4
:10EAD000B11D8093CB389093CC38A093CD38B093B0
:10EAE000CE381092EB388091B238882371F0809143
:10EAF000940090919500909300398093FF3881E0C5
:10EB00008093EC380E94277202C00E94007112307C
:10EB100028F48CE00E941A8110E00BC0133031F011
:10EB2000153031F0173029F411E003C012E001C0B4
:10EB300013E0812F90E00F90DF91CF911F91FF9014
:10EB4000EF900895CF93DF93EB010E949D710097A2
:10EB500029F4CE010E947874009751F02091B038CA
:10EB60003091B1382F5F3F4F3093B1382093B03898
:10EB7000DF91CF9108950895FC0180816823862F4D
:10EB800090E002C0959587954A95E2F70895CF9356
:10EB9000DF931F92CDB7DEB7FC01922F8FB7898329
:10EBA000F8942081562F50955223292F01C0220F0F
:10EBB0004A95EAF72623252B208389818FBF0F9062
:10EBC000DF91CF910895CF93DF93E0917B012DEFFB
:10EBD0002E0F2D3740F0FC011082E058FF4F1082BD
:10EBE0003196108217C0DC01ED932E2FC0E8D1E0E2
:10EBF00038813D93215021962111FACFE150F0E068
:10EC0000E058FE4F2181FC01E058FF4F20833196F0
:10EC100021E02083DF91CF910895609380016250BD
:10EC2000E1E8F1E0DC012D91CD01208361503196C6
:10EC30006111F8CF08951F920F920FB60F92112411
:10EC40000BB60F922F933F934F935F936F937F93E6
:10EC50008F939F93AF93BF93EF93FF93809147015F
:10EC600080931C378091253722E8829FC0011124B0
:10EC7000895D984C0E94E375809125378F5F8330C2
:10EC800018F48093253702C0109225370E94AC7388
:10EC9000FF91EF91BF91AF919F918F917F916F9174
:10ECA0005F914F913F912F910F900BBE0F900FBE30
:10ECB0000F901F9018951F920F920FB60F9211246C
:10ECC0001092AD380F900FBE0F901F9018951F92A5
:10ECD0000F920FB60F921124109224370F900FBE8F
:10ECE0000F901F9018951F920F920FB60F9211243C
:10ECF0000F900FBE0F901F9018951F920F920FB696
:10ED00000F9211240F900FBE0F901F9018951F9215
:10ED10000F920FB60F9211240F900FBE0F901F90FD
:10ED200018951F920F920FB60F9211240F900FBEDD
:10ED30000F901F9018951F920F920FB60F921124EB
:10ED4000109221370F900FBE0F901F901895CF9300
:10ED5000DF93EC0189919991009729F060E070E0D0
:10ED60000E94427AF7CFDF91CF910895CF92DF9240
:10ED7000EF92FF920F931F938091851590918615C6
:10ED8000892B49F4109281151092821510928315E7
:10ED90001092841541C00E94046F8B019C01E09188
:10EDA0008515F0918615408151816281738184813E
:10EDB0009581A681B781840F951FA61FB71F801B61
:10EDC000910BA20BB30B0084F185E02D3097C1F0BD
:10EDD000C080D180E280F380448155816681778153
:10EDE0004C0D5D1D6E1D7F1D401B510B620B730B87
:10EDF000481759076A077B0730F7DB01CA01E3CFE1
:10EE0000800F911FA21FB31F8093811590938215CD
:10EE1000A0938315B09384151F910F91FF90EF90ED
:10EE2000DF90CF90089589EB92E00C94637AEF9293
:10EE3000FF920F931F93CF93DF938C01FC0180818E
:10EE40009181009799F089359105D9F0F8011182E7
:10EE5000108283E068C0828593854817590709F0BE
:10EE600049C00084F185E02D3097A9F710928615EE
:10EE70001092851589E590E0F8019183808381E007
:10EE800052C0673891F16238A9F7C0918515D091C9
:10EE90008615E12CF12C209769F3CE010E94BE7AF1
:10EEA000892BF1F0AE0168E88A859B850E94167A6D
:10EEB000892BA1F41B861A8688859985E114F104B3
:10EEC00021F0F7019187808704C090938615809385
:10EED0008515198618860E94B676D7CF0E941377BB
:10EEE0007E010884D985C02DD6CFE0918515F0919B
:10EEF0008615BACFF0938615E0938515A085B18568
:10EF0000109709F4B7CF1A968D919C911B974817CB
:10EF1000590739F418968D919C911997918780879C
:10EF2000EDCFFD01EBCFDF91CF911F910F91FF90BE
:10EF3000EF900895CF93DF93EC010E9413772A8519
:10EF40003B859091851580918615232B91F0E92FB3
:10EF5000F82F309771F0EC17FD0739F480913316D4
:10EF6000909134169387828710C00084F185E02D3C
:10EF7000F0CF20913316309134163B872A8798873B
:10EF80008987D0938615C0938515DF91CF910C9416
:10EF9000B676CF93DF93EC010E94907ACE01DF9199
:10EFA000CF910C949A77CF93DF93EC010E94A07AD3
:10EFB000CE01DF91CF910C949A77CF93DF93EC0140
:10EFC0000E94B27ACE01DF91CF910C949A7721E022
:10EFD00030E0FC0182859385892B11F020E030E040
:10EFE000C901089581E090E0209185153091861542
:10EFF000232B11F480E090E00895CF93DF93EC0190
:10F00000E0918515F0918615E817F90769F4888570
:10F01000998590938615809385150DC0808591857F
:10F02000C817D90721F0FC013097C1F706C08885C1
:10F030009985918780870E94B676198618861B86E7
:10F040001A86DF91CF910895EF92FF920F931F934D
:10F05000CF93DF938C017A01FC018081918100972D
:10F0600041F08A34910511F1F8011182108283E098
:10F070004AC088E895E10E94ED7AEC01209761F0A2
:10F080004E815F8168857985CE0102960E94C9779D
:10F090000990D881C02DF2CF81E0809387158AE452
:10F0A00090E0F8019183808381E02DC06838E1F71A
:10F0B00088E895E10E94ED7AEC01209781F3CE017A
:10F0C0000296E816F906D9F4BE0188E895E10E9497
:10F0D0000D7BE0903316F09034168E859F859093CB
:10F0E000341680933316E889F989309719F08A89A4
:10F0F0009B891995F0923416E0923316D0CF09907F
:10F10000D881C02DDACFDF91CF911F910F91FF9061
:10F11000EF9008951092871588E895E10E94E97AAA
:10F1200060E070E083EC92E00C94427AEF92FF9200
:10F130000F931F93CF93DF93EC01E0903316F09081
:10F140003416FF86EE86398B288B1B8B0A8B8091B9
:10F150008715882379F083EC92E09093341680939E
:10F160003316CE0102960E94C977F0923416E092CF
:10F17000331604C04E835F8368877987BE0188E8B1
:10F1800095E10E940D7BBE0188E895E1DF91CF916A
:10F190001F910F91FF90EF900C94287BCF93DF93FA
:10F1A000EC0180918715882329F0CE0102960E94F8
:10F1B000FD7704C01B861A861D861C86BE0188E862
:10F1C00095E1DF91CF910C940D7B1F93CF93DF934B
:10F1D000DC011496ED91FC9115973097E1F0162F14
:10F1E000EC01909334168093331682E08887CD012A
:10F1F00006961995082E000C990B0297029710F0AD
:10F20000133839F4BE01CE01DF91CF911F910C94D8
:10F21000157981E08887DF91CF911F910895FC01D6
:10F22000208520FD0C94E5780895CF92DF92EF922F
:10F23000FF920F931F93CF93DF93E0903316F090DC
:10F2400034160091351610913616F801E817F907B3
:10F2500039F0309709F44BC00190F081E02DF6CFE2
:10F26000009709F444C06B01EC018885882309F1FB
:10F2700018860115110561F00C171D0729F0AE0164
:10F2800067E8C8010E940F79F80100811181F1CF70
:10F29000EC81FD81309769F0CC15DD0551F0D093FC
:10F2A0003416C093331640E050E063E8CE01069672
:10F2B0001995E0913516F0913616CE17DF0741F417
:10F2C0008881998190933616809335160CC0FC0185
:10F2D000309749F080819181C817D907C1F788819B
:10F2E000998191838083F0923416E0923316DF91F6
:10F2F000CF911F910F91FF90EF90DF90CF900895E5
:10F300001F93CF93DF9310928F15C0913516D09134
:10F31000361611E0209779F08985882341F0188707
:10F32000198640E050E062E8CE010E94E57809903D
:10F33000D881C02DEFCFDF91CF911F91089580919B
:10F34000321691E0980F9093321608958AE88093D0
:10F350003216109230161092311610923616109204
:10F3600035161092341610923316089580918F1529
:10F3700081110E94807990913116992309F44EC031
:10F38000E09130162E2F30E085E0E89FF001112447
:10F39000E057FA4E608160938E15418152815093FF
:10F3A0008D1540938C150380F481E02D2F5F3F4F26
:10F3B0002F71332720933016915090933116309748
:10F3C00031F5809135169091361690938B15809378
:10F3D0008A1580918A1590918B15892BF9F080916F
:10F3E0008F1581110E94807940918C1550918D1557
:10F3F00060918E1580918A1590918B150E940F79DE
:10F40000E0918A15F0918B1580819181DECF613872
:10F4100011F481E08087CF010E940F7980918F15D0
:10F420002091311690E0820F911D08959C019091DA
:10F4300031169032A9F0E0913016E90FEF7185E0B6
:10F44000E89FF0011124E057FA4E60835283418314
:10F45000348323839F5F9093311680E090E008957A
:10F4600081E090E00895CF93DF93C0913316D0915F
:10F4700034160E940F79D0933416C0933316DF915F
:10F48000CF910895AB013091351620913616E32FB8
:10F49000F22FE817F907B1F0309721F00190F081D1
:10F4A000E02DF7CF009771F0FC013083218390931A
:10F4B00036168093351621E020871782168261E880
:10F4C0000C94337A0895009749F0FC01208521506F
:10F4D000223020F421E0218720938F1508950C9489
:10F4E000258580913716909138160097C1F01092BB
:10F4F000381610923716DC0114966D917C91159791
:10F500001296ED91FC9113971995E0913716F091B1
:10F510003816309721F0808191810C943F850895B1
:10F52000CF93DF93EC014C835D836E837F830E94D6
:10F53000046F688379838A839B83DF91CF910895D9
:10F54000FC01408151816281738184819581A68112
:10F55000B781840F951FA61FB71F80839183A28355
:10F56000B3830895CF93DF93EC010E94046F688307
:10F5700079838A839B83DF91CF910895CF92DF9225
:10F58000EF92FF92CF93DF93EC010E94046FC8804B
:10F59000D980EA80FB80DC01CB018C199D09AE0982
:10F5A000BF090196A11DB11D21E030E0CC80DD80B6
:10F5B000EE80FF80C816D906EA06FB0610F020E0B0
:10F5C00030E0C901DF91CF91FF90EF90DF90CF90B5
:10F5D0000895FC01118210820895FC0180819181BF
:10F5E0000895DC01ED91FC91309741F0808191818B
:10F5F000009711F0FC01FACFCF01089580E090E070
:10F600000895DC01ED91FC911197309721F0208154
:10F6100031812D933C93CF010895DC01ED91FC9154
:10F620003097A9F0A0E0B0E0208131816E177F070C
:10F6300041F4109709F4DC012D933C931182108260
:10F640000895DF012115310511F0F901EDCF08957D
:10F650000F931F93CF93DF938C01EB010E940D7BDF
:10F6600019821882C8010E94F17A009711F4F801FA
:10F6700001C0FC01D183C083DF91CF911F910F9115
:10F680000895DC01ED91FC9180E090E0309729F045
:10F6900001960190F081E02DF9CF0895009721F0B7
:10F6A000FC0180819181089580E090E008952F927F
:10F6B0003F924F925F926F927F928F929F92AF9202
:10F6C000BF92CF92DF92EF92FF920F931F93CF934F
:10F6D000DF93CDB7DEB768970FB6F894DEBF0FBEE5
:10F6E000CDBFE3EBF8E354A445A436A427A490A42B
:10F6F00081A472A463A4248D2983858D8A83B68C0A
:10F70000A78C908D9B83218D2C83828D8D83938DEF
:10F710009E8324892F83858988879689998727895D
:10F720002A8780898B8791899C8722892D87838965
:10F730008E8794859F872585288B8685898B9785DD
:10F740009A8B20852B8B81858C8B92859D8B238535
:10F750002E8BF480E580D680C78080818F8B91814D
:10F76000988F128103810E941E6F2F923F924F92B9
:10F770005F926F927F928F929F92AF92BF922A81F7
:10F780002F9329812F932E812F932D812F932C81BD
:10F790002F932B812F932A852F9329852F932885AB
:10F7A0002F932F812F932E852F932D852F932C858B
:10F7B0002F932B852F932A892F9329892F9328897B
:10F7C0002F932F852F932E892F932D892F932C895B
:10F7D0002F932B892F93CF92DF92EF92FF920F936B
:10F7E0001F93288D2F932F892F939F938F937F9310
:10F7F0006F93E1E4F9E381811F928F9380811F92DF
:10F800008F9386E694E19F938F930E94FB9C0FB6A3
:10F81000F894DEBF0FBECDBF68960FB6F894DEBF7A
:10F820000FBECDBFDF91CF911F910F91FF90EF9051
:10F83000DF90CF90BF90AF909F908F907F906F9010
:10F840005F904F903F902F900895CF93DF93EC01FE
:10F850004A815B8160E070E08C819D810E94319CD7
:10F86000288139818A819B81289FA001299F500D81
:10F87000389F500D112460E070E08E819F81DF91F0
:10F88000CF910C94319CFC018281938120E030E087
:10F8900028173907D1F0A481B581A20FB31F4C916D
:10F8A000411110C081E08C9380819181289FA0013B
:10F8B000299F500D389F500D112486819781840F08
:10F8C000951F08952F5F3F4FE3CF80E090E00895AC
:10F8D000FC01868197814281538120E030E024172A
:10F8E0003507D1F08617970781F4A481B581A20F5F
:10F8F000B31F8C91181614F481508C9384819581D8
:10F90000FC01E20FF31F80810895A081B1818A0F6D
:10F910009B1F2F5F3F4FE3CF8FEF0895FC012681A0
:10F92000378162177307A0F0A281B38140815181B2
:10F93000A49FC001A59F900DB49F900D1124280F86
:10F94000391F81E090E06217730720F080E008958E
:10F9500080E090E00895CF92DF92EF92FF920F93B4
:10F960001F93CF93DF937C018B016A0189E396E1BA
:10F970000E94ED7AEC01892B51F0EC81FD813097EA
:10F9800011F0C8011995CE010E944E7BF3CFA6015C
:10F99000B801C701DF91CF911F910F91FF90EF90B8
:10F9A000DF90CF900C948B7E0F931F93CF93DF93B8
:10F9B0000E94D77E8C0189E396E10E94ED7AEC01EA
:10F9C000892B49F0EA81FB81309709F01995CE0126
:10F9D0000E944E7BF4CF0115110539F0C801DF916B
:10F9E000CF911F910F910C947F7EDF91CF911F914A
:10F9F0000F910895CF92DF92EF92FF920F931F9392
:10FA00000E94BC7F0E94C7800E94977E0E94D57E84
:10FA1000C12C88E0D82E87E0E82EF12C00E01EE112
:10FA200020E030E040E052E060E070E082E090E012
:10FA30000E94297E1F910F91FF90EF90DF90CF9051
:10FA40000895CF93DF93EC010E94EA7E009761F066
:10FA50000E944A80E091240BF091250BBE018BEAB5
:10FA60009CE7199581E090E0DF91CF91089508958A
:10FA70000F931F93CF93DF93CAE7D6E14881598153
:10FA80006A817B8100E010E022E63DE78AE596E1AD
:10FA90000E9496780E94A270BC0180E090E02881CC
:10FAA00039814A815B810E94F891AB01BC0127E852
:10FAB0003DE786E496E10E949678DF91CF911F9111
:10FAC0000F91089580917A1690917B16A0917C16E3
:10FAD000B0917D1640917616509177166091781608
:10FAE00070917916880F991FAA1FBB1F48175907D5
:10FAF0006A077B0710F4DB01CA0180937A169093A2
:10FB00007B16A0937C16B0937D160C94387DCF9312
:10FB1000DF930E94C7800E943180EC011982188215
:10FB20000E94A07E28813981009719F1FC0140854F
:10FB30004423F9F0FC0142815381F901EE0FFF1FCC
:10FB4000EE0FFF1FEC0FFD1F53834283FC01448126
:10FB500055812F5F3F4FF901EE0FFF1FEE0FFF1F83
:10FB6000EC0FFD1F51834083398328830E944E7B15
:10FB7000D9CFC901880F991F880F991F02960E943B
:10FB80002C8088819981892B31F08BE396E1DF917C
:10FB9000CF910C94977FDF91CF910895AF92BF9250
:10FBA000CF92DF92EF92FF920F931F93CF93DF9349
:10FBB0001F921F92CDB7DEB75B010E9431808C018E
:10FBC000FC01E080F180FA82E9820E94798097014D
:10FBD000220F331F220F331F2E5F3F4F82179307D1
:10FBE00098F0C12CD12CCE14DF0471F0F8014481BF
:10FBF000558162817381C5010E94A47EFFEFCF1AF7
:10FC0000DF0A0C5F1F4FEFCF0F900F90DF91CF9166
:10FC10001F910F91FF90EF90DF90CF90BF90AF902A
:10FC200008950F93013099F480916E1690916F169C
:10FC3000A0917016B091711680937A1690937B16EE
:10FC4000A0937C16B0937D160F910C94387D0F9184
:10FC500008954F925F926F927F928F929F92AF9290
:10FC6000BF92CF92DF92EF92FF920F931F932A01E0
:10FC70003B01480159014AE05BE0BC018BE396E19E
:10FC80000E947A7FEBE3F6E143AA54AA65AA76AA1A
:10FC900087AA90AEA1AEB2AEC3AED4AEE5AEF6AE1C
:10FCA00081E19EE71F910F91FF90EF90DF90CF9041
:10FCB000BF90AF909F908F907F906F905F904F908C
:10FCC0000C949B7EEF92FF920F931F93CF93DF9341
:10FCD0008C01EB017A010E940E7FF801F086E78229
:10FCE0006EE07BE0CE01DF91CF911F910F91FF90ED
:10FCF000EF900C94327F0C94167F0C94217DDC01E4
:10FD00001796ED91FC9118970190F081E02D3097B6
:10FD100009F019940895DC011796ED91FC9118975C
:10FD20000280F381E02D309709F01994089582E85C
:10FD300096E10C94E97A9093811680938016089549
:10FD400082E896E10C94ED7AEF92FF920F931F9365
:10FD5000CF93DF938C01EB017A0182E896E10E9458
:10FD6000ED7A0097D9F0DC0112962D913C91139712
:10FD70002C173D0781F41696ED91FC91179730975B
:10FD800069F09701AE01B801DF91CF911F910F91FA
:10FD9000FF90EF9019940E944E7BE3CFDF91CF91BB
:10FDA0001F910F91FF90EF9008950C940A7FCF93CD
:10FDB000DF93E091600BF091610B1995EC01892BB9
:10FDC00029F06A817B8181E00E940F81CE01DF9161
:10FDD000CF9108950F931F93CF93DF93EC01E091A0
:10FDE000620BF091630B19958C016A817B8181E034
:10FDF0000E940F8181E090E0012B11F480E090E0FF
:10FE0000DF91CF911F910F910895E091640BF091D4
:10FE1000650B199484E896E10C94E97AFC017383EC
:10FE20006283BC0184E896E10C94287BBC0184E8E1
:10FE300096E10C940D7BCF93DF93EC0184E896E17F
:10FE40000E94ED7A009749F0FC01228133812C1742
:10FE50003D0729F00E944E7BF5CF80E090E0DF91D6
:10FE6000CF9108950F931F93CF93DF938B010E943F
:10FE70001B7FEC01892B31F01D830C83C8010E948C
:10FE8000057F8E83DF91CF911F910F910895DC0143
:10FE90001996ED91FC911A970280F381E02D30972D
:10FEA00009F0199408950F931F93CF93DF931F9236
:10FEB0001F92CDB7DEB78C0188E10E942D81BC0175
:10FEC000CE0101960E944781D8011996ED91FC91CF
:10FED0001A970190F081E02D309729F0BE016F5FF5
:10FEE0007F4FC80119950F900F90DF91CF911F910F
:10FEF0000F910895EF92FF920F931F93CF93DF938B
:10FF00008C01EB017A0140E15BE00E94627EF80126
:10FF1000F286E18664E17BE0CE01DF91CF911F9113
:10FF20000F91FF90EF900C94327F0C947B7ECF93D7
:10FF3000DF93EC0161E479E388E10E942381CE0143
:10FF4000DF91CF910C947D7EE0914C0BF0914D0BA5
:10FF50001994E091080BF091090B1994E091520B60
:10FF6000F091530B1994E091540BF091550B1994A7
:10FF700080E090E0089508958DEC92E00E94257C49
:10FF80008DED92E00E94257C85ED92E00C94257C1D
:10FF90000F931F93CF93DF93EC01BC018DED92E0A3
:10FFA0000E948E7C892BA9F00990D881C02DFE017A
:10FFB00061917191CF010E94DA80BE016E547F4F32
:10FFC000CE018E579F4FDF91CF911F910F910C94CF
:10FFD000FE80BE0185ED92E00E948E7C892BD1F0DF
:10FFE0000E94C780688179818A819B810E94DA8022
:10FFF0008CA990E00E948B800CA910E00E943880B0
:020000021000EC
:10000000BE016C5F7F4FA801DF91CF911F910F91CF
:100010000C94289CDF91CF911F910F91089520910E
:10002000991D30919A1D2817390798F04091971D16
:100030005091981D480F591F5093981D4093971D3C
:10004000281B390B30939A1D2093991D81E090E075
:10005000089580E090E0089590939A1D8093991DF3
:1000600008958091971D9091981D8C5E924E0895F1
:100070008091961D90E08C51934E089581E090E020
:100080002091E21C3091E31C24513D4111F480E0A9
:1000900090E008950E943E80892B61F06091E21CFF
:1000A0007091E31C4091991D50919A1D84E19DE14E
:1000B0000C94289C2091971D3091981D2115310595
:1000C000B9F08091991D90919A1DC096E4E1FDE1EF
:1000D000AF01445E5C414817590734F4DF01A20FB9
:1000E000B31F4C914193F4CF1092981D1092971D1D
:1000F00008958091991D90919A1D08958091961D63
:1001000090E3981B2091991D30919A1DA901490FE8
:10011000511DCA0108951F93CF93DF931091961D2F
:10012000212F30E02817390774F0EC010E947E80FF
:100130008C0F9D1F8138910530F41C1B1093961D68
:1001400081E090E002C080E090E0DF91CF911F91CC
:1001500008950F931F93CF93DF93E1E1F9E3119299
:10016000119289E3E134F807D1F7C9E0D9E301E15D
:1001700019E36EE27BE0CE010E94478122960C17C4
:100180001D07B9F7DF91CF911F910F91089510923C
:10019000981D1092971D10929A1D1092991D80E340
:1001A0008093961D84E19DE19093E31C8093E21C73
:1001B0000C94A980EF92FF920F931F93CF93DF933C
:1001C0008C017B010E94C780E701C138D10510F086
:1001D000C0E8D0E0AE01B8018091E21C9091E31C30
:1001E0000E94289CD0939A1DC093991DCE01DF9147
:1001F000CF911F910F91FF90EF900895FC0190E334
:10020000A1E1B9E301900D929A95E1F788E0FB0135
:10021000A9E0B9E301900D928A95E1F70895E82FDE
:10022000F0E0EE0FFF1FEF5EF64C7183608381E01C
:1002300090E00895E82FF0E0EE0FFF1FEF5EF64C20
:1002400080819181089590E0880F991F8752974C83
:100250000E94478181E090E0089590E0880F991F07
:100260008752974C0895E091D00AF091D10A1995E0
:10027000E0914A0BF0914B0B1995E091220BF09114
:10028000230B1995E091060BF091070B1994FB01D4
:1002900020813181FC0131832083089542E050E0C8
:1002A0000E941B9C21E030E0892B11F020E030E01F
:1002B000C9010895BC0181E499E30C94478182EB64
:1002C0009DE10E94E777892B21F082EB9DE10C9460
:1002D000DD770895E0919E1DF0919F1D309709F004
:1002E000199480E00895EF92FF920F931F93CF939C
:1002F000DF938C01EA01FC0180819181009741F03C
:100300008A33934081F1F8011182108283E0F8C0B2
:1003100080E024E0829FF0011124E056F24E118229
:1003200010828F5F8430A9F780939D1D80913316D2
:10033000909134169093B11D8093B01D0E949F79C7
:100340008093433940E450E060E070E082EB9DE14F
:100350000E94C9770E9407868AE393E0F80191839F
:10036000808381E0CDC06230D9F48091443990918E
:100370004539892B89F380915539863029F480914C
:100380006D3981FD0E945F8181E00E944E868091DF
:10039000443990914539892BF9F20E94CD82DCCF06
:1003A000633060F5611114C02097B1F2D093423AE6
:1003B000C093413A83E00E944E86809144399091E7
:1003C0004539892B11F00E946A810E945F81C4CF58
:1003D000613011F6209709F4BFCFD0933E3AC09315
:1003E0003D3A85E00E944E8680914439909145398E
:1003F000892B09F4B1CF0E946A81AECF673809F02A
:1004000040C010929C1D80EAE82E8DE1F82E80916C
:100410009C1D8430C0F4F70182819381C817D907ED
:1004200049F4808191810E943386F7011182108204
:1004300013821282F4E0EF0EF11C80919C1D8F5FFD
:1004400080939C1DE4CFE3E4FAE3848D958DC81777
:10045000D90719F4158E148E118EB0962AE3E33C59
:10046000F20799F7E9EDFAE381859285C817D90774
:1004700011F4158214823D968BE3EB35F807A1F752
:100480006BCF683809F068CFC25BDD4109F064CFFB
:1004900082EB9DE10E94E777892B09F45DCF1092F2
:1004A0009C1DE0919C1DE43008F056CF20E2E29FB5
:1004B000F0011124ED5BF54C818D8823D9F082EB9E
:1004C0009DE10E94DD7780919C1DE0E28E9FC0013E
:1004D00011248D5B954C9093423A8093413A82E08F
:1004E0000E944E868091443990914539892B11F0B4
:1004F0000E946A8180919C1D8F5F80939C1DD1CF4B
:10050000DF91CF911F910F91FF90EF900895CF93BE
:10051000DF93A091413AB091423A109719F0ED0162
:100520006C9605C0C0913D3AD0913E3A2996809193
:100530003C3A86FF23C010929B1D80E0E0EAFDE17B
:100540008430C1F04081518114962D913C911597D2
:100550004217530761F4228133812115310539F0A7
:1005600080939B1D398328831B821A8205C0349691
:100570008F5FE6CF80939B1D0E945F818881998168
:10058000009741F04A815B8160914339DF91CF91BF
:100590000C94337ADF91CF9108950F931F93CF93EB
:1005A000DF9380915539863009F07AC080914439C3
:1005B00090914539803F910508F472C08897EC010D
:1005C000D695C7959E01220F331F8E012817390734
:1005D00010F40F5F1F4FCE0188969093453980939A
:1005E000443990934E3980934F391092713910925B
:1005F00070390E940186809590959093713980930F
:10060000703910925739109256390E94F0858095B2
:10061000909590935739809356390E946A81C8010A
:100620008896909345398093443990934E398093BE
:100630004F3980913F3A9091403ABC016C0F7D1F39
:10064000A8010E94289CBE0184E699E30E949D8532
:100650008091483980936439809149398093653914
:1006600080914A398093663980914B3980936739FC
:1006700010927139109270390E9401868095909580
:10068000909371398093703910925739109256397E
:100690000E94F085809590959093573980935639B4
:1006A000DF91CF911F910F910C946A81E091E00A44
:1006B000F091E10A199480E090E00895AF92BF9222
:1006C000CF92DF92EF92FF920F931F93CF93DF931E
:1006D000CDB7DEB7E1970FB6F894DEBF0FBECDBF42
:1006E0007C016B01CE0101965C0181E3F501119261
:1006F0008A95E9F781E089838CE00E941A818C83D6
:100700001D821F828091BE1D91E0980F9093BE1DA7
:10071000898713E018878DEC9BEA9B878A8789E19C
:100720000E942D816EE27BE00E944E81892B31F088
:1007300082E08E838FEF8C878D8709C089E10E94CC
:100740002D81BC01CE010C960E9447811E838DEC49
:100750009BEA9D8B8C8B61E479E3CE0146960E94E7
:1007600047810E9431809FA78EA70E94798099AB14
:1007700088ABC5010E94D88F8C011127C8010E9447
:100780008B80892B31F10E943880A801BC01C50102
:100790000E94FB8F0091D60A1091D70A0E947E809A
:1007A0005C010E943880B501F8011995E114F1044B
:1007B00081F0009739F0019761F441E050E064E086
:1007C00070E004C041E050E060E070E0C601F70175
:1007D0001995E1960FB6F894DEBF0FBECDBFDF913D
:1007E000CF911F910F91FF90EF90DF90CF90BF902E
:1007F000AF9008950F931F93CF93DF934115510549
:1008000079F0FA018B01EC01828193810E94C87F0B
:10081000B801CE01DF91CF911F910F910C945E83AF
:10082000DF91CF911F910F910895EF92FF920F9357
:100830001F93CF93DF93CDB7DEB7E1970FB6F89450
:10084000DEBF0FBECDBF0E9479807C010E94318047
:100850008E010F5F1F4FA801B7010E94EA90892BFC
:1008600009F441C088A999A99701281B390BC9012E
:100870000E940F80892BB9F18E8181110CC0BE01BD
:100880006A5E7F4F88E10E942381E091260BF09100
:10089000270B199528C02A853B852D3C9BEA3907F3
:1008A00019F02F3F3F4FF9F4823019F0E8E0F0E003
:1008B00002C0E2E0F0E0E00FF11FE017F107F9F20B
:1008C000319783858F3FC9F3BE01645F7F4F89E114
:1008D0000E94238189E10E942D8161E479E30E94D5
:1008E0004E81892B61F6E1960FB6F894DEBF0FBEFC
:1008F000CDBFDF91CF911F910F91FF90EF900895A1
:100900000E94A2708093BE1DE091E00AF091E10A7E
:100910001994892B29F0E091E00AF091E10A04C0D2
:10092000E091E20AF091E30A1994FC01680F791F43
:1009300080E048E1E617F70781F0219198E0382F31
:100940003227532F517030FD84278695513009F49A
:1009500080682695915099F7EDCF08951F920F92D8
:100960000FB60F9211240BB60F922F933F934F9314
:100970005F936F937F938F939F93AF93BF93EF9307
:10098000FF9380919400909195009093F638809316
:10099000F53881E08093E73880917100807D809305
:1009A00071000E94717A8091E7388823D9F1809193
:1009B0009400909195004091F5385091F638841745
:1009C0009507A0F48091BB389091BC38A091BD38B8
:1009D000B091BE38875F924CAF4FBF4F8093BB380A
:1009E0009093BC38A093BD38B093BE38209194004A
:1009F00030919500241B350B8091BB389091BC3809
:100A0000A091BD38B091BE38820F931FA11DB11DBA
:100A10008093BB389093BC38A093BD38B093BE3858
:100A20001092E738FF91EF91BF91AF919F918F9115
:100A30007F916F915F914F913F912F910F900BBEDE
:100A40000F900FBE0F901F9018959FB7F894E1E795
:100A5000F0E08081807D808388B38F6288BB1092B4
:100A60009000E1E9F0E0108210929200109295005F
:100A7000109294008081856080839FBF08959C01BF
:100A80009FB7F894309399002093980088B38F62B1
:100A900088BBE1E7F0E08081826080839FBF08959A
:100AA000FB0141505109460F571FE417F50778F431
:100AB000208130E0322F22276181260F311D820FE5
:100AC000931F8217930708F401963296EECFE4172E
:100AD000F50751F4208130E0322F2227820F931F37
:100AE0008217930708F401960895CF93DF93C0917E
:100AF0004E39D0E0DC2FCC2720914F3930E0245103
:100B00003109C20FD31F48E050E068E579E39E0148
:100B1000280F311DC9010E945085AE0160E679E3BE
:100B20000E945085009721F098278927982702C0B6
:100B30008FEF9FEFDF91CF910895FC012381260F66
:100B400020934B39A72FBB2792819A0F90934A3954
:100B5000318130934939408140934839E92FF0E0A1
:100B6000EA17FB0748F481E0830F8093493981112C
:100B700003C04F5F4093483930E077272617370787
:100B800088F49F5F90934A3991110CC08091493944
:100B90008F5F80934939811105C0809148398F5FFB
:100BA0008093483908952091413A3091423ABC01EE
:100BB000C90108960E949D85E091413AF091423A20
:100BC000A8E4B9E38C91808711968C911197818765
:100BD00012968C911297828713968C918387089531
:100BE00044E150E06CE479E380E090E00E945085BD
:100BF000009721F098278927982708958FEF9FEF76
:100C0000089586E00C94758581E10C94758580E0EB
:100C1000E82FF0E0EE0FFF1FED53F54C118210822C
:100C20008F5F8430A9F780E090E2899FF001112462
:100C3000ED5BF54C118E8F5F8430B1F780E094E06E
:100C40009093C31D8093C21D80E09DE0989FF001AA
:100C50001124E752F54C158214828F5F8A30B1F768
:100C60008093C11D08959C0190E09430A1F0E92F7C
:100C7000F0E081E0890FEE0FFF1FED53F54C40814E
:100C800051814217530729F49093C11D118210829C
:100C90000895982FEACF9093C11D0895AF92BF9207
:100CA000CF92DF92EF92FF920F931F93CF93DF9338
:100CB000843009F4DFC1C091413AD091423A24E72F
:100CC00039E33093403A20933F3A309347392093A9
:100CD0004639833059F4898D8F70833009F06AC0AA
:100CE00088899989892B09F0BFC67EC0823009F0B6
:100CF0007FC08091C71D8F5F8093C71D811113C076
:100D00008091C61D8F5F8093C61D81110CC080919C
:100D1000C51D8F5F8093C51D811105C08091C41DC5
:100D20008F5F8093C41D1092453910924439109200
:100D3000D83A1092D73A898D982F9D7F953041F4FB
:100D40008A8D8F5F8A8F843109F08EC6198E8CC68A
:100D5000882309F489C628893989232B09F440C0DE
:100D60009A8D2FEF290F2A8F91117EC69B8D983077
:100D700031F02FEF280F223048F4953039F4198ED6
:100D800080E880933C3A0E94878228C5953038F4E9
:100D900023E0092E01C0220F0A94EAF701C020E3E4
:100DA0002A8F9F5F9B8F8F708330A1F048F4813032
:100DB00009F43AC3823009F057C610926D3937C32F
:100DC000863009F4A8C4883009F4A5C4843009F039
:100DD0004BC6A1C484E080933C3A0E94878230C510
:100DE0008F70833009F040C688E080933C3AEBC4B2
:100DF000853019F5E0913D3AF0913E3A8481958134
:100E0000892B09F431C61092423A1092413A88E691
:100E100099E39093403A80933F3A90934739809377
:100E200046391092D83A1092D73A1092453910921A
:100E3000443988E080933C3A1BC180914C39853419
:100E400009F012C600914E3910E0102F0027809152
:100E50004F39080F111D8091443990914539801701
:100E6000910708F401C610934539009344398091E5
:100E700052398F7309F0F8C5F0905339F110F4C569
:100E80008091D33A9091D43AC091580BD091590B9C
:100E90008C179D0759F44091D53A5091D63A20913C
:100EA0005A0B30915B0B42175307A1F020915C392C
:100EB00030915D398217930709F0D6C520915E39CC
:100EC00030915F398091D53A9091D63A28173907F9
:100ED00009F0CAC50E94F085019609F0C5C5809148
:100EE0005539863009F429C18131E9F1813009F0A1
:100EF000BBC580916039883009F0B6C51092603961
:100F00008091623990916339873F6FEF960710F0B7
:100F1000099601C008969093633980936239809155
:100F2000583990915939A0915A39B0915B398093D1
:100F30005C3990935D39A0935E39B0935F398091AD
:100F4000D33A9091D43AA091D53AB091D63A8093C1
:100F5000583990935939A0935A39B0935B3980E44A
:100F6000809354395EC50C51110910934539009393
:100F7000443988E699E39093403A80933F3A8091D0
:100F8000663990916739892B29F00E940486019671
:100F900009F06AC520916239309163392115310514
:100FA00009F462C589ED9AE390933E3A80933D3A05
:100FB000A0906039B0906139E0905A0BF0905B0BD3
:100FC00040915C0B50915D0BA0915839B09159390B
:100FD00000915A3910915B3960915E0B70915F0BF3
:100FE000E0913D3AF0913E3A8BE3EB35F80708F09B
:100FF0003BC584819581009721F12817390709F5B0
:1010000086819781009719F08A159B05D1F480811C
:101010009181C817D90729F4C280D380CE14DF0488
:10102000B1F08417950729F4C280D380C616D7067D
:1010300071F08A179B0729F4828193810817190799
:1010400031F03D96F0933E3AE0933D3AC9CF10928D
:10105000423A1092413A82E080933C3A88E699E322
:1010600090934739809346391092D83A1092D73AE4
:101070000E9487828091D73A9091D83A009709F4DC
:10108000F3C49C01245E3F4F30934539209344398B
:1010900030934E3920934F39E0913D3AF0913E3AEA
:1010A00020852093543921E12093553908969827BB
:1010B000892798279093653980936439109267390E
:1010C000109266398481958190936139809360395B
:1010D0008681978190936339809362398091D33A66
:1010E0009091D43AA091D53AB091D63A809358399C
:1010F00090935939A0935A39B0935B39808191818B
:10110000A281B38180935C3990935D39A0935E395D
:10111000B0935F3984E799E39093403A80933F3AE4
:101120000E94048680959095009711F48FEF9FEFB1
:10113000909367398093663974C40E940186019642
:1011400009F092C4409162395091633941155105BB
:1011500009F48AC48091603990916139009709F44B
:1011600083C46091583970915939E0915A39F0919E
:101170005B39C3E4DAE3298D2223A9F0AC81BD8178
:101180004A175B0781F4AE81BF818A179B0759F428
:10119000A881B9816A177B0731F4AA81BB81EA175C
:1011A000FB0709F45CC1A0962AE3C33CD20719F7F8
:1011B00080916D398F738230D9F45093C01D409364
:1011C000BF1D80E0843091F0E82FF0E0EE0FFF1FAC
:1011D000ED53F54C208131818F5F4217530791F712
:1011E0001092C11D80E0C0E0D0E07CC08093C11DA2
:1011F00080916D3982FD38C484E180936D3988E235
:1012000090E0909345398093443980E580936C3920
:101210003091673980916B398093673920916639B5
:1012200080916A398093663920936A399091653943
:1012300080916939809365399093693980916439D7
:101240008093C11D40916839409364398093683917
:101250003F5F30936B3931110DC02F5F20936A3996
:10126000211108C09F5F90936939911103C08F5F6E
:101270008093683980916039909161399093C01D55
:101280008093BF1D20916239309163393093613969
:1012900020936039909363398093623980915839F3
:1012A00090915939A0915A39B0915B3980935C394A
:1012B00090935D39A0935E39B0935F398091D33AB2
:1012C0009091D43AA091D53AB091D63A80935839BA
:1012D00090935939A0935A39B0935B3987C39730AB
:1012E00089F08F5F8430C1F060E2869F9001112405
:1012F000F901ED5BF54C918D9111F1CF8093C11DFA
:10130000EF010FC0209721F0428D9A8D941748F776
:10131000E901CD5BD54CE5CF8093C11D209709F441
:10132000A3C3D093423AC093413A83E08A8F888F17
:101330001E8A84E08F8B1B8E809162399091633975
:101340009D838C8380916039909161399F838E83D6
:101350008091583990915939A0915A39B0915B399F
:1013600088839983AA83BB8381E0898F8091C41D80
:101370008C878091C51D8D878091C61D8E87809139
:10138000C71D8F8781E090E0998B888B80916739AA
:101390008B87809166398A878091653989878091AA
:1013A0006439888781E090E00E94D38580916C3910
:1013B000982F907F9135C0F182958F7090E00597BE
:1013C000880F991F880F991FEF2DF0E0E817F90794
:1013D0004CF5E45BF64C20A5222321F1213011F4D9
:1013E000F394F2CF2230C9F421A52430B1F4F09265
:1013F000C11D82A590E0982F882723A5822B90936A
:10140000C01D8093BF1D893C910510F088EC90E0D1
:101410009B8B8A8B9D8B8C8B07C021A5222311F07F
:10142000F20ED2CFF092C11D80E180936D39809190
:101430006D39826080936D3982E08093743984E0E5
:10144000809375391092763988EC809377398CE2E5
:1014500090E0909345398093443980E675C2D093EB
:10146000423AC093413A10923C3A80916D39782FBC
:101470007470F72E82FF03C0198E80E20EC2909125
:101480006C3992959F70990F990F9093C11D091B0C
:101490001109045111091093453900934439922FD1
:1014A0009F70923029F4982F9F73923139F41FC0A6
:1014B000913021F4982F9F739230C9F0012B19F4C9
:1014C000982F9370A1F0209164399885291332C226
:1014D00020916539998529132DC2209166399A8505
:1014E000291328C2209167399B85291323C284FFC1
:1014F00049C0688979896115710509F443C0CE0135
:101500000C960E949D853091683980914839381336
:1015100039C02091693980914939281333C090919D
:101520006A3980914A3998132DC080916B39409166
:101530004B39841327C03C872D879E878F878B8DDF
:10154000811119C09E89888D2A8D821B292F26958D
:1015500026952695821B980F9E8B87FD81952F8956
:10156000322F36953695231B820F8F8B9695969545
:101570009695890F888F81E080933C3A888D8A8F79
:10158000198A188A298DE22FEF708E2F90E0FC01C6
:101590003197E830F10508F067C28827E656FF4F1B
:1015A0008F4F0C94399280913C3A80FF14C083E0B5
:1015B000898F80E480933C3A198A188A8091443953
:1015C00090914539009709F4FAC022E420933C3AFF
:1015D0000E94D385F4C080916D398F73823009F0F9
:1015E00043C222CF80913C3A80FF60C080916D3928
:1015F0008F73823109F05AC080916C39982F907F97
:101600009135C0F182958F7090E00597880F991FF2
:10161000880F991FEF2DF0E0E817F9074CF5E45B10
:10162000F64C20A5222321F1213011F4F394F2CFBE
:101630002230C9F421A52430B1F4F092C11D82A555
:1016400090E0982F882723A5822B9093C01D80932C
:10165000BF1D893C910510F088EC90E09B8B8A8B34
:101660009D8B8C8B07C021A5222311F0F20ED2CFC7
:10167000F092C11D83E0898F8091643988878091C1
:1016800065398987809166398A87809167398B8728
:1016900081E090E00E94D38582E480933C3A198AED
:1016A000188A109245391092443989C080E280939B
:1016B0003C3A0E948782E091413AF091423A118E81
:1016C00097CD80916D3980FF28C024FD26C0888980
:1016D0009989892B09F0C8C1809144399091453985
:1016E00001960E94D38580913C3A982F9061909307
:1016F0003C3A2091443930914539232B19F08261CD
:1017000080933C3A0E94878281E090E0998B888B9D
:1017100088E0898F1B8E81E10EC185FF1CC08091FE
:1017200072399091733998278927982740913F3AC9
:101730005091403A480F591F5093403A40933F3AD6
:101740004091443950914539BA01681B790B709327
:101750004539609344394091443950914539411598
:10176000510551F024FD08C090913C3A926090934D
:101770003C3ACA010E94D38580916E3990E0982F3F
:10178000882720916F39820F911D9093C01D8093FF
:10179000BF1D2C893D892817390710F0892B21F4AA
:1017A0003093C01D2093BF1D8091BF1D9091C01D1F
:1017B0009B8B8A8B80913C3A837009F455C11092BF
:1017C000D83A1092D73A0E94878280913C3A85FF9E
:1017D00007C01092D83A1092D73A198E84E1ABC064
:1017E00084FF0AC01092D83A1092D73A81E090E074
:1017F000998B888B84E08DCF2091D73A3091D83A5D
:1018000021153105E1F080FF02C0198A188A888904
:101810009989009781F48A899B898217930720F41C
:101820009093D83A8093D73A8091D73A9091D83A0A
:10183000998B888B04C09093D83A8093D73A1B8EAB
:1018400080914639909147399093403A80933F3A3E
:101850008091D73A9091D83A892B59F08889998903
:10186000009739F08896909345398093443988E100
:101870000BC080913C3A81FFF7C088E290E09093E2
:1018800045398093443980E180936D395CC0809103
:101890003C3A80FFE9C0198E80E180933C3A0E9477
:1018A0008782E2C08091443990914539009711F0C8
:1018B0000E94D38590916D3980913C3A90FF0BC086
:1018C00080FF06C087E0898F1A8E198A188A19C08E
:1018D00086E0898F16C080FF1EC085E0898F198A37
:1018E000188AC2C08091443990914539009711F00F
:1018F0000E94D38580916D3980FF0DC087E0898F6C
:101900001A8E81E090E00E94D38580E180933C3A7A
:101910000E9487820FC08091443990914539892B6C
:1019200049F4A2C080913C3A80FF9EC087E0898F35
:101930001A8E9AC080E180936D3988E290E090938E
:1019400045398093443980E580936C39888580934C
:1019500068398985809369398A8580936A398B854E
:1019600080936B398C85809364398D85809365393C
:101970008E85809366398F858093673986E0809362
:1019800055398C819D8190936139809360398E8126
:101990009F8190936339809362398091D33A90917B
:1019A000D43AA091D53AB091D63A809358399093D1
:1019B0005939A0935A39B0935B3988819981AA81AA
:1019C000BB8180935C3990935D39A0935E39B0936D
:1019D0005F39898D84FF05C010926F3910926E397E
:1019E00005C010926E3988EC80936F3980E4809343
:1019F0005439809144399091453990934E39809370
:101A00004F391092733910927239109271391092C5
:101A100070390E94018680959095909371398093DA
:101A2000703985E480934C3910924D3910925339B6
:101A3000109252398091C81D9091C91D01969093C2
:101A4000C91D8093C81D90935039809351391092CD
:101A50005739109256390E94F08580959095909351
:101A600057398093563904C0109245391092443941
:101A700010923C3ADF91CF911F910F91FF90EF9020
:101A8000DF90CF90BF90AF900895FC0180E090E090
:101A90002081222329F02181820F911D3296F8CFD7
:101AA0000895EF92FF920F931F93CF93DF937A01E4
:101AB0002830310514F5DB014D915C915427452701
:101AC000542702C0440F551FEA94E2F7452F5527CB
:101AD000F901EA59F44FC081D0E04C235D2368E05E
:101AE00070E0EB01C21BD30BFA0102C0F695E7953B
:101AF000CA95E2F7DC01EC9376C0D90153E0B595C5
:101B0000A7955A95E1F7E114F10431F0AB01FC011E
:101B10008C010A0F1B1F2FC0FB01AC017B01EA0ED9
:101B2000FB1EEE16FF0629F06191EA016993AE01F2
:101B3000F8CF8901077011270115110509F453C069
:101B4000FC01EA0FFB1FD7012C9130E0D801AA5904
:101B5000B44F9C91492F50E042235323C8E0D0E07A
:101B60009E01201B310BEA0102C0D695C7952A952C
:101B7000E2F7C08338C0E017F10781F0EA018881FD
:101B800099819827892798270E2C02C0880F991FC2
:101B90000A94E2F791934F5F5F4FEDCF27703327A1
:101BA0002115310501F1A60FB71F8D919C91982742
:101BB0008927982702C0880F991FEA94E2F7892F96
:101BC0009927D901AA59B44F4C9150E08423952309
:101BD00048E050E0BA01621B730B02C096958795EE
:101BE0006A95E2F78083DF91CF911F910F91FF906B
:101BF000EF9008958F929F92AF92BF92CF92DF9213
:101C0000EF92FF920F931F93CF93DF931F921F9238
